:020000040800F2
:1080000000800120B17101087F130108811301086C
:10801000831301088513010887130108000000007D
:1080200000000000000000000000000089130108AB
:108030008B130108000000008D130108DD8100088A
:10804000F5710108F5710108F5710108F571010874
:10805000F5710108F5710108F5710108F571010864
:10806000F5710108F5710108F5710108F571010854
:10807000F5710108F5710108F5710108F571010844
:10808000F5710108F5710108F5710108F571010834
:10809000F5710108F5710108F5710108318E0008CC
:1080A000F5710108F5710108F5710108F571010814
:1080B000A1F10008F5710108F5710108F5710108D9
:1080C000F5710108F5710108F571010825F1000845
:1080D000F5710108F5710108F5710108F5710108E4
:1080E000F5710108F5710108F5710108F5710108D4
:1080F000F5710108F5710108DDFF0008F57101084F
:10810000F5710108F5710108F5710108F5710108B3
:10811000F5710108F5710108F5710108F5710108A3
:10812000F5710108F5710108F5710108F571010893
:10813000F5710108F5710108F5710108F571010883
:10814000F5710108F5710108F571010871A50008C4
:10815000F5710108F5710108F5710108F571010863
:10816000F5710108F5710108F5710108F571010853
:10817000F5710108F5710108F5710108F571010843
:04818000F57101088C
:1081880010B5054C237833B9044810B10448AFF34F
:1081980000800121217010BD0806002000000000A9
:1081A800D492010808B5064B1BB106480649AFF33F
:1081B80000800648016811B1054B03B1984708BD16
:1081C80000000000D49201080C06002004060020DC
:1081D80000000000684620F007018D4601B5094BF4
:1081E8001A7842B15A6801325A60074A1168013157
:1081F8001160002200E001221A70BDE801408546A6
:10820800704700BF2406002098530020074B41F612
:108218004B525A60064AF02182F8231000229A60D5
:108228006FF0040007221A600AF0F2BF10E000E0C5
:1082380000ED00E0014B5868704700BF240600209D
:108248002DE9F341714F012001460024022509F070
:108258003BFF092338466946012600938DF8044000
:108268008DF806408DF805508DF8074009F074FD2B
:1082780048F216033846694600938DF804608DF875
:1082880006408DF805508DF8074009F065FD48F265
:1082980017033B8338464FF48073694600938DF883
:1082A80004508DF806408DF805508DF8074009F008
:1082B80053FD21464FF4800009F05CFE07F5806706
:1082C8002846314609F000FF40F6FC7338466946F7
:1082D80000934FF480588DF804408DF806408DF8CF
:1082E80005508DF8074009F037FD38466946CDF846
:1082F80000808DF804608DF806408DF805508DF8E3
:10830800074009F029FDA7F81A80042007F58067BF
:10831800314609F0D9FE4AF2C2333846694600931D
:1083280044F204088DF804408DF806408DF8055095
:108338008DF8074009F010FD38466946CDF80080F1
:108348008DF804608DF806408DF805508DF80740CB
:1083580009F002FDA7F81880DFF8B8800820314638
:1083680009F0B2FE4FF68C73404669460093102719
:108378008DF804408DF806408DF805508DF80740BB
:1083880009F0EAFC4046694600978DF804608DF8CC
:1083980006408DF805508DF8074009F0DDFCA8F877
:1083A8001A7038461A4F314609F08EFE4FF6FF73A1
:1083B8003846694600938DF804608DF806408DF8BC
:1083C80005508DF8074009F0C7FC4FF610737B8302
:1083D800EF233B834FF0080838466946CDF8008004
:1083E8008DF804608DF806608DF805508DF807400B
:1083F80009F0B2FCA7F81A8000BF00BF00BF00BF99
:1084080000BFA7F81880BDE8FC8100BF000002404B
:1084180000100240000C0240C90801F0F7BD07280F
:1084280020D8DFE800F004070A0D1013161B4FF4DC
:10843800807210E04FF400720DE04FF480620AE0A1
:108448004FF4006207E04FF4805204E04FF400520A
:1084580001E04FF48042044B5A837047024B4FF4BB
:1084680000425A83704700BF00100240072820D8F6
:10847800DFE800F004070A0D1013161B4FF4807292
:1084880010E04FF400720DE04FF480620AE04FF400
:10849800006207E04FF4805204E04FF4005201E01C
:1084A8004FF48042034B1A837047024B4FF400424B
:1084B8001A8370470010024038B50546002445FA73
:1084C80004F3DB07E0B202D5FFF7D0FF01E0FFF7C6
:1084D800A6FF0134082CF2D138BD08B507282ED8DC
:1084E800DFE800F004060B10151E232800200FE01B
:1084F800144B1869C0F3802008BD124B1869C0F3EB
:10850800C02008BD0F4B1869C0F3003008BD01201A
:1085180000F0FAFEB0F5006F34BF0020012008BD5E
:10852800084B1869C0F3403008BD064B1869C0F302
:10853800803008BD034B1869C0F3C03008BD002067
:1085480008BD00BF000C024007282DD8DFE800F066
:1085580004090E13181D2227144B5869C0F3002074
:108568007047124B5869C0F3402070470F4B586949
:10857800C0F3802070470D4B5869C0F3C020704786
:108588000A4B5869C0F300307047084B5869C0F36C
:1085980040307047054B5869C0F380307047034B33
:1085A8005869C0F3C030704700207047001002407F
:1085B80010B50020FFF7C8FF041C18BF01240120D4
:1085C800FFF7C2FF10B144F00204E4B20220FFF743
:1085D800BBFF08B144F004040320FFF7B5FF08B15E
:1085E80044F008040420FFF7AFFF08B144F010047A
:1085F8000520FFF7A9FF08B144F020040620FFF783
:10860800A3FF08B144F040040720FFF79DFF08B11D
:1086180044F08004204610BD034B202208B15A8341
:1086280070471A83704700BF00100240082008B541
:1086380000F06AFE592805D9074B1A7852B9012269
:108648001A7008BD082000F05FFE542802D8024BBB
:1086580000221A7008BD00BF2C060020044B1878B1
:108668000138C0B201288CBF00200120704700BF2C
:108678002C060020044B1878012802D102221A7017
:1086880070470020704700BF2C06002020B9034B1C
:108698001869C0F34020704700207047000402406A
:1086A80008B580B9094B1A78094B186822B95B6874
:1086B800000C40EA034008BD596842F210720023DA
:1086C8000DF03EFA08BD002008BD00BF514C002047
:1086D800904C002010B508BB72B6114B0A461878AA
:1086E800CB171049C1E9002330B908684C68020467
:1086F800230443EA104307E00A6842F21070A2FB21
:1087080000234C6800FB0433C1E90023064A002318
:108718001360064A1360064A536262B610BD00BF72
:10872800514C0020904C00206C4C0020BC4C002088
:1087380000040140024B1869C0F30020704700BFD5
:108748000008024010B598B90A4A0B4B1278196014
:108758000A4C186832B10DF009F809490DF00EF904
:10876800206010BD0DF002F806490DF007F92060F1
:1087780010BD00BF514C0020884C00204C4C0020FC
:1087880000401C4600FF7F47164B70B553F8206029
:10879800154B360253F82030144C96FBF3F203FBCA
:1087A8001266350495FBF3F103FB115555B1012110
:1087B800215442F2107404FB06F191FBF3F104FB1F
:1087C800021102E001EB02412554094B21F07F44DC
:1087D80003EB40131A6902F07F4222431A61BDE895
:1087E8007040AFE7444C0020404C0020514C002022
:1087F8009C4C002038B5044600282FD101F04403D2
:10880800042B1F4B9A680BD1C80602D542F480721C
:1088180008E022F480729A60DA6842F4807205E017
:1088280022F480729A60DA6822F48072DA60154B5A
:10883800C1F3C0021A70144B01F001021A7011F052
:108848004002124B01F0040103D001221A7029B131
:1088580002E01A7011B101220D4B1A700D4B0E4D2A
:108868001A5D0E4B18681AB10CF080FF0C4902E033
:108878000CF07CFF0B490DF081F845F8240038BD59
:10888800003C0140504C0020484C0020544C002033
:10889800524C0020514C00204C4C0020884C0020A9
:1088A80000401C4600FF7F472DE9F041594D8CB030
:1088B8000024C0230226284607A907938DF82060C4
:1088C8008DF821608DF822408DF8234009F044FA94
:1088D80028460621032209F0C2FA03222846072166
:1088E800A5F5823509F0BBFA0121304609F01CFCD8
:1088F800284609F0E7FE01A809F0CCFF4FF6FF78FB
:10890800284601A9ADF80440CDF80880ADF80C4020
:10891800ADF8064009F080FF224623460321284689
:108928000AF0F4FB04A80AF02FFA284604A9ADF8C7
:1089380018400AF09DFA284604A9ADF810400AF03C
:1089480097FA04A80AF020FA284604A9ADF81840B6
:108958000AF08EFA0423284604A9ADF810300AF06C
:1089680087FA284641F65F610AF02DFB2846012167
:108978006C6209F0E6FF0821304609F03FFE4FF42B
:1089880080730125099309A808238DF829308DF8EB
:1089980028408DF82A5009F005F91F4B1F4E9A6898
:1089A8000BA822F480729A60DA68274622F4807253
:1089B800DA6017238DF82C3007238DF82D308DF8C9
:1089C8002E408DF82F500AF0D9FB3169204621F04E
:1089D8007F41FFF7B7FEF17C2046FFF70BFF104BF6
:1089E800C8221A600F4B4FF400421A602046FFF766
:1089F800CBFE0D4B20221A700C4B10221A700C4B18
:108A080006221A700B4BC3F800800B4B1D700CB07C
:108A1800BDE8F08100080240003C01409C4C002069
:108A2800444C0020404C00205C4C0020494C002065
:108A3800554C0020584C0020534C00200C4B1A6910
:108A480012F0040F1A690CBF08200020110703D484
:108A5800002814BF0C2004201B691A06044B58BFB9
:108A680040F002001B69DB0558BF40F00100704769
:108A7800000C0240034B08B1034A00E0034ADA60E5
:108A8800704700BF00ED00E00400FA050100FA0598
:108A98000C4900234FF0FF3203F1200041F8202059
:108AA80003F160000133082B41F82020F4D10023A2
:108AB8001946044A9A180133F02B82F80013F8D1AA
:108AC800704700BF00E100E038B53C484FF48052E1
:108AD800038800219BB243F020030380038823F01E
:108AE80010031B041B0C0380354B1A8309F016FD79
:108AF8003248012109F048FD0028F9D02F4809F033
:108B08000AFD304B05461B780446082B0FD92B4825
:108B1800002109F003FD2948012109F035FD00284D
:108B2800F9D0264809F0F7FC2D0240EA0504254B48
:108B38001B78102B0ED92148002109F0EFFC1F48A3
:108B4800012109F021FD0028F9D01C4809F0E3FCB7
:108B5800240204431B4B1B78182B0ED917480021FD
:108B680009F0DCFC1548012109F00EFD0028F9D0B8
:108B7800124809F0D0FC24020443114B4FF48052F0
:108B88005A830E4A13889BB243F01003138013884C
:108B980023F020031B041B0C13800B4B18780B4B82
:108BA80024FA00F41A780A4B186820402AB10346C0
:108BB80000E058405B10FCD138BD38BD003800409B
:108BC800000402405C4C0020554C0020534C00200F
:108BD800584C0020F8B55E4B5E4C1B78002B66D0D5
:108BE800FFF772FF5C49206022680B689A4222688E
:108BF8000B6821DD594ED21A73689A420ADA58482E
:108C080005682A4645682B4625680968554C691A3F
:108C1800246845E0544D2B78002B29D1504805682D
:108C28002A46456809682B462768B5684D4C0135C2
:108C3800C91B2468691813E09A4280F287800A6881
:108C4800464E2368D21A73689A420EDA4448056879
:108C58002A4645682B460D682168424C691A2468E3
:108C68006143521A63EBE1731EE03F4D2B7843B129
:108C78000020FFF715FD3D4B4042186000232B7084
:108C8800F8BD374805682A464568D4F800C02B4621
:108C98000F68B568334901350C68C7EB0C016918D2
:108CA8006143521843EBE173C0E90023F8BD304B30
:108CB8001A78304B5B6A0AB1C3F580332360254AC2
:108CC800254B1068196888421068196816DD411A22
:108CD800B1F5004F2249086804464868054605DA98
:108CE80010681B681F4AC31A126825E018681368C1
:108CF8001C4AC31A126803F5803311E0884221DA4E
:108D080018681168411AB1F5004F154908680446FA
:108D18004868054609DA18681368124AC31A1268BF
:108D28005343E41A65EBE3750AE010681B680D4AC3
:108D3800C31A126803F580335343E41845EBE3750F
:108D4800C1E90045034B1A68034B1A60F8BD00BF20
:108D5800544C00206C4C0020BC4C00202C060020F9
:108D6800904C0020884C0020524C002008590020CC
:108D7800484C002000040140C2B2194B072A1A705F
:108D880001D808220AE00F2A01D8102206E0172A83
:108D980001D8182202E01F2A01D820221A70114B8C
:108DA800020A1A70104AC0F30743137000221146D2
:108DB80003E0520042F0010201319942F9D30B4914
:108DC800C0F300600A600A4A0121107001FA03F03A
:108DD800013B01FA03F1074A01389060516070477E
:108DE8005C4C0020554C0020494C0020584C002079
:108DF800534C00202C060020074B1878074B1B7893
:108E080043EA0020064B1B7843EA0020054B1B78F9
:108E18000BB140F080707047494C0020554C002041
:108E28005C4C0020534C0020684620F007018D461A
:108E380001B54FF4807008F00FFFD0B14FF4807087
:108E480008F018FF0020FFF7C5FE002007F022FDFC
:108E58000A4B1B786BB90A4B9A6822F480729A60A5
:108E6800DA6822F48072DA60064B1A6922F08062AE
:108E78001A61BDE801408546704700BF504C00208C
:108E8800003C01409C4C0020014B53F820007047E7
:108E9800404C0020014B53F820007047444C002000
:108EA800014B43F820106FE4404C0020014B43F87D
:108EB800201069E4444C002070477047704700BF99
:108EC8002DE9F04F01218BB04FF4805009F02CF9B7
:108ED8006A4D012000240226E023014608938DF8FC
:108EE80026408DF827408DF824608DF8256009F01C
:108EF800EBF8284608A908F02FFF052128460A465E
:108F080008F0ADFFDFF8808128460621052208F029
:108F1800A6FF05222846072108F0A1FF01251023F6
:108F28004FF4827A4FF4007B404603A9ADF818301D
:108F38000193ADF80C40ADF81040ADF81A40ADF80B
:108F48001C40ADF80EA0ADF81260ADF81450ADF8A5
:108F580016B009F0EDF94046294609F084FA294689
:108F68004FF4804009F0D4F808F554484FF46042B3
:108F78003046294608928DF826408DF827408DF80E
:108F880024608DF8256009F09FF8404608A908F08C
:108F9800E3FE40460D21052208F061FF40460E2100
:108FA800052208F05CFF052240460F2108F057FF14
:108FB800A8F5E638019B404603A9ADF81830ADF88E
:108FC8000C40ADF81040ADF81A40ADF81C40ADF8B3
:108FD8000EA0ADF81260ADF81450ADF816B009F057
:108FE800A7F94046294609F03EFA254F29464FF48D
:108FF800004009F08DF84FF4E05204202946089209
:109008008DF826408DF827408DF824608DF825606E
:1090180009F05AF8384608A908F09EFE38460A2191
:10902800062208F01CFF38460B21062208F017FF1D
:1090380038460C21062208F012FFADF80C40ADF8B6
:109048001040ADF81A40ADF81C400E4C019B20466C
:1090580003A9ADF80EA0ADF81260ADF81450ADF844
:1090680016B0ADF8183009F063F920462946B14624
:1090780009F0F9F90BB0BDE8F08F00BF000002401D
:1090880000080240003C00400030014070B5044632
:109098000D461646032869D8DFE800F00204080DDB
:1090A800022209E0334B10225A8308E0314B4FF477
:1090B80000425A8325E040222F4B5A8310E02F4864
:1090C800022109F061FA0028F9D02C48294609F054
:1090D80025FA2A48012109F057FA0028F9D020E09A
:1090E8002748022109F050FA0028F9D024482946D7
:1090F80009F014FA2248012109F046FA0028F9D0AB
:109108000FE02048022109F03FFA0028F9D01D4855
:10911800294609F003FA1B48012109F035FA00280D
:10912800F9D0A6B1032C21D8DFE804F00204080D19
:10913800022209E00F4B10221A830EE00D4B4FF468
:1091480000421A830DE040220B4B1A8307E0032CE0
:109158000ED8DFE804F004020604084802E00848D4
:1091680000E0084809F0D7F9C0B270BD002070BD12
:10917800002070BD00000240001002400030014095
:1091880000380040003C00402DE9F04101219CB02E
:109198004FF4800008F098FF01214FF480700025FB
:1091A80008F0C2FF032733231AA950481A938DF8F1
:1091B8006C708DF86F5008F0CFFD1AA94C48012447
:1091C8001A978DF86C708DF86F5008F0C5FD1AA9C4
:1091D8004848494E1A948DF86C708DF86F5008F015
:1091E800BBFD21464FF4800008F06EFF21464FF486
:1091F800807008F099FF304608F02AFB3F4B4FF08B
:10920800070802933E4B304603934FF4806307935D
:109218004FF4006308934FF4005309934FF480739D
:109228000A9301A94FF400330B9301950495CDF8E7
:10923800148006950C950D940E950F9508F094FBE7
:10924800214630462F4E08F0CAFB16A816951795EA
:109258001895199508F070F9304610A910958DF8F1
:1092680044408DF845401295139514958DF8548017
:1092780008F033F93046214608F02CFA30460A2126
:109288002246234608F0A4F930460E21022223463E
:1092980008F09EF930460F213A46234608F098F91F
:1092A800304608210422234608F092F93046092165
:1092B8002346052208F08CF930460B212346062266
:1092C80008F086F9424623463046294608F080F9D8
:1092D8003046214608F007FA3046214608F046F99C
:1092E800304608F0C3F91CB0BDE8F0810008024020
:1092F8000004024000000240106402404C2001407B
:1093080038060020002001400928F8B51CD005D8EF
:1093180004280ED008280FD040B17AE00B2863D07B
:109328005FD30C2863D0FF2873D16EE0464B1888B2
:109338006DE0454B58886AE0434B588940F27123E9
:1093480080B258430013F8BD3F4B988880B20CF0A8
:1093580009FA0BF0EBFD00223C4B0BF03BFE2EA371
:10936800D3E900230BF036FE04460D4622462B4671
:1093780029A1D1E900010BF079FC29A3D3E9002345
:1093880006460F46204629460BF04EFF02460B467E
:10939800304639460BF048FF0CF0DEF80BF0C6FDFE
:1093A80000222B4B0BF040FF0EF098F81EA3D3E9D8
:1093B80000230BF00FFE1EA3D3E900230BF058FC8B
:1093C80002460B461CA1D1E900010BF02DFF1CA39E
:1093D800D3E900230BF04AFC0CF0BEF80CF090FB2C
:1093E800F8BD194BD88804E0174B188901E0164BD3
:1093F800988944F2740380B2584340F6FF7390FB97
:10940800F3F0A0F500503A38F8BD0F4B988880B2B9
:10941800F8BD0020F8BD00BF6666666666660A404D
:109428009A99999999990140C3F5285C8FA272403D
:109438000000000000FEAA409A999999FD6F2F41FB
:10944800C3F5285C8F127140380600200000303FB9
:1094580000002440AFF300800C4B072202FB0030D1
:1094680090F800380B7090F801384B7090F802387B
:109478008B7090F80338CB7090F804380B7190F823
:1094880005384B7190F806388B71704748060020F4
:10949800254938B500224FF400635A540133B3F517
:1094A800804FFAD14FF40064002006210122FFF713
:1094B800EDFD002005210246FFF7E8FD002001220E
:1094C8000146FFF7E3FD8007F3D50020022102469D
:1094D800FFF7DCFD0020C4F307210246FFF7D6FDA5
:1094E8000020E1B20246FFF7D1FD0025A5F13F01BA
:1094F8004A4242EB0102002001460135FFF7C6FD52
:10950800402DF3D1002005210246FFF7BFFD0020C2
:1095180001220146FFF7BAFDC307F3D44034B4F57E
:10952800804FC1D138BD00BF48060020F7B50725D8
:10953800454300200C4602460321FFF7A7FD05F529
:1095480000650020C5F307210246FFF79FFD0020B4
:10955800E9B20246FFF79AFD002001460246FFF7EE
:1095680095FD0746002001460246FFF78FFD064697
:10957800002001460246FFF789FD05460020014606
:109588000246FFF783FD8DF80300002001460246DE
:10959800FFF77CFD8DF80400002001460246FFF726
:1095A80075FD8DF80500002001220146FFF76EFDCC
:1095B80023788DF80600BB4210D16378B3420DD1F1
:1095C800A378AB420AD1DDF80300D4F80330C3EB2B
:1095D800000CDCF1000040EB0C0000E00020FEBDB8
:1095E80038B51B4B04460D461955002006210122AB
:1095F800FFF74CFD002005210246FFF747FD00203C
:1096080001220146FFF742FD8207F3D5002002211F
:109618000246FFF73BFD0020C4F307210246FFF78F
:1096280035FD0020E1B20246FFF730FD0020294653
:109638000122FFF72BFD002005210246FFF726FD3A
:10964800002001220146FFF721FDC307F3D438BDEE
:109658004806002038B50725454305F500650C4642
:1096680028460978FFF7BCFF681C6178FFF7B8FF48
:10967800A81CA178FFF7B4FFE81CE178FFF7B0FF5A
:10968800281D2179FFF7ACFF681D6179FFF7A8FF56
:10969800A179A81DBDE83840A2E72DE9F843164690
:1096A800424A044688460023121803E018F80310BB
:1096B800D1540133B342F9D1002006210122FFF72A
:1096C800E5FC002005210246FFF7E0FC002001220E
:1096D8000146FFF7DBFC8307F3D500200221024691
:1096E800FFF7D4FC0020C4F307210246FFF7CEFCA5
:1096F8000020E1B20246FFF7C9FC0025771E44E0CE
:10970800013414F03F0918F8051006D0C7EB050E10
:10971800DEF1000242EB0E0200E00122D2B200208C
:10972800FFF7B4FCB9F1000F2ED1BD422CD20020B6
:1097380005210246FFF7AAFC002001220146FFF797
:10974800A5FC10F00100F2D106210122FFF79EFCD2
:10975800002005210246FFF799FC0020012201465E
:10976800FFF794FC8007F3D5002002210246FFF79B
:109778008DFC0020C4F307210246FFF787FC002078
:10978800E1B20246FFF782FC0135B542B8D10020AC
:1097980005210246FFF77AFC002001460122FFF767
:1097A80075FCC107F3D4BDE8F88300BF4806002064
:1097B800014B185C704700BF4806002010B5054CE7
:1097C8000023201802E0C45CCC5401339342FAD140
:1097D80010BD00BF48060020F7B50020032102464F
:1097E800FFF754FC002001460246FFF74FFC00201B
:1097F80001460246FFF74AFC404D002443F6FF7637
:10980800A11B4A4242EB010200200146FFF73EFC41
:1098180060550134B4F5804FF2D10020052102468D
:10982800FFF734FC002001220146FFF72FFC10F05F
:109838007104F2D1FEF7FEFC40F2CF7607462F4DB9
:1098480006E095F8FF47A4F14202544244EB0204B3
:10985800FEF7F0FCC01B0028B8BF4042B04202DC53
:10986800002CEED000E01CB1254B1B78002B39D022
:1098780040F2FF700021FFF7B3FEFFF709FE00205A
:1098880020494022FFF709FF4FF480701E49B42297
:10989800FFF703FF40201D492022FFF7FEFE02AD1F
:1098A800002345F8043D4FF4C364204604222946AA
:1098B8000434FFF7F2FEB4F5FF6FF6D102AD0023D2
:1098C80045F8043D4FF4A764204604222946043491
:1098D800FFF7E3FEB4F5C36FF6D140F2FF70422103
:1098E800FFF77EFE002040220649FFF767FF402071
:1098F80007492022FFF762FFFEBD00BF480600208F
:10990800844C002004000020B07B0108907B0108F3
:109918009C4C0020F8B505460C4606F027FE064686
:1099280028B128462146BDE8F84006F025BE324653
:10993800C4F307410120FFF7A9FB0B4D070232468C
:10994800C4F307212F600120FFF7A0FB47EA0006B8
:10995800360201202E60E1B20246FFF797FB06436C
:1099680036092E60F8BD00BF48460020254B03216C
:1099780010B501FB003292F905403F2C01DD3F2470
:10998800547101FB003393F905203F3201DAC122FB
:109998005A711C4B032202FB003291791F2901D90D
:1099A8001F2191714FF440229A60032202FB003379
:1099B8001B79012B03D1134B4FF450229A60114BA2
:1099C800032103EBC002D27C01FB00311AB94A79AA
:1099D80002F07F0205E0497902F0030201F07C0100
:1099E8000A439968074C41EA02229A60032303FB61
:1099F80000439979A3681943A160FFF78BFFA36817
:109A0800636110BD48460020204B052110B501FBBD
:109A18000032147E012C01D90124147601FB003395
:109A28005A7E032A01D903225A76184B052101FBD5
:109A38000032947E0F2C01D90F24947601FB003359
:109A4800DA7E032A01D90322DA76104C052303FBB8
:109A58000042117F0F2901D90F21117703FB004321
:109A6800197F1A7E41F4202141EAC2315A7E41EA27
:109A780042319A7EDB7E41EA022141EA4311A1602C
:109A8800FFF748FFA368236210BD00BF48460020C7
:109A9800524B0B2110B501FB003292F82440032CE5
:109AA80002D9032482F8244001FB003393F82620CE
:109AB800032A02D9032283F82620484B0B2101FBF5
:109AC800003292F828400F2C02D90F2482F828403F
:109AD80001FB003393F82920072A02D9072283F8CB
:109AE80029203E4B0B2101FB003292F82A400F2C13
:109AF80002D90F2482F82A4001FB003393F82D2065
:109B08000F2A02D90F2283F82D2034490B2202FB99
:109B1800001393F82E400F2C02D90F2483F82E40FF
:109B280002FB001292F82430DB0343F400248C601B
:109B380092F8251019B1294A43F404239360274B5E
:109B48000B2202FB003292F827201AB19A6842F4DD
:109B580000529A600B2279B902FB003292F8281061
:109B680092F82640C90141EAC4219C6892F829204C
:109B7800214341EA02121DE002FB003292F82C3028
:109B880016491BB18B6843F480538B60134B0B222F
:109B980002FB003292F82E1092F82D409A6842EAA1
:109BA800C41201F0070442EA041209079A6002D5B8
:109BB80042F400629A60094C0B2303FB004393F8BC
:109BC8002B2022B993F82A20A3681343A360A16825
:109BD800FFF7A0FEA368236310BD00BF484600201E
:109BE80038B51F4B4FF460229A60C2009918C97C9F
:109BF80011B14FF4702199609A18517B147B0903B5
:109C080041EA84319C6821439960937B012B03D1FD
:109C1800134B41F480619960114BC1005C189A683C
:109C2800E57B247C42EA0522012C9A6004BF42F0BD
:109C380080029A605B185B7C094A012B03D1936808
:109C480043F040039360064C04EBC003997CA3687F
:109C580043EA0111A160FFF75DFEA368636338BDA5
:109C68004846002010B5144B0022C1009A605A18CB
:109C780092F83D2012B14FF400729A605B1893F885
:109C88003E300D4A1BB1936843F4807393600A4CCD
:109C9800C300E21892F83F100F2902D90F2182F869
:109CA8003F10E31893F83F10A3681943A160FFF72A
:109CB80031FEA368236410BD48460020214B0120D3
:109CC80010B5032200240521187118740220987415
:109CD80083F8240083F82800597199711A735A730C
:109CE8009C73DC735C74DC741C765C769C76DC7626
:109CF8001C7783F83D4083F83E4083F83F4083F863
:109D0800254083F8274083F8264083F8292083F8E4
:109D18002A1083F82B4083F82C4083F82E2083F8F0
:109D28002D402046FFF770FE2046FFF71FFE204615
:109D3800FFF756FF2046FFF795FF2046BDE8104085
:109D4800A6E600BF48460020054B042903EBC003E4
:109D580083F83F1002D0002283F83D2082E700BF3D
:109D680048460020044B03EBC00383F83D1011B1B3
:109D7800042283F83F2075E748460020024B03EB96
:109D8800C00383F83E106DE748460020024B03EB02
:109D9800C00090F83F00704748460020024B03EB94
:109DA800C00090F83D00704748460020024B03EB86
:109DB800C00090F83E00704748460020034B0B2235
:109DC80002FB003383F8241062E600BF48460020F7
:109DD800034B0B2202FB003383F8251058E600BF23
:109DE80048460020034B0B2202FB003383F8271060
:109DF8004EE600BF48460020034B0B2202FB00330F
:109E080083F8261044E600BF48460020034B0B2287
:109E180002FB003383F828103AE600BF48460020CA
:109E2800034B0B2202FB003383F8291030E600BFF6
:109E380048460020034B0B2202FB003383F82A100C
:109E480026E600BF48460020034B0B2202FB0033E6
:109E580083F82C101CE600BF48460020034B0B2259
:109E680002FB003383F82D1012E600BF484600209D
:109E7800034B0B2202FB003383F82E1008E600BFC9
:109E880048460020034B0B2202FB003090F82400C8
:109E9800704700BF48460020034B0B2202FB0030EE
:109EA80090F82500704700BF48460020034B0B225E
:109EB80002FB003090F82700704700BF484600209A
:109EC800034B0B2202FB003090F82600704700BFBE
:109ED80048460020034B0B2202FB003090F8280074
:109EE800704700BF48460020034B0B2202FB00309E
:109EF80090F82900704700BF48460020034B0B220A
:109F080002FB003090F82A00704700BF4846002046
:109F1800034B0B2202FB003090F82C00704700BF67
:109F280048460020034B0B2202FB003090F82D001E
:109F3800704700BF48460020034B0B2202FB00304D
:109F480090F82E00704700BF48460020024B0522BB
:109F580002FB0033197657E548460020024B0522DC
:109F680002FB003359764FE548460020024B052294
:109F780002FB0033997647E548460020024B05224C
:109F880002FB0033D9763FE548460020024B052204
:109F980002FB0033197737E548460020024B0522BB
:109FA80002FB0030007E704748460020024B052225
:109FB80002FB0030407E704748460020024B0522D5
:109FC80002FB0030807E704748460020024B052285
:109FD80002FB0030C07E704748460020024B052235
:109FE80002FB0030007F704748460020024B0322E6
:109FF80002FB00331971B9E448460020024B0322E2
:10A0080002FB00335971B1E448460020024B032299
:10A0180002FB00339971A9E448460020024B032251
:10A0280002FB00300079704748460020034B0322AA
:10A0380002FB003090F90500704700BF4846002039
:10A04800024B032202FB003080797047484600200B
:10A05800024B03EBC0031973C2E500BF484600205A
:10A06800024B03EBC0035973BAE500BF4846002012
:10A07800024B03EBC0039973B2E500BF48460020CA
:10A08800024B03EBC003D973AAE500BF4846002082
:10A09800024B03EBC0031974A2E500BF4846002039
:10A0A800024B03EBC00359749AE500BF48460020F1
:10A0B800024B03EBC003997492E500BF48460020A9
:10A0C800054B10B503EBC003D9740446FFF788FDB0
:10A0D8002046BDE8104049E448460020024B03EB07
:10A0E800C000007B704700BF48460020024B03EBCE
:10A0F800C000407B704700BF48460020024B03EB7E
:10A10800C000807B704700BF48460020024B03EB2D
:10A11800C000C07B704700BF48460020024B03EBDD
:10A12800C000007C704700BF48460020024B03EB8C
:10A13800C000407C704700BF48460020024B03EB3C
:10A14800C000807C704700BF48460020024B03EBEC
:10A15800C000C07C704700BF484600202DE9F0478A
:10A16800314F98463B1893F8443004460D4616463E
:10A17800DDF820A0DDF82490042B1AD8DFE803F0DE
:10A1880003080D121700FFF783FC3B19012212E0A8
:10A19800FFF726FD3B1902220DE0FFF735FC3B19BE
:10A1A800032208E0FFF7E2FB3B19042203E0FFF774
:10A1B80059FD3B19002207EBC40483F84420A27C14
:10A1C800194B012A0DD002D3022A23D111E015B16F
:10A1D8001B689B0C2B70EEB1134B1B689B0A3370EA
:10A1E80018E0B8F1000F15D01B689B0AC8F80030BA
:10A1F80010E0B8F1000F04D01B68DB0B5B01C8F856
:10A208000030BAF1000F05D0074B1B68C3F3842355
:10A218008AF80030B9F1000F03D0034B1B6889F8A6
:10A228000030BDE8F08700BF48460020054B0B22F0
:10A2380002FB003393F82B201AB9012283F82B2054
:10A2480026E4704748460020054B0B2202FB0033EA
:10A2580093F82B201AB1002283F82B2018E47047BA
:10A2680048460020064B40F2826203EBC000407C67
:10A2780040F63B43002814BF10461846704700BFFD
:10A288004846002070B5104C054604EBC0039E7C80
:10A29800032E03D003229A74FFF7A2FC2846FFF787
:10A2A8009FFC2468200344BF6FEA04346FEA143427
:10A2B800032E06D0044B284603EBC5039E74FFF714
:10A2C8008FFC204670BD00BF4846002070B50A4C80
:10A2D8009DF810609DF8145004EBC00484F8381001
:10A2E80084F8392084F83A3084F83B6084F83C508C
:10A2F800BDE87040B6E400BF4846002006281CD8D8
:10A30800DFE800F004070A0D101317000B4B1B6859
:10A318000DE00A4B1B6C0AE0084B1B6B07E0074B70
:10A328001B6A04E0054B5B6901E0044B5B6B0B6047
:10A338007047024B93F82B300B607047484600205B
:10A3480070477047704770477047704770471223CF
:10A358000B800148704700BF4400002004230B8095
:10A3680000487047560000200020704700207047C2
:10A378000020704770B5084C0022236806E03F2B88
:10A3880003D8865CE5182E71013301328A42F6D172
:10A39800014A0020136070BD9046002010B5044C9F
:10A3A8000A460448214609F0F9FB204610BD00BFC3
:10A3B800A36100204C91010810B5044C0A460448DA
:10A3C800214609F0EBFB204610BD00BFA361002029
:10A3D8005A91010810B5044C0A460448214609F070
:10A3E800DDFB204610BD00BFA36100206591010878
:10A3F80010B5044C0A460448214609F0CFFB204614
:10A4080010BD00BFA36100206D91010810B5044C78
:10A418000A460448214609F0C1FB204610BD00BF8A
:10A42800A361002085910108202802D0212822D18B
:10A4380012E08A784878120442EA002208780F4B22
:10A448000243C87842EA00629A610A791A774A791F
:10A458005A778A799A770EE0084B9A69100A0A7037
:10A468004870100C120ECA701A7F88700A715A7FD1
:10A478009B7F4A718B710020704700BF4400002009
:10A48800F7B5274C4FF4C053002603270093204606
:10A49800022369468DF804308DF805708DF8066042
:10A4A8008DF8076007F058FC20460B210A2207F0B8
:10A4B800D6FC0A2220460C2107F0D1FC01254FF4D6
:10A4C80000732046694600938DF805708DF8046086
:10A4D8008DF806508DF8076007F03EFC0A222046EA
:10A4E800092107F0BCFC4FF48063204669460093BD
:10A4F8008DF806508DF807508DF8057007F02CFC84
:10A508000A210A46204607F0AAFC29464FF4804053
:10A5180007F00AFE8020294607F0E2FDFEBD00BFD5
:10A528000000024007B54FF4C06008F01DFE432349
:10A538008DF804300322012301A88DF805308DF829
:10A5480006208DF8073008F019FE0EBD7823584311
:10A558000723B0FBF3F0002301338342FCD9704793
:10A568004FF47A735843F1E7684620F007018D46A7
:10A5780001B503480AF00AF9BDE80140854670476D
:10A58800344D00200023F0B5094C0A4F40F2FF7506
:10A598001E460AE0226810F803C007F802C001321C
:10A5A800AA4288BF3246226001338B42F2D1F0BD05
:10A5B800204C0020A3590020074910B50A684AB169
:10A5C800002304315C5CC45401339342FAD1024B3A
:10A5D80000211960104610BD90460020084B1B68EA
:10A5E800082B0BD90023064A111D595CC1540133AD
:10A5F800092BF8D100231360012070470020704711
:10A608009046002007B5054B054803F120023C336E
:10A6180000930121034B08F021FF0EBD44000020E8
:10A62800344D0020A001002001480AF083B800BF83
:10A63800344D002038B54A4CA07808B104228CE08B
:10A648006378C12B4AD015D80D2B0CD80C2B38D2D7
:10A65800052B28D002D8042B7ED120E0062B26D04B
:10A66800072B79D126E08C2B32D0B52B33D0822B17
:10A6780072D129E0CC2B3DD006D8C32B34D030D3AF
:10A68800C82B34D0C92B03E0D42B4ED002D8D22B00
:10A6980062D132E0D62B4CD0FE2B5DD14DE0BDE827
:10A6A800384005F01FBFBDE8384005F013BF49200A
:10A6B8002C4901E02C494A200122BDE83840FFF727
:10A6C8007DB84D202949F7E7BDE8384005F012BFAD
:10A6D8004B202749F0E75820264928E048202649FA
:10A6E800EAE74020254922E0442025491FE05F2071
:10A6F8002449E1E74E2024491DE0204C184D502004
:10A7080004F110010422FFF759F8A87804EB40136C
:10A71800D97CFEF76FF8A87804EB4014216921F082
:10A728007F41BDE83840FEF70DB81849542004228F
:10A73800C3E717495C200222BFE7104D4C2005F102
:10A748000C010122FFF73AF8A07805EB4015297BA8
:10A75800BDE8384005F0F0BE03220E4B1A7038BD34
:10A7680028530020A54C0020A64C0020A94C00200E
:10A77800A74C0020B44C0020A44C00209C4C002086
:10A78800A04C0020BB4C0020AA4C0020B04C00205C
:10A79800B84C00209C53002010B5904A9378022BA7
:10A7A80000F01581032B00F02781002B40F08981F0
:10A7B80053784D2B00F0A28021D8452B69D00ED8B4
:10A7C800422B53D005D8402B42D0412B40F0758105
:10A7D80043E0432B4FD0442B40F06F8151E0482B8E
:10A7E8006DD005D8462B59D0472B40F066815EE0E6
:10A7F8004B2B77D07CD8492B40F05F8165E0542BF8
:10A8080000F0AF8010D8512B00F08B8005D84F2B6B
:10A8180079D0502B40F051817DE0522B00F091808F
:10A82800532B40F04A8194E0832B00F0BC8006D87B
:10A83800552B00F0A080572B40F03F81A8E0852BD6
:10A8480000F0BB80C0F0B380FF2B40F03681BAE047
:10A85800624B40F2FF70D97804E0604B0020D97851
:10A868005F4B1970BDE81040FEF7BABED1785C4B5B
:10A8780001205970F6E7594B0420D978584B1971C3
:10A88800F0E7564B5649D3F803301C2041F81C3FDB
:10A898000BE0D178524B05205971E3E74F4B5049F3
:10A8A800D3F803300C2041F80C3F042277E04B4BDF
:10A8B8004B49D3F80330082041F8083FF5E7D3782F
:10A8C8004749262001F8263F68E0444BDA78444B94
:10A8D8000AB9DA7503E043490122DA754A60D97D7D
:10A8E8001720BFE73D4B0320D9783D4BD970B9E716
:10A8F8003A4B0220D9783A4B9970B3E7D178384B64
:10A9080015205975AEE7354B1920D3F80310344B91
:10A91800C9B25976A6E7314B1620D978304B9975CC
:10A92800A0E72F4B197D1C4611F0010F04D0D378F6
:10A93800DB0701D4FEF7ACFD284B1420D97821752C
:10A9480090E7264B2649D3F80330202041F8203FD2
:10A95800ABE7224B2249D3F80330102041F8103FCF
:10A96800A3E7D2F80330012B10D8D3781C491A205A
:10A9780001F81A3F12E0194BD3F80320012A05D831
:10A98800DB7817491B2001F81B3F07E0042295E0FC
:10A99800124B1349DB78272001F8273F0122BDE835
:10A9A8001040FEF77ABED2F803200F4B03E00B4BA2
:10A9B800D3F803200D4B1A6010BD084BD3F80320C1
:10A9C800094B5A6010BD054BDA78094B77E051788E
:10A9D800084BD2F8032043F8212010BD285300204B
:10A9E800040000209C530020D446002098530020E7
:10A9F80096530020A85300205378282B3AD00BD820
:10AA0800022B29D003D8ABB1012B56D11BE0092B5F
:10AA18005AD0272B51D128E02B2B3AD004D8292BF8
:10AA28002DD02A2B49D12FE02D2B3CD036D32E2BDD
:10AA380043D13DE0254BD2F803201A60FDF7FAFB1D
:10AA4800234B986010BD214BD2F803205A60FDF7C4
:10AA5800F1FB1F4BD86010BD1C4BD2F803209A6045
:10AA6800FDF7E8FB1A4B186110BDD2F80320174B0D
:10AA7800DA6010BDD2F80320144B1A6110BDD2F869
:10AA88000320124B5A6110BDD2F803200F4B9A6174
:10AA980010BDD2F803200D4BDA6110BDD2F80320A7
:10AAA8000A4B1A6210BDD2F80320084B5A6210BD37
:10AAB800D2F80320054B9A6210BD0322054B1A7089
:10AAC80010BD044B04221A7010BD00BFC04C0020FA
:10AAD800D44600209C53002038B54E4B1A7D9AB9B5
:10AAE8004D4AD2F80320511C4FF00A0104D14B4AB9
:10AAF80012685143996101E04A439A61FDF79AFB54
:10AB0800444B0122D8611A75434B5A78042A7FD8DE
:10AB1800DFE802F003182F4F1100FDF78BFB3D4BC8
:10AB2800DA69801A9A690028B8BF404290423CD935
:10AB380000221A7538BD987803F09AF8354C38BB5E
:10AB4800207547E0987805F093FC324C054610B123
:10AB5800002323753EE0A36933B3FDF76BFBE3697C
:10AB6800C01AA3690028B8BF404298421CD925756D
:10AB780044E02B4C627E1AB9987805F0CDFC30BBC6
:10AB8800637E23B1244B987805F0C6FCF8B1214CBC
:10AB9800A3694BB1FDF74EFBE369C01AA36900280E
:10ABA800B8BF4042984227D81A4B1A6A013A1A622B
:10ABB80038BD1B4C627E1AB9987805F0B5FC30B9DF
:10ABC800637E63B1144B987805F0AEFC38B9114B2D
:10ABD80000221A75134B1A6822F0100212E00D4C6D
:10ABE800A3698BB1FDF726FBE369C01AA3690028A6
:10ABF800B8BF4042984207D900232375094B1A6809
:10AC080042F010021A6038BD024B1A6A013A1A6201
:10AC180038BD00BFD44600202853002088530020A8
:10AC2800040000203053002010B51F4B9A78012AE9
:10AC38001CD003D3022A1D4C21D11BE058780828C8
:10AC480002D8FDF74AFC0EE00A2803D1174B002270
:10AC58005A6016E00B2802D1FDF76CFD03E0FF28CF
:10AC68000FD1FDF7A5FC114B58600AE05878FEF7A4
:10AC78004BFBF8E75878FDF767FC606001E00423B8
:10AC880023700B4B1B7873B1084B5A68094B1A6039
:10AC9800094B22B91A6842F008021A6010BD1A68F6
:10ACA80022F008021A6010BD285300209C5300208F
:10ACB80097530020885300203053002038B5204B8C
:10ACC8005A78812A3AD19A78922A37D19A79A32A3E
:10ACD80034D15A79B42A31D11A79C52A2ED1DB78E0
:10ACE800D62B2BD1174B04221A83FFF79DFCFDF7B7
:10ACF800A1FA40F2E7340546FDF79CFA401B00280C
:10AD0800B8BF4042A042F7DD72B6FDF7C1FE0E4B58
:10AD180000241C6021460D4806F061FE0B4806F031
:10AD280097FD06F0CDFB06F02FFF4FF0804007F0AF
:10AD3800C9FC2046BDE83840FDF79CBE38BD00BFC1
:10AD4800285300200010024010E000E01064024088
:10AD580038B59B4C63788A2B00F0598200F28280C8
:10AD6800732B00F0C7813ED80D2B00F06A811BD8E9
:10AD7800042B00F029810BD8012B00F01684C0F0B9
:10AD8800F980022B00F0FE80032B40F01C8408E1C0
:10AD9800062B00F03581C0F02781072B00F03781A2
:10ADA8000C2B40F010843DE16E2B00F082810ED810
:10ADB800112B00F06A8103D80E2B40F004844FE178
:10ADC8006C2B00F068816D2B40F0FD836AE1702BDD
:10ADD80000F07C81C0F07381712B00F07D81722BB3
:10ADE80040F0F1837FE17E2B00F0D2811BD8782BD5
:10ADF80000F0AC810BD8752B00F08981C0F0808100
:10AE0800762B00F09581772B40F0DD8397E17A2B44
:10AE180000F0A981C0F0A0817C2B00F0AB817D2BD4
:10AE280040F0D183ADE1842B00F0C3810BD8802B97
:10AE380000F00082C0F0F181812B00F0AF81822BFD
:10AE480040F0C183FDE1872B00F0C58103D8862B34
:10AE580040F0B983B8E1882B00F0C381892B40F01A
:10AE6800B283CAE1B22B00F028833ED8A82B00F0A9
:10AE7800C8821ED8A32B00F074820ED8A02B00F035
:10AE8800568203D88C2B40F09E83E9E1A12B00F079
:10AE98005682A22B40F097835AE2A52B00F07B82C2
:10AEA800C0F06782A62B00F09182A72B40F08B831D
:10AEB8009EE2AD2B00F0D6820BD8AA2B00F0B2820E
:10AEC800C0F0A782AB2B00F0B582AC2B40F07B839F
:10AED800B9E2AF2B00F0D782C0F0CC82B02B00F0E3
:10AEE800DA82B12B40F06F83DEE2C82B00F0EA81F2
:10AEF80021D8B82B00F021830ED8B52B00F0EE82B4
:10AF080003D8B32B40F05F83DFE2B62B00F0F48266
:10AF1800B72B40F0588307E3C22B00F0BC8103D85D
:10AF2800C12B40F05083ADE1C32B00F0BF81C62B8D
:10AF380040F0498309E3D12B00F037830BD8CA2BA3
:10AF480000F02583C0F01683CB2B00F02783CC2B91
:10AF580040F03983BEE1D42B00F0C58103D8D22B51
:10AF680040F0318327E3D62B00F0C581FE2B40F05B
:10AF78002A83C9E1124B9878D3F80310BDE838400A
:10AF880005F020B90E4A0F48D2F8031001F180539A
:10AF9800013B834200F2C7819078BDE8384005F054
:10AFA800B7B8074A0748D2F8031001F18053013BAC
:10AFB800834200F2B8819078BDE8384005F0C6B801
:10AFC80028530020FEFFFF1FD4F80310534801F157
:10AFD8008052013A824204D8A078BDE8384005F092
:10AFE80039B94F4A137038BD4E4BD3F80310B1F13D
:10AFF800007F80F098819878BDE8384005F00AB95C
:10B00800A378494AE17802EB4312517206E0454AB7
:10B0180045499378D27801EB43118A72434A01215A
:10B02800D15438BD3F4A404BD2F80310927803EB15
:10B0380042135A7B11B942F002020FE022F00202D9
:10B048000CE0A278384BD4F8031003EB42135A7B78
:10B0580011B942F0010201E022F001025A7338BD31
:10B06800304C0221A07805F015F9D4F8035004F00B
:10B0780013F8002DB8BF6D42854200F35481D4F80F
:10B088000300BDE8384005F025BCD4F80300BDE84E
:10B09800384005F06BBC234BD3F80300BDE83840BB
:10B0A80005F0D8BA1F4BD3F80300BDE8384005F0C7
:10B0B800D7BAD4F80300BDE8384005F0D7BA194B21
:10B0C800D3F80300BDE8384005F068BAD4F80300A7
:10B0D800BDE8384005F06EBA124BD3F80300BDE85E
:10B0E800384005F07DBA0F4BD3F80300BDE838406F
:10B0F80005F07CBAD4F80300BDE8384005F0BEBBC3
:10B10800084BD3F80300BDE8384005F075BAD4F809
:10B118000300BDE8384005F075BA00BFFEFFFF1F09
:10B128009C530020285300209C4C0020F84C002001
:10B13800494BD3F80300BDE8384005F069BA464BDF
:10B14800D3F80300BDE8384005F068BAD4F8030026
:10B15800BDE8384005F068BA3F4BD3F80300BDE8B6
:10B16800384005F069BAD4F80300C0B2BDE83840E9
:10B1780005F06ABA384BD3F80300BDE8384005F04B
:10B1880033BB354BD3F80300BDE8384005F06ABB44
:10B19800D4F80300BDE8384005F032BB2E4BD3F895
:10B1A80003109878003118BF0121BDE8384005F038
:10B1B8007BB8D4F80330002B00F0088205F052FC6D
:10B1C800002840F00382AEE0234BD3F80300BDE82B
:10B1D800384005F057BAD4F80300BDE8384005F008
:10B1E8004BBA1D4BD3F80300A0F10A03282B00F239
:10B1F8009A80BDE8384005F04BBA174BD3F80300E6
:10B208000028C0F29080BDE8384005F047BAD4F86D
:10B218000300BDE8384005F047BA0F4BD3F80320C8
:10B22800022A00F280809A780C49DB788A1882F822
:10B23800243038BDA078D4F80310BDE8384005F0B4
:10B2480029B8054BD3F80310B1F1805F6BD8987813
:10B25800BDE8384004F09ABF28530020D4460020A7
:10B26800574C584BA078E17803EB4013D97205F09E
:10B278002FF8E178A078C1F10801C9B2BDE83840DB
:10B28800FEF762BD4E4B4F4A9978D3F8033002EB74
:10B298004112137238BDD4F80330B3F1805F42D83D
:10B2A800474A4849927852018B5038BD444AD2F8EF
:10B2B8000330B3F1805F36D89178424A02EB4112ED
:10B2C800536038BDA2783F4B03EB4213D4F80320F8
:10B2D800DA7738BD3A4B3B4A9978D3F8033002EB1A
:10B2E8004112D38138BDA278364B03EB4213D4F810
:10B2F80003205A6138BD324B324A9978D3F803306B
:10B3080002EB4112938338BD2D4BD3F80320052A55
:10B3180009D89878D9782B4B03EB40131973BDE8FB
:10B32800384005F009B9284B04221A7038BDD4F802
:10B338000310A078C9B2BDE83840FEF713BD204B12
:10B34800D3F803109878C9B2BDE83840FEF716BDA7
:10B358001B4BD3F803109878C9B2BDE83840FEF704
:10B368002DBDD4F80310A078C9B2BDE83840FEF767
:10B378002FBD134CA078FEF78FFDD4F803100346B9
:10B38800C9B2A0781BB9BDE83840FEF735BDBDE8A5
:10B398003840FEF759BDA078FEF77EFD38B9D4F8DD
:10B3A8000310A078C9B2BDE83840FEF72FBDD4F825
:10B3B8000310A078C9B2BDE83840FEF759BD00BFF8
:10B3C800285300209C4C00209C530020474CA07818
:10B3D800FEF762FDD4F803100346C9B2A0781BB982
:10B3E800BDE83840FEF71CBDBDE83840FEF736BD65
:10B3F8003E4BD3F803109878C9B2BDE83840FEF741
:10B4080019BDD4F80310A078C9B2BDE83840FEF7DA
:10B418009DBD364BD3F803109878C9B2BDE83840C3
:10B42800FEF79CBDD4F80310A078C9B2BDE8384037
:10B43800FEF79CBD2D4BD3F803109878C9B2BDE830
:10B448003840FEF79BBD294CD4F80310A078C9B248
:10B45800FEF79CFDA278264B03EBC203D4F8032029
:10B468005A7138BDD4F80310A078C9B2BDE8384085
:10B47800FEF7BCBD1D4BD3F80310987849B2BDE860
:10B488003840FEF7BBBDD4F80310A078C9B2BDE8B8
:10B498003840FEF7DDBD154BD3F803109878C9B2D4
:10B4A800BDE83840FEF7DCBD104BD3F803109878A0
:10B4B800C9B2BDE83840FEF7DBBDD4F80310A07868
:10B4C800C9B2BDE83840FEF7DBBD084BD3F803101E
:10B4D8009878C9B2BDE83840FEF7E2BDA278054BBE
:10B4E80003EB4213D4F803209A6138BD2853002097
:10B4F800744C00209C4C0020354C364BA078D4F876
:10B50800032043F8302022B903EBC0035979FEF732
:10B518003DFDA078304B1B5C012B57D12C4BD978C3
:10B52800BDE83840FCF778BF294B2A4A9978D3F808
:10B53800033002EBC102137138BDD4F80310A078B0
:10B54800C9B2BDE83840FEF74DBC214A234B90787C
:10B55800D2F8031003EB401319B1196941F0806167
:10B5680002E0196921F080611961090EBDE83840CF
:10B57800FDF740B9164B9878D978184B03EB401370
:10B588001A6922F07F4242EA01621A61EEE7A07866
:10B59800D4F80310BDE83840FDF788BC0C4BD3F84D
:10B5A8000300BDE83840FDF7E7BBD4F80300BDE869
:10B5B800384005F06FB9064B9878D3F80310BDE80A
:10B5C8003840FDF76DBC064B03221A7038BD00BF2A
:10B5D80028530020744C0020FB4C00209C4C002079
:10B5E8009C5300207FB5AF4CAF4D237864226B701D
:10B5F8002A70D4F80300222B686001F0FD8257D826
:10B608000F2B01F0B18026D8072B00F0F68510D853
:10B61800032B00F0DF8006D8012B00F0A980022B55
:10B6280041F04A85BDE0052B00F0AB8100F2C081F6
:10B63800E2E00B2B00F0F88706D8092B00F08F8684
:10B6480000F2918600F087BE0D2B01F0228001F2F6
:10B65800448001F002B8192B01F07E8113D8152B14
:10B6680001F0E48007D8132B01F08280142B41F0FD
:10B67800238501F0B8B8172B8C4B01F0558101F2E6
:10B688005F8101F04FB91E2B01F09F8109D81B2B58
:10B6980001F08681C1F071811C2B41F00D8501F00C
:10B6A8008FB9202B01F00E8201F2538201F0C9B943
:10B6B800812B01F057832ED8412B01F0398315D8FF
:10B6C800252B01F0EF8207D8232B01F0A182242B30
:10B6D80041F0F28401F0B8BA272B01F01283C1F0CF
:10B6E800EC82402B41F0E88401F01FBB452B01F0B0
:10B6F8002B8306D8432B01F0218301F2228301F02A
:10B708001ABB472B01F02683C1F02183802B41F01F
:10B71800D38401F022BB882B01F0BE8312D8842B7E
:10B7280001F05D8307D8822B01F03483832B41F02D
:10B73800C38401F034BB862B01F0738301F2E283EA
:10B7480001F06ABB8C2B01F03A8406D88A2B01F0F1
:10B758001D8401F22F8401F001BCF22B01F0A084BA
:10B76800FF2B01F0A0848D2B41F0A68401F04DBC85
:10B77800A3788BB94B4C0020012104F08BFDD4F841
:10B788000310A07804F0C4FCA37849490022CA54E5
:10B798004849CA5401F093BC434B04221A7001F083
:10B7A8008EBC404DAC7884B92046012104F072FD6E
:10B7B800D5F80310A878494204F0AAFCAB783C4AB3
:10B7C800D4543C4AD45401F07ABC374B04221A7042
:10B7D80001F075BCA6785EB9304602F041FA05F072
:10B7E80085F8A378324AD654324AD65401F067BC59
:10B7F80004232B7001F063BCA378002B40F0BC80BD
:10B80800284B5B78032B00F2B280DFE803F0021AC2
:10B818005576274B00251D70264B224C1D7004F0D1
:10B82800D5FE18B1A078294604F034FDA078D4F8E4
:10B83800031004F0C7FCA078002104F02BFD01F0F0
:10B848003EBC1B4B00251D701A4B164C1D7004F096
:10B85800BDFE18B1A078294604F01CFDA478134B4E
:10B86800104D1B1993F82430012B07D002D3022B5B
:10B8780011D107E0204604F081FD06E0204604F0DF
:10B888008BFD02E02046FCF70BFFD5F80330C1180A
:10B89800204604F097FC034B0021987804F0FAFC4A
:10B8A80001F00DBC285300209C530020D4460020F2
:10B8B800984C00207D4C0020142819DC364B0026BB
:10B8C8001E70364B364C1E70364B53F8205004F021
:10B8D8007DFE18B1A078314604F0DCFCA07829463A
:10B8E80004F070FCA078002104F0D4FC01F0E7BB60
:10B8F8002D4B04221A7001F0E2BB142832DC264BCF
:10B9080000251D70254B264C1D7004F05FFE18B1F4
:10B91800A078294604F0BEFCA078244B204D1B18C3
:10B9280093F82430012B06D002D3022B13D105E063
:10B9380004F024FD04E004F02FFD01E0FCF7B0FE64
:10B94800AB78D5F80310174A591852F821208118F6
:10B95800184604F037FC124B0021987804F09AFC42
:10B9680001F0ADBB104B04221A7001F0A8BB0E4BBE
:10B9780003221A7001F0A3BB0B4B04221A7001F0CA
:10B988009EBBA3781BB9FFF7E3F901F098BB064B00
:10B9980004221A7001F093BB984C00207D4C0020C3
:10B9A80028530020345300209C530020D446002004
:10B9B800A378044C002B40F00784034B25465B78A2
:10B9C80004E000BF9C53002028530020FE2B00F207
:10B9D800F883DFE813F0FF00040109010E011301E9
:10B9E80018011D01210125012A01300143015601D9
:10B9F80060016A0177018F0193019701F603F6034D
:10BA0800F603F603F603F603F603F603F603F60366
:10BA1800F603F603F603F603F603F603F603F60356
:10BA2800F603F603F603F603F603F603F603F60346
:10BA3800F603F603F603F603F603F603F603F60336
:10BA4800F603F603F603F603F603F603F603F60326
:10BA5800F603F603F603F603F603F603F603F60316
:10BA6800F603F603F603F603F603F603F603F60306
:10BA7800F603F603F603F603F603F603F603F603F6
:10BA8800F603F603F603F603F603F603F603F603E6
:10BA9800F603F603F603F603F603F603F603F603D6
:10BAA800F603F603F603F603F603F603F6030702B6
:10BAB8000B020F02130217021B021F0223022702A6
:10BAC8002B022F02330237023B023F024302470296
:10BAD8004B024F02D202D7025302DC02E102650296
:10BAE80069026D027102750279027D02F603E602AF
:10BAF800F603F603F603F603F603F603F603F60376
:10BB0800F603810285028A028F02940299029E023C
:10BB1800F603F603F6032B03300335033A033F031A
:10BB28004F035F036F03740379037E038303880362
:10BB38008C03910396039B03A003A503AA03AF03F9
:10BB4800B303B703BB03BF03F603F603F603F60319
:10BB5800F603F603F603F603EA02EE02F202F60231
:10BB6800F603F603F603FA02C403C803CD03FE0284
:10BB7800F603020306031B03D103ED03F6031F03B9
:10BB8800F6032303F203F603F603F603F603F603BC
:10BB9800F603F603F603F603F603F603F603F603D5
:10BBA800F603AD02B102B502B902BD02C102C50277
:10BBB800C902CD02F603F603F603F603F603F6030D
:10BBC800F603F603F603F603F603F603F603F603A5
:10BBD800F6032703002004F0D1FB6060F6E20020A2
:10BBE80004F0DAFB6060F1E2002004F07BFB6060A7
:10BBF800ECE2002004F08EFB6060E7E2002004F035
:10BC0800F1FB6060E2E2002004F0D4FB6060DDE25A
:10BC18009D4B5B7A6360D9E29B4B9B7A6360D5E26C
:10BC2800002004F025FC6060D0E2984B1B69C3F348
:10BC380080236360CAE2964B587E30B904F074FCE6
:10BC4800003018BF01206060C0E2002004F06CFCE6
:10BC5800D0F1010038BF00206060B7E28C4B587EFD
:10BC680030B904F059FC003018BF01206060ADE223
:10BC7800002004F051FCD0F1010038BF00206060C2
:10BC8800A4E2814B5B7B980702D5002363609DE2A9
:10BC9800012363609AE27C4B5B7BD90702D50023C2
:10BCA800636093E20123636090E2002004F0B2FB3A
:10BCB800022803D004F092FD606087E204F010FED1
:10BCC800606083E2002004F0ABFB18B103F0E4F9F4
:10BCD80060607BE26F4CA078FEF7C4FAA2786A4BEA
:10BCE80003EB42135B7A5843FF2390FBF3F06A4B54
:10BCF80058606BE204F046FE606067E204F03CFEC8
:10BD0800606063E200206060634D04F0B1FB18B12D
:10BD18006B6843F001036B6004F034FE20B15E4BA6
:10BD28005A6842F002025A6004F050FC20B15A4BA3
:10BD38005A6842F004025A60564CA07804F06AFB34
:10BD480020B9554B5A6842F008025A60A07804F0AE
:10BD580061FB012804D1504B5A6842F010025A6026
:10BD68004C4B987804F056FB022804D14A4B5A6889
:10BD780042F020025A60454B1B695A0504D5464BD0
:10BD88005A6842F040025A60444B1A6912F0080F90
:10BD98001A4604D0404B596841F080015960136934
:10BDA800DB0604D53C4B5A6842F480725A6001F0B5
:10BDB80077FF20B1384B5A6842F400725A6001F09C
:10BDC80069FF20B1344B5A6842F480625A6001F02E
:10BDD8006DFF002800F0FA812F4B5A6842F4006288
:10BDE8005A60F3E104F0C4FC6060EFE104F0C6FCC3
:10BDF8006060EBE104F0C8FC6060E7E104F0D4FBAC
:10BE08006060E3E104F0DCFB6060DFE104F052FC19
:10BE18006060DBE104F054FC6060D7E104F034FDBD
:10BE28006060D3E104F052FC6060CFE104F054FCA0
:10BE38006060CBE104F056FC6060C7E104F058FC98
:10BE48006060C3E104F05AFC6060BFE104F060FC8C
:10BE58006060BBE104F066FC6060B7E104F06AFC76
:10BE68006060B3E104F0C6FC6060AFE104F000FD7F
:10BE78006060ABE104F0DEFC6060A7E1002004F044
:10BE8800CFFA6060A2E100BF9C4C0020000C024089
:10BE980004000020285300209C5300200004024086
:10BEA80004F0F6FD606091E104F090FB60608DE1C4
:10BEB80004F07CFC606089E104F072FC606085E15C
:10BEC80004F07AFC606081E104F07CFC60607DE154
:10BED80004F07EFC606079E104F07AFD606075E151
:10BEE8000A20FDF711FA606070E10B20FDF70CFAEB
:10BEF80060606BE10820FDF707FA606066E10C20DE
:10BF0800FDF702FA606061E10920FDF7FDF9606064
:10BF18005CE10020FEF7A6F9994B9A78994B03EB60
:10BF280042139B7A5843FF2390FBF3F060604DE186
:10BF380004F030FC606049E104F00EFC606045E10B
:10BF480004F010FC606041E104F051FD60603DE1E7
:10BF580004F058FD606039E104F06CFD606035E183
:10BF680004F0EEFB606031E1874B1B6863602DE1F4
:10BF78000B20FDF7C9F9606028E1844B93F8243061
:10BF8800636023E1002004F045FA60601EE10020B0
:10BF980004F0DEF9606019E1002004F0D3F9606074
:10BFA80014E1784BDB7A636010E1764B1B7A6360AF
:10BFB8000CE1744B1B68636008E1724B5B6863605B
:10BFC80004E1734B1B68636000E16E4BDB7F6360C9
:10BFD800FCE06C4BDB896360F8E06E4B1B686360C8
:10BFE800F4E06D4A00231178636011B16B490120B8
:10BFF800486013706A4B19781A4621B1674B596823
:10C0080041F00201596000231370DFE0654B1B7893
:10C018006360DBE05B4B5B696360D7E0594B9B8BEC
:10C028006360D3E0574B1B7B6360CFE00020FDF7D4
:10C03800B5FE6060CAE00020FDF7B8FE6060C5E0AC
:10C048000020FDF71FFF6060C0E00020FDF724FF1F
:10C058006060BBE00020FDF71FFF504C484B20B943
:10C068009878FDF72DFF6060B0E09878FDF750FFF5
:10C078006060ABE00020FDF70FFF484C404B20B953
:10C088009878FDF727FF6060A0E09878FDF754FFE7
:10C0980060609BE00020FDF7FFFE404C384B20B964
:10C0A8009878FDF721FF606090E09878FDF73AFFF7
:10C0B80060608BE00020FDF721FF606086E00020D3
:10C0C800FDF76CFF606081E00020FDF76FFF6060A6
:10C0D8007CE00020FDF772FF606077E00020FDF74C
:10C0E80075FF606072E0304B5B7963606EE0002042
:10C0F800FDF794FF606069E00020FDF797FF60603E
:10C1080064E00020FDF7EAFF60605FE00020FDF7D3
:10C11800EDFF60605AE00020FDF7F0FF606055E039
:10C128000020FDF7F3FF606050E00020FDF7FEFF00
:10C1380060604BE01D4B1B78636047E0114B9B69C7
:10C14800636043E0184B1B6863603FE0164B1B7944
:10C1580063603BE00020FDF7A9FE606036E0094B14
:10C16800DB7C636032E00020FCF794FE60602DE029
:10C17800FCF742FE606029E004F0A2FB606025E065
:10C18800285300209C4C0020E0580020D446002072
:10C19800644C0020804C0020984C00209C530020C8
:10C1A8007D4C0020994C0020744C0020704C0020DD
:10C1B8000020FCF769FE606008E0FCF785FC606021
:10C1C80004E00323237001E004232370A94B1B78A8
:10C1D800002B00F07487A84B5A68A84B1A60A84B2C
:10C1E8002AB91A6842F008021A6000F068BF1A6893
:10C1F80022F008021A6000F062BFA3781BB1042382
:10C208002B7000F05CBF6378C12B60D018D80D2B61
:10C218000ED80C2B41D2052B2CD003D8042B40F080
:10C22800958022E0062B2AD0072B40F08F802DE046
:10C238008C2B3ED0B52B43D0822B40F0878033E047
:10C24800CC2B60D006D8C32B4FD047D3C82B53D0A4
:10C25800C92B03E0D42B64D002D8D22B76D159E075
:10C26800D62B65D0FE2B71D169E0002004F01EF9B1
:10C2780000F025BF002004F00FF900F020BF49208E
:10C2880080490122FDF709FA00F019BF4A207E49CA
:10C298000122FDF702FA00F012BF4D207B4901226E
:10C2A800FDF7FBF900F00BBF002004F009F900F0DE
:10C2B80006BF4B2076490122FDF7EFF900F0FFBEDB
:10C2C800582074490422FDF7E8F900F0F8BE482028
:10C2D80071490122FDF7E1F900F0F1BE40206F49F4
:10C2E8000422FDF7DAF900F0EABE44206C49042282
:10C2F800FDF7D3F900F0E3BE5F206A490122FDF79C
:10C30800CCF900F0DCBE4E2067490222FDF7C5F9E2
:10C3180000F0D5BE502065490422FDF7BEF900F0B3
:10C32800CEBE542062490422FDF7B7F900F0C7BE1B
:10C338005C2060490222FDF7B0F900F0C0BE4C2035
:10C348005D490122FDF7A9F900F0B9BE4A4B032265
:10C358001A7000F0B4BEFEF76DF900F0B0BEFEF73B
:10C368001BFA00F0ACBE554B9978022900F0F78013
:10C37800032900F0F980404A002940F03C815B78AD
:10C38800502B00F0AB8024D8462B61D011460DD835
:10C39800422B53D005D8402B47D0412B40F0278162
:10C3A8004AE0442B464A4FD050D84AE04B2B00F085
:10C3B800898006D8482B52D04ED3492B40F017819C
:10C3C80051E04D2B00F084807FD34F2B40F00F813C
:10C3D80081E0812B00F09980114612D8542B00F08F
:10C3E800868004D8522B364A7DD07ED879E0572BE8
:10C3F80000F08380802B00F08480552B40F0F7807C
:10C4080078E0852B104600F0928005D8832B00F049
:10C41800888000F2898081E0FE2B00F0978000F28E
:10C428009880F02B40F0E3808CE040F2FF70FDF73D
:10C43800BFF9114B5860E0E0214B88E0204B5B7856
:10C4480008E013794B60D8E0D369FBE75379F9E743
:10C458001B4BDB685360D0E0194B9B68F2E7184B25
:10C4680093F82630EEE7164BDB7D003318BF012327
:10C47800F0E700BF975300209C530020885300200A
:10C4880030530020A54C0020A64C0020A94C0020C9
:10C49800A74C0020B44C0020A44C00209C4C002049
:10C4A800A04C0020BB4C0020AA4C0020AC4C002023
:10C4B800B04C0020B84C0020A84C00202853002085
:10C4C80004000020964BDB78C4E7954B9B78B9E7CE
:10C4D800934B5B7DB6E7924B5B7EBBE7904B9B7DB6
:10C4E800B8E7137DAEE7136AACE71369AAE78C4B8C
:10C4F8009B7EAFE78A4BDA7E64E0894B93F827305E
:10C50800A0E7884B93F825309CE7864B93F82530B5
:10C51800A3F10400434243EB00039BE7814B1B6AF2
:10C5280090E7804B1B688DE77F4B1B680CE07D49CB
:10C538007E484B68434303F5405339334B6023F03F
:10C54800004387E77A4B1B78436056E0784B1B78AB
:10C5580078E7784B1B78003318BF012372E75A78C5
:10C56800754B53F822202DE05B78282B28D00CD867
:10C57800022B1FD004D8714AB3B1012B37D116E072
:10C58800092B3AD0272B32D117E02B2B6B4A22D01C
:10C5980004D8292B19D02A2B29D119E02D2B20D0EA
:10C5A8001CD32E2B23D11FE0654B1B6852E7644B2D
:10C5B8005B684FE7624B9A6804E0614BDA6801E018
:10C5C8005F4B1A695D4B5A6017E05D4B5B6941E749
:10C5D8005B4B9B693EE75A4BDB693BE7584B1B6A51
:10C5E80038E7574B5B6A35E7554B9B6A32E7534B45
:10C5F80003221A7001E004231370524B1B78002B9E
:10C6080000F05D854D4B5A684F4B1A604F4B2AB965
:10C618001A6842F008021A6000F051BD1A6822F048
:10C6280008021A6000F04BBDA378022B11D1637881
:10C63800372B0AD8404903F5A770800001EB830126
:10C648000422FDF72AF800F03ABD03232B7000F00E
:10C6580036BD04232B7000F032BDA378022B13D112
:10C668003B4B5B78372B0AD8334903F5A77080001A
:10C6780001EB83010422FDF7A1F800F020BD2F4B48
:10C6880003221A7000F01BBD2C4B04221A7000F014
:10C6980016BDA378E3B92E4B5B78012B09D003D3E1
:10C6A800022B264C10D109E0002001F0D1FA00F04D
:10C6B80006BD002001F0D4FA00F001BD002001F011
:10C6C800D7FA606000F0FBBC0323237000F0F7BCCE
:10C6D8001A4B04221A7000F0F2BCA37813B1022B93
:10C6E8003DD103E0FBF798FF00F0E9BC184B5B78FD
:10C6F800072B0AD820B91846FBF791FE00F0DFBCDB
:10C708001846FBF7B3FE00F0DABCFF2B22D1411C20
:10C718000ABF0D4BC0B21878FBF7CEFE00F0CFBCB5
:10C7280004000020D4460020985300206D4EC641D6
:10C73800F04C002096530020A85300209C53002062
:10C74800C04C00209753002088530020305300200D
:10C7580028530020944B03221A7000F0B0BC924B6F
:10C7680004221A7000F0ABBCFEF75EFA00F0A7BC1A
:10C7780062788E4B092A27D8DFE802F005080B0EED
:10C7880012181B1E21251A6810181CE01A68101AA6
:10C7980019E01A68504316E01A6892FBF0F012E0AC
:10C7A8001A6892FBF0F100FB11200CE01A681040A7
:10C7B80009E01A68104306E01A68504003E01A6856
:10C7C800D2431A6000E018601A68794B2AB91A68CF
:10C7D80042F008021A6000F072BC1A6822F00802DF
:10C7E8001A6000F06CBC714B1A68714B8242196870
:10C7F80004DD41F0040121F0030108E00BBF21F042
:10C80800060121F0070141F0010141F00201196020
:10C81800674B2AB91A6842F008021A6000F04FBC48
:10C828001A6822F008021A6000F049BC63780C2BE1
:10C8380000F24584DFE803F0071019222B343E4646
:10C848004E565E666E005A4B1B681A0740F13784D5
:10C85800584B186200F033BC554B1B681B0700F19E
:10C868002E84544B186200F02ABC514B1B68D90720
:10C8780040F125844F4B186200F021BC4C4B1B68DB
:10C88800DA0700F11C844B4B186200F018BC484BC7
:10C898001B685B0740F11384464B186200F00FBC1D
:10C8A800434B1B6813F0050F00F00984414B1862D5
:10C8B80000F005BC3E4B1B68990740F100843D4BD6
:10C8C8001862FCE33A4B1B689A0700F0F883394B6F
:10C8D8001862F4E3364B1B68DB0640F1F083354BF6
:10C8E8001862ECE3324B1B68990640F1E883314B40
:10C8F8001862E4E32E4B1B685A0640F1E0832D4B87
:10C908001862DCE32A4B1B681B0640F1D883294BCD
:10C918001862D4E3264B1B68D90540F1D083254B18
:10C928001862CCE31862CAE39A6A072A00F2C7833E
:10C938001C6A03EB82010132CC629A621862BEE380
:10C948009B6A1C4A002B00F0BA83013B936202EBFE
:10C958008303DB6A1362B2E363782E2B03D8164A8B
:10C968000121D154ABE3FF2B04D1124B012283F8F0
:10C978004C20A4E303232B70A1E3104B5B782E2BF0
:10C9880003D80D4A0021D15499E3FF2B04D1094B58
:10C99800002283F84C2092E3034B03221A708EE3A3
:10C9A800FEF79AF88BE300BF9C53002088530020C1
:10C9B80030530020D4460020044D00202853002086
:10C9C800974B002283F8252079E36378142B35D818
:10C9D800A278A2B9934A9449927E41F82300002A8A
:10C9E80000F06D83002B00F06A8303F5C2700130FC
:10C9F800800001EB83010422FCF74FFE5FE3FF2A6E
:10CA080018D163B9894D4FF4C3642919204604220B
:10CA18000434FCF742FEB4F5CD6FF6D14FE303F5CD
:10CA2800C27081490130800001EB83010422FCF7C8
:10CA380034FE44E37E4B04221A7040E303232B7038
:10CA48003DE36378142B39D87A4A9278BAB9764A92
:10CA580052F82320764B5A60774B1B78002B00F056
:10CA68002E83764B1A60764B22B91A6842F0080278
:10CA78001A6024E31A6822F008021A601FE3FF2AEA
:10CA880018D163B9694D4FF4C364291920460422AB
:10CA98000434FCF793FEB4F5CD6FF6D10FE303F53C
:10CAA800C27061490130800001EB83010422FCF768
:10CAB80085FE04E35E4B04221A7000E35C4B0322FC
:10CAC8001A70FCE26578142D3FD85A4CA0780206FB
:10CAD8001BD5C30704D503F05FFC534B43F825006F
:10CAE800504B9B7E002B00F0EA82524B5B78002B68
:10CAF80000F0E58203F5C2704B490130800001EB7C
:10CB080083010422FCF7C9FDD9E2D0B903F044FC43
:10CB1800444B45499B7E41F82500002B00F0CF820D
:10CB28006378002B00F0CB82A27803F5C270013045
:10CB3800D3188018800001EB83010422FCF7ADFDB7
:10CB4800BDE23B4B04221A70B9E2394B03221A703A
:10CB5800B5E26278394B0A2A40D8DFE802F0060BC2
:10CB680011161C24292E33373A00364A19681268E0
:10CB78008A1803E0334A196812688A1A1A602DE085
:10CB880030491A6809684A43F8E72E4A1968126852
:10CB980091FBF2F2F2E72B4A1968126891FBF2F066
:10CBA80002FB1012EAE7274A11681A680A40E5E70B
:10CBB800244A11681A680A43E0E7224A11681A6889
:10CBC8004A40DBE71F4B1A68D243D7E71A681D4B68
:10CBD800D4E71C4A1968106811601860174B1A6866
:10CBE800174B22B91A6842F008021A6067E21A68FD
:10CBF80022F008021A6062E2104B1B68C4F8033086
:10CC0800A37813B9FEF7A4F859E204232B7056E26F
:10CC18000A4B1B68C4F80330FDF7BEFD4FE200BFA6
:10CC2800D44600200400002034530020204D00206A
:10CC38009C5300202853002097530020885300203D
:10CC480030530020A4530020A24B5B78052B00F240
:10CC58003682DFE803F003090F151B219E4B1A6883
:10CC680002F00F021A602AE29B4B1A6822F01002A7
:10CC78001A6024E2984B1A6822F020021A601EE219
:10CC8800954B1A6822F040021A6018E2924B1A6813
:10CC980022F080021A6012E28F4B1A6822F4807226
:10CCA8001A600CE263782E2B04D88C4A02EB8303BB
:10CCB800186504E203232B7001E2884B884AD3F8F5
:10CCC8000C111160D3F81011864A1160D3F81421A1
:10CCD800D3F818111A62804A1160D3F81C218249CE
:10CCE8001A75D3F82021DA61D3F824219A6193F8D0
:10CCF8002821885C08B101208854002283F82C215F
:10CD0800DDE1A3786BB9734B5B78142B05D8744AB3
:10CD18001168764A42F82310D1E1754B03221A7044
:10CD2800CDE1734B04221A70C9E100F065FDC6E13C
:10CD380000F06AFDC3E100F068FDC0E100F066FDA7
:10CD4800BDE100F064FDBAE100F062FDB7E100F07A
:10CD580060FDB4E100F05EFDB1E1604B002283F8B4
:10CD68002520ACE1637813B1012B10D104E05B4BB3
:10CD7800012283F82520A2E1B0F5006F04D2574ABA
:10CD880082F8253010629AE104232B7097E103237F
:10CD98002B7094E1514B022283F825208FE14F4BF1
:10CDA8000022514C83F84C2083F82C2103F14C01CC
:10CDB8004FF0FF351046A054013200232F2A41F8C6
:10CDC800045FF8D1454A82F82530136293621375DF
:10CDD800434A1360434A13603F4A13606FE1454B6F
:10CDE8001B7D980715D403F059FE10B90A232B7040
:10CDF80065E1D4F803104FF00403B1F5006F05D2D4
:10CE0800364A82F82530C2F8301158E1384A137092
:10CE180055E108232B7052E1304B002283F825207E
:10CE28004DE1354B01221A70324A344B9178B0F5F6
:10CE3800006F197003D2147D14F0010409D0002288
:10CE48005A709A70DA701A715A719A71DA71197285
:10CE580035E101A9FCF700FB284B9DF804201C7262
:10CE68005A709DF805209A709DF80620DA709DF892
:10CE78000A201A719DF809205A719DF808209A71A4
:10CE88009DF80720DA710122D05C197A0132411825
:10CE9800082A1972F8D112E163787BB9164A012180
:10CEA80011701449154A89781170154909680133B8
:10CEB80011F8010B082B9854F9D100E1012B40F02F
:10CEC800FE800522EA716B711E220723AA712B715D
:10CED800F5E000BF2853002030530020D44600203E
:10CEE80088530020A4530020044D00203453002010
:10CEF8009C530020040000208C5300208D530020F8
:10CF0800000000206E4B5B78032B00F2D880DFE82E
:10CF180003F0020F1B206B4A6B4B92F82510D97156
:10CF2800117DD2F830219971110A59711A71C6E030
:10CF3800644A654B92F82510D971117D126A99716E
:10CF4800110A59711A71BAE0604B1A685E4B5A603F
:10CF5800B5E05F4B1A685C4B5A60B0E0584B5A78A2
:10CF6800002A40F0AC809978002940F0A88040F26F
:10CF7800D243984240F0A38040F2FF70FCF730FBA8
:10CF8800FCF786FA0120FBF775FD98E06278514BB3
:10CF9800003218BF01221A70E2784F4B1A70494BC1
:10CFA80093F834214D4B1A704D4A002313704D4AA3
:10CFB800137084E0434B012283F835217FE06678C3
:10CFC80016B1012E1ED10FE0042240F2FB7003A916
:10CFD800FCF7F4FBD4F80320039B9A4202D1012307
:10CFE8006B606CE06E606AE0A3782A2B06D140F291
:10CFF800FB703D490422FCF750FB60E0324B0322F2
:10D008001A705CE003232B7059E02D4B5B78032BDF
:10D0180042D8DFE803F00902313D2A4A0023D2F85A
:10D02800381102F59C7224E0264BD3F83821092ADE
:10D0380007D803EB82010132C1F83C01C3F838215B
:10D048003DE0214B09221A7039E052F8044F84421E
:10D058000ED1264A013902EB830203E050680133FE
:10D0680042F8040B8B42F9D3164BC3F8381126E06B
:10D0780001338B42E9D122E0124A0023C2F8383149
:10D08800194602F59E7299500433282BFBD116E0FD
:10D098000D4B0A225A6012E00B4B03221A700EE065
:10D0A800FDF70CFE0BE040F2D243984207D1054B46
:10D0B800012283F8642102E0034B02221A707FBD2B
:10D0C80028530020D44600209C5300208853002079
:10D0D800A4530020684C00207F4C0020FA4C00200C
:10D0E8007E4C0020334D00202B5300201048002098
:10D0F8003049002370B50B602F49304A0B60304926
:10D108003048136293620B60137582F84C3082F8D2
:10D118002C314FF0FF344C321946C15401332F2BB8
:10D1280042F8044FF9D1284B0020197B03F004FA88
:10D13800002326491A465A500433B3F5806FFAD1B2
:10D14800234B9B7E5BB1234D4FF4C36429192046C2
:10D1580004220434FCF732FBB4F5CD6FF6D11C4B36
:10D16800DC7E64B9194E4FF4A76506EB84012846A6
:10D1780004220134FCF722FB0435382CF5D1144A7B
:10D188001379012B08D0112B05D0A3F12104634298
:10D1980043EB040300E00123084C84F86531537D18
:10D1A80013B1FBF75BFA08B9002300E0012384F808
:10D1B800253070BD88530020A4530020D446002099
:10D1C80030530020044D00209C4C0020A853002020
:10D1D80004000020204D0020F7B50F4E05460C46F0
:10D1E80096E803008DE803000C496F46C1F8033048
:10D1F8000B4B8A7000220D704C701A70FEF7F2F912
:10D2080031787368074A82F866119DE8030086E85A
:10D2180003001846FEBD00BF9C5300202853002081
:10D2280097530020D4460020014B93F866017047BD
:10D23800D446002073B51F4D034602AA0C4695E854
:10D24800030002E9030059781B4A002611709978F7
:10D258005170D97891701979917159795171997979
:10D268001171DB79D370154B1E70FEF7BBF9144BA7
:10D278001A7872B922702B786270A3706B78E37099
:10D28800EB792371AB7963716B79A3712B79E371B6
:10D2980009E0012A07D10B4A334612F8011FE1546D
:10D2A8000133082BF9D1034B02AA12E9030083E8E2
:10D2B80003007CBD9C530020285300209753002076
:10D2C8008C5300208D5300202DE9F04F9C4B91B0DA
:10D2D8001B789C4A13B992F867316BB19A4B1B784B
:10D2E800062B09D00A2B07D00F2B05D01F2B03D0F4
:10D2F800944B002183F8341192F83431072B39D13B
:10D30800904B93F86531002B30D1904A12781ABBB4
:10D318008F4B9E785F788F4B8DF828601D785C78EE
:10D32800BE19D8798DF82A50AD1999798DF82B4006
:10D3380064195A798DF82C0000191B798DF82D1075
:10D3480009188DF82E2052188DF82F309B188DF85B
:10D3580029708DF830302CE0012A2AD17E4A985C59
:10D368000AA958540133092BF9D122E0794801F070
:10D3780049F922E0082B20D1764A00230120537076
:10D3880010705360724A8DF82A00917852788DF89F
:10D3980028108DF829208A1812188DF82B308DF84E
:10D3A8002C308DF82D308DF82E308DF82F308DF8EB
:10D3B80030200AA80921FDF7E5F8684B1B784BB324
:10D3C800674B1B78072B20D1614B98785978654BB0
:10D3D8008DF835101A78411880230A318DF83630C7
:10D3E8008A238DF834008DF837308DF83B200023E0
:10D3F80052180DA809218DF838308DF839308DF87C
:10D408003A308DF83C20FDF7BDF8564A00231370DA
:10D41800524A13704B4D4D4A002385F8343113702E
:10D4280085F8673195F8643113B10120FBF722FBC9
:10D4380095F83521434B52B193F86521D2F1010299
:10D4480038BF002283F86521002283F8352195F83A
:10D4580065313C4C83B13C4800F08DFF60B1FAF770
:10D46800E9FE414B414A186000231370032284F8F7
:10D47800342194F8252038E0324E96F86541002C86
:10D4880043D107AD2846FDF7A9F800283DD023462B
:10D498002A5D01349B18082CDBB2F9D19DF82420B1
:10D4A8009A422ED1284B9DF81D201A709DF81E20F7
:10D4B8005A709DF81F209A709DF820209A719DF847
:10D4C80021205A719DF822201A719DF82320DA70C4
:10D4D800FAF7B0FE244B254A186000231370194A46
:10D4E800072182F8341192F82520511EC9B201296A
:10D4F80019461F4B03D9052A01D001221EE01970D5
:10D508003CE0104B83F8344138E096F825300D4C58
:10D51800013BDBB2012B31D8236AB3F5006F29D266
:10D52800FBF79CF830B3206A0749431C2362FBF7DA
:10D5380093FF092384F834310D4B01221A701DE042
:10D5480096530020D4460020285300208C530020F6
:10D55800040000209C5300208D530020334D0020F0
:10D56800FA4C00207E4C0020F44C0020F94C00209E
:10D57800975300208F4B002283F825208D4C94F878
:10D588002530042B234604D18B4E3278110640F106
:10D59800E28093F834313BB1042B05D0082B03D03B
:10D5A800062B01D0FEF71EF8824C94F83431092B73
:10D5B80040F0A780FAF73EFE804BA2681B68801AED
:10D5C8000028B8BF4042984209D97D4B1A78012AF1
:10D5D80001D102221A70FAF72DFE764B9860FAF7FD
:10D5E80029FE744A754BD2685B68801A0028B8BF58
:10D5F8004042984209D9724B5A78012A01D1022235
:10D608005A70FAF717FE6B4BD860FAF713FE694A9F
:10D618006A4B12699B68801A0028B8BF404298423A
:10D6280009D9674B9A78012A01D102229A70FAF730
:10D6380001FE604B18615F4B93F84C20002A60D0C4
:10D6480093F82C1100295CD15E4A93F828A112683E
:10D65800D3F80C9101925C4AD3F8108112681C6AC5
:10D6680002925A4AD3F814C11268D3F81871039277
:10D67800DA69187D04929A69D3F81C61D3F82051AD
:10D68800D3F824B10592CDF800A00A46DFF830A1FE
:10D698001AF80230022B1BD1DFF838A15AF82230D1
:10D6A800B3F1FF3F0FD0D1B206460091A446DDF892
:10D6B80014B0049D039F1C46DDF80880DDF8049033
:10D6C8000121002004E0DFF8F8A000230AF8023066
:10D6D80001322F2ADAD1374B009AC3F80C91C3F8DC
:10D6E80010811C62C3F814C1C3F818711875C3F807
:10D6F8001C61C3F82051C3F824B183F8282183F8AA
:10D708002C112C4A92F83431092B06D192F8253085
:10D71800022B02D1052382F82530D2F83811254B87
:10D72800002943D093F83421092A3FD193F82520C2
:10D73800012A3BD1186A002203F59C7353F8044F61
:10D74800A04204D11B4B052283F825202EE001328C
:10D758008A42F3D12AE094F834313BB3042B25D024
:10D76800082B23D0062B21D0194DD4F830016A702C
:10D77800D6F80330B0F5006F6B6012D23146FBF774
:10D7880069FFD4F830013146FBF7D0FE30B1D4F848
:10D7980030310133C4F83031652300E007232B70A2
:10D7A80004E007232B70002384F8253011B0BDE86E
:10D7B800F08F00BFD446002028530020C04C002022
:10D7C800044D002088530020A4530020305300202B
:10D7D8009C53002024470020704710B5FAF72AFD13
:10D7E800044C2368C01AB0F5FA7F02D9FAF722FD73
:10D7F800206010BDA857002008B5FBF71FF9014BA2
:10D80800586008BD9C5300207047704770477047A8
:10D8180070477047704700BF2DE9F041A74B044699
:10D828005B7E5BB902F078FE061C204618BF012615
:10D8380002F07AFE003018BF01200CE002F06CFE06
:10D84800D0F10106204638BF002602F06DFED0F167
:10D85800010038BF00209A4B03EB44131B7A03F0F6
:10D868007F0513F0800F974B1B6907D013F4806F67
:10D8780014BF4FF000084FF0010801E0C3F38028FF
:10D888006B1E072B00F2DD81DFE813F008000800AB
:10D8980008000800EA00EA00EA00EA008A4F3B5D57
:10D8A800013B0E2B00F2CD81DFE813F00F002900B9
:10D8B8002F003A0040004800530064008800A70089
:10D8C800AB00CB01C600CD00B201204602F08AFDB4
:10D8D8007B4B07EB840703EB44135B7B023D7860CB
:10D8E8000121BB602046EDB202F0D4FC012D764E3A
:10D8F80001D8022300E004233355BDE8F081704AC3
:10D908006301D11802204873F0E0002800F09981E3
:10D91800204602F041FD6D4B43F82400042380E1CA
:10D92800674A6301D1180120487303E1002E00F013
:10D938008881204602F0E6FD062372E1604B002153
:10D9480003EB441359732046596802F0E1FB0722A0
:10D9580021E1002E40F075812046314602F0D8FBC7
:10D96800574B204603EB44135968494202F0D0FB59
:10D97800082210E1002E00F06481204602F00CFD20
:10D9880000210646204602F0C3FB504B002553F801
:10D9980024202046921B43F82420494B03EB4413D0
:10D9A80059685D7302F056FC2046314602F00AFCC5
:10D9B8002046294602F06EFC0922ECE0204602F0DF
:10D9C80057FD002800F03D810021204602F0A0FB11
:10D9D800033D0121204602F05DFCEDB2002002F07B
:10D9E80059FF012D07D82046012102F053FC344B82
:10D9F80003EB4413C9E00E22CDE0002E00F0218194
:10DA0800D6E0002E40F01D81204602F0C5FC3146CC
:10DA18000546204602F07CFB294B022103EB441308
:10DA28005E7395FBF1F1204602F0CCFB20463146AF
:10DA380002F030FC0D22AEE0204602F019FD00286D
:10DA480000F0FF80ECE007EB84031D4A996802EBC5
:10DA5800441251732046596802F0FCFB0023E0E0B1
:10DA6800194F3B5D013B0E2B00F2EB80DFE813F012
:10DA78000F003000440054006900E9007A00E90012
:10DA8800E9009700A2008500C500DC00D000204610
:10DA980002F0A8FC0A4B07EB840703EB44135B7BFB
:10DAA80078600121BB60204602F0F4FB062D01D00E
:10DAB800082D01D102226EE004226CE0040000204F
:10DAC8009C4C0020000C02403C480020644C002084
:10DAD800062D5D4B4FEA441202D19A18022103E049
:10DAE800082D02D19A1800215173620199582046D5
:10DAF80002F00EFB03224EE06B1FDBB2012B05D8B0
:10DB080020B1062D514B26D1042245E0B8F1000F73
:10DB180000F097800C2384E0052D4B4B4FEA44120C
:10DB280002D19A18012103E0072D02D19A18002189
:10DB38005173620199582046494202F0E9FA0522D8
:10DB480029E06B1FDBB2012B07D836B1052D3F4BFF
:10DB580001D1022220E00F221EE0B8F1000F70D0A0
:10DB680007235EE0B8F1000F6BD1374B022203EBBD
:10DB780044135A73204659680AE0B8F1000F60D17F
:10DB8800314B012203EB44135A735968204649422A
:10DB980002F0BEFA0A222D4B1A55BDE8F081B8F101
:10DBA800000F4ED0204602F0F7FB07EB8403D86045
:10DBB8000B2336E0B8F1000F43D1204602F0ECFB0E
:10DBC800214B224D03EB44135968064683F80D8018
:10DBD800204602F03FFB05EB8403D9680223761840
:10DBE80096FBF3F1204602F0EDFA2046414602F09A
:10DBF80051FB0D232B55BDE8F081204602F038FC7F
:10DC0800F8B10E2300203B55BDE8F04102F042BEBA
:10DC18002046012102F03EFB2046002102F078FA5E
:10DC28000E233B55BDE8F08107EB8403064A99684B
:10DC380002EB441251732046596802F00BFB002393
:10DC48003B55BDE8F08100BF9C4C00203C480020BB
:10DC5800024B1A5C0AB901221A5470473C4800204A
:10DC6800024B1A5C0AB10F221A5470473C48002034
:10DC7800014B185C704700BF3C480020034B002054
:10DC88001870034B997AFAF7C7BB00BFFB4C00200A
:10DC98009C4C0020014B1878704700BF4C4800206E
:10DCA800014B5878704700BF4C480020014B9878CA
:10DCB800704700BF4C4800202DE9F3416E4BDA78DD
:10DCC80022B96FF000425A600122DA701C7A5CB9FE
:10DCD800E0B2FAF702FC684B03F10902A0540134E0
:10DCE800082CF5D101221A72644FDFF8B081644E16
:10DCF80027240025E8B2FAF7F0FBEB5D834216D043
:10DD0800AB1CE85508EB83035B68022B05D0032B9B
:10DD180008D0012B0BD150B104E040B9325D012A83
:10DD280005D103E0335D012B01D1022333550135C1
:10DD38000134082DDED1534C637E23B94E4B587CF9
:10DD480002F0EAFB30B9637E4B4C7BB1607C02F099
:10DD5800E3FB58B9484B9A7C52B901229A74484B54
:10DD6800DA7E012A04D10222DA7601E00023A374C4
:10DD7800444C637E23B9404B587C02F0D5FB30B944
:10DD8800637E3D4C7BB1607C02F0CEFB58B93A4BC8
:10DD9800DA7C52B90122DA74394B1A7F012A04D18C
:10DDA80002221A7701E00023E374364EF36993B137
:10DDB800354C25787DB9FAF73DFA344B1B68C01A03
:10DDC800F3690028B8BF4042984204D9284602F0B7
:10DDD80099FB012323702B4E336A93B12C4C257881
:10DDE8007DB9FAF727FA2B4B1B68C01A336A00284B
:10DDF800B8BF4042984204D9284602F083FB012369
:10DE080023700820FBF780FA63281B4C01D80123F4
:10DE180005E00820FBF778FA692801D90023637028
:10DE28000820FBF771FA40F212239842124C01D9EC
:10DE3800012306E00820FBF767FAB0F5027F01D25C
:10DE4800002323700920FBF75FFA78280A4C01D9D0
:10DE5800012305E00920FBF757FA592801D80023C8
:10DE6800A3706178044A0C4B19B9117809B99278F2
:10DE7800B2B104221A8315E04C480020554800200E
:10DE8800044D002004000020F94C0020F44C002030
:10DE9800604C0020EC4C002000100240C04C0020D8
:10DEA80004225A835C4C02F007FE607C02F0B8FA48
:10DEB8000146607C002942D0584B02221A54FCF7D4
:10DEC800BFF8637C564A02EB4312517AB0EBD10F8C
:10DED80002D01846FAF7A0FA4F4C00232375607C4D
:10DEE80002F0C6FA70B1627C4E49D31CC85C0128A6
:10DEF80001D10220C854012101FA02F2464B197DD2
:10DF08000A431A754849494A0B7843B14248007D8B
:10DF1800034204D11370464B1B7803B90B70137876
:10DF28003BB13D4A127D1A409A4202D1414B01222F
:10DF38001A70002002B0BDE8F041FFF76DBC384D03
:10DF48003D4F05EB401393F80CE03C4A83003C4EF0
:10DF5800BEF1000F08D0121800923618FB180A46B6
:10DF68000196FCF7FBF87AE1F9181218331802F059
:10DF78006DFA607C02F0CEF930BBFAF75BF9637C8E
:10DF88000A2104EB8304626805EB4315801AAA8B07
:10DF98000028B8BF40424A43904271DD1F4AD25C14
:10DFA8001AB9284AD25C002A6AD01D4A184602EBE0
:10DFB8004312917AFAF730FA174B18495B7C002222
:10DFC800CA542049CA545BE0607C05EB4013DB7FF0
:10DFD800002B39D002F09EF90646607C02F082F9E7
:10DFE8000E4A8642607C174B125C0DD0032A02D180
:10DFF8001B5C002B3AD005EB4015E97FFAF70CFAC9
:10E00800054B03215B7C2FE0022A01D11B5C6BB31B
:10E0180005EB4015697A22E04C480020FB4C0020B3
:10E028009C4C0020044D00207F4C00207E4C00209A
:10E03800684C0020334D0020804C0020704C00209C
:10E04800994C0020F84C0020864B1B5C022B02D117
:10E05800854B1B5C53B1854B03EB4013597AFAF798
:10E06800DBF9834B02215B7C7E4AD154804C7E4B8A
:10E07800657C00225A55FAF7DDF804EB85046060E8
:10E088007B4C7A4D607C05EB40139B69E3B1FAF752
:10E09800FDFAC8B1607C02F03DF9637C0028B8BF86
:10E0A800404205EB4315AA6990420DD9184602F083
:10E0B80029FA637C6F4A0121D1546F4A0F33D15C2E
:10E0C800012901D10221D154694C00232375607CB8
:10E0D80002F0CEF970B1627C6749D31CC85C012894
:10E0E80001D10220C854012101FA02F2604B197DC6
:10E0F8000A431A756149624A0B7843B15C48007D4E
:10E10800034204D113705F4B1B7803B90B7013786B
:10E11800574A33B1117D1940994202D15A4B012116
:10E128001970507C02F0F6F8514C18B9607C02F076
:10E13800D9F818B1657C554B5B5D2BB3637C4B4AB2
:10E1480002EB4312D28912B9504AD35C13B3FAF7DF
:10E1580071F8474C0A21637C04EB83029269801AA8
:10E16800424A0028B8BF404202EB4312D2894A43D0
:10E1780090420FDD464DEA5C62B91846FCF756F846
:10E18800637C0122EA5405E0FAF754F8384B03EBB4
:10E198008505A861364C3F4D607C02F0BBF802460D
:10E1A800607C002AB8BF524255F830309A420AD2F1
:10E1B800FBF714FF637C05EBC3056A7982420DD136
:10E1C8001846002108E0FBF709FF637C05EBC3054F
:10E1D8006979884202D01846FBF7D8FEFAF72AF880
:10E1E800234CE369C01A0028B8BF40420A2836DD2C
:10E1F800607CFFF711FB607C02F08CF820B3607C38
:10E208001A4D05EB40135B69002B1DDD02F0C4F8C5
:10E218000646607CFAF744FA637C361A05EB431528
:10E228006A69002EB8BF764296420DDD184602F0A4
:10E2380069F9637C184A0121D1540F4A1533D15C1E
:10E24800012901D10221D154094C637C0133DBB28D
:10E2580063740BB100236374F9F7ECFFE06102B05B
:10E26800BDE8F081FB4C0020F84C00209C4C0020BD
:10E278004C480020984C0020044D00207F4C002082
:10E288007E4C0020684C0020334D0020FC4C0020C0
:10E29800FD4C0020744C00207D4C0020084B186871
:10E2A800024604E02C2902D100221A7004E01178F9
:10E2B800134601320029F5D1014A01331360704732
:10E2C8006C48002010B50B4C6368A268934208D2D2
:10E2D800E218127B013302700120636084F84C005D
:10E2E80010BD04F10C00FCF767F9A0600020606025
:10E2F80010BD00BF6C48002010B5094C0A46236DBC
:10E30800E11881F85400591C0D28216502D03F29D5
:10E3180000D822B90348FCF735F90023236510BD5E
:10E328006C480020C048002010B50121044686B082
:10E338002020FFF7E1FF002C04DA2D200121FFF750
:10E34800DBFF644200230A2100E0034694FBF1F25C
:10E3580001FB124401A830341C54581C141EF4DC70
:10E368001C4601ABE05C0121FFF7C6FF14F1FF3446
:10E37800F7D206B010BD2DE9F74304460DF10700AA
:10E38800FFF7A0FF002800F0C380934B934A93F84F
:10E39800941019BB51789DF80700403188420DD17F
:10E3A800D3F89810002940F0B380012183F8941025
:10E3B800117931F0010140F0AB80A7E00D2801D0C0
:10E3C8001B2802D10022844B05E0D3F898207E2A2E
:10E3D80000F29E800132C3F8982099E0117931F05B
:10E3E800010103D19DF80700FFF786FF9DF807306C
:10E3F800794D1F2B0AD9D5F898207E2A77D8A918E5
:10E40800013281F89C30C5F8982070E0082B07D1BC
:10E41800D5F89830002B6AD0013BC5F8983066E0F3
:10E428000D2B64D1D5F89830002B60D06B4B1A793E
:10E43800112A16D1587801214030C0B2FFF75CFF8D
:10E44800002605F19C0704E0F05D0121FFF754FF69
:10E458000136D5F898309E42F6D30D200121FFF7FA
:10E468004BFF5D490023C1F81C31D1F898700D6845
:10E478001A46184601F590789C4627E001280DD0E9
:10E4880002D3022821D117E0554E965D202E1CD0CC
:10E49800C81880F820610133012016E0504E965DBF
:10E4A800202E0DD1012B03D9C81880F820C10133C3
:10E4B80008EB0305022008E0494E965D202E04D0A3
:10E4C80001EB030989F8206101330132BA42D5D141
:10E4D800414A0021C2F81C31D31883F820110123C6
:10E4E800156082F89F3182F89410C2F898109DF850
:10E4F80007301B2B0CD1384B0021C3F8981083F838
:10E508009410364B1B79012B02D10D20FFF7F4FE36
:10E51800314B93F89F01002858D00026DFF8E0809F
:10E5280083F89F6135464FF0070909FB05872D4899
:10E53800394608F0B3FE28B9BE797B79F107237014
:10E5480034D508E016F80830002B41D001350736DD
:10E55800FF2DEAD13CE0FFF7A1FE23780546042B06
:10E568000BD1214908F09AFEF8B128461F4908F056
:10E5780095FE68B128461E490EE00D2B13D11D49A2
:10E5880008F08CFE88B128461B4908F087FE08B9B8
:10E59800012305E01949284608F080FE10B9022336
:10E5A800637003E0284608F05FFE6070B20704D588
:10E5B800FFF774FE08F058FEA070730705D5FFF743
:10E5C8006DFE08F051FEC4F803000120BDE8FE838B
:10E5D80000232370F9E700BF6C48002004000020E6
:10E5E800084900208C4900209D910108A19101084B
:10E5F800A5910108AB910108B1910108B6910108F4
:10E60800E07B010838B50C4D0446A878012140305C
:10E61800C0B2FFF771FE687801214030C0B2FFF741
:10E628006BFE2078FFF780FE6068FFF77DFE0D2007
:10E638000121BDE838405FE60400002038B500221B
:10E6480004460D46C0F347110220FAF71FFDE1000A
:10E6580041F006010022C9B20220FAF717FD210A8B
:10E6680021F01F01002241F010010220FAF70EFDEF
:10E67800E9B200220220FAF709FD290A0220012244
:10E68800BDE83840FAF702BD10B5C0F3471104469B
:10E6980000220220FAF7FAFCE10041F0060100220C
:10E6A800C9B20220FAF7F2FC210A21F01F01002268
:10E6B80041F00C010220FAF7E9FCFF2100220220B8
:10E6C800FAF7E4FC00210A460220FAF7DFFCFF21F2
:10E6D800044601220220FAF7D9FC44EA002080B25D
:10E6E80010BD38B500220C460546C0F3471102207C
:10E6F800FAF7CCFCE90041F006010022C9B2022079
:10E70800FAF7C4FC290A21F01F01002241F0100188
:10E718000220FAF7BBFCE1B200220220FAF7B6FCAD
:10E72800C4F3072100220220FAF7B0FCC4F3074122
:10E7380000220220FAF7AAFC210E02200122BDE8DD
:10E748003840FAF7A3BC70B5C0F34711044600225D
:10E758000220FAF79BFCE10041F006010022C9B251
:10E768000220FAF793FC210A21F01F01002241F050
:10E778000C010220FAF78AFCFF2100220220FAF796
:10E7880085FC00210A460220FAF780FC0021054694
:10E798000A460220FAF77AFC002104460A460220BB
:10E7A800FAF774FCFF21064601220220FAF76EFCF4
:10E7B800360446EA0060284340EA042070BDF8B5F4
:10E7C80004460E461546002A2AD0C0F347110022F7
:10E7D8000220FAF75BFCE10041F00601C9B2002211
:10E7E8000220FAF753FC210A21F01F0141F0100121
:10E7F80002200022FAF74AFC00246F1E05E0315D72
:10E8080002200022FAF742FC0134BC42F7D3751902
:10E8180015F8011C02200122BDE8F840FAF736BCC1
:10E82800F8BD70B504460E46154662B3C0F34711ED
:10E8380000220220FAF72AFCE10041F00601C9B2E1
:10E8480000220220FAF722FC210A21F01F0141F0E0
:10E858000C0100220220FAF719FC0220FF210022F5
:10E86800FAF714FC0024013D05E000210A46FAF7F6
:10E878000DFC305501340220AC42F6D3FF210122B1
:10E88800FAF704FC705570BD38B5002204460D46F1
:10E89800C0F347110220FAF7F9FBE10041F0040147
:10E8A8000022C9B20220FAF7F1FB02202946012210
:10E8B800BDE83840FAF7EABB10B5C0F34711044683
:10E8C80000220220FAF7E2FBE10041F003010022F6
:10E8D800C9B20220FAF7DAFBFF2100220220FAF778
:10E8E800D5FB0220FF210122BDE81040FAF7CEBB7C
:10E8F80010B54FF40060FFF7C7FE134C206040F6D8
:10E908000200FFF7C1FE606040F60800FFF7BCFE9A
:10E91800A06040F60A00FFF7B7FEE0604FF4016020
:10E92800FFF7B2FE206140F61200FFF7ADFE60610E
:10E9380040F61800FFF7A8FEA06140F61A00FFF79E
:10E94800A3FEE06110BD00BF0C4A002008B50A4BC9
:10E95800196A596293F828300BB141F0100189B255
:10E968004FF49870FFF76AFE4FF49A700021BDE8E3
:10E978000840FFF763BE00BF0C4A002008B50A4BE9
:10E988000122596A83F82820196241F0100189B2DE
:10E998004FF49870FFF752FE4FF49A701121BDE8BA
:10E9A8000840FFF74BBE00BF0C4A002008B50B4BD0
:10E9B80001225A6283F8282011214FF49870FFF73A
:10E9C8003DFE00214FF49A70FFF738FE4FF40170B6
:10E9D8004FF60E71BDE80840FFF730BE0C4A002024
:10E9E8002DE9F84F4FF40870FFF74EFEC00719D510
:10E9F8004FF49070FFF748FE994B00F00F02C106E4
:10EA08001A620FD593F8282062B10024998C4FF42C
:10EA1800987083F82840FFF711FE4FF49A7021464A
:10EA2800FFF70CFE8E4B5A6A013A072A36D8DFE800
:10EA380002F004110B1C353535261B6A022B11D048
:10EA4800032B26D0012B03E01B6A012B21D0032BBB
:10EA580022D123E01B6A022B20D0042B02D0012BE9
:10EA68001AD116E0FFF744FF13E01B6A013B072B9E
:10EA780012D8DFE803F00E0E11131111110E1B6AE4
:10EA8800013B072B08D8DFE803F004040704070755
:10EA98000709FFF75BFF01E0FFF770FF704C636A3F
:10EAA800012B00F0DF814FF40870FFF7EDFDC20580
:10EAB80040F14D81636A032B40F03781694E4FF472
:10EAC800805031464FF48672FFF7ABFE3378757885
:10EAD800B77903EB0525063D022F11D10026E66222
:10EAE800304602F051FB4FF48033E3625E4B06225E
:10EAF8001A700823E36326636663A663042323E08E
:10EB0800236BE06AEB1883420ED9B0F5802F06D24A
:10EB180002F03AFBE36A03F58033E36204E040F273
:10EB28000A73A363052306E04D4B5049186B2A4628
:10EB380002F074FA04234A4A116B69181163494AAE
:10EB48001178494A063911704649474A48789371FD
:10EB5800507088784E239070C8781373D0700879F5
:10EB680072231071537348792E2300249373202342
:10EB7800032F5071D471D37340F0C780384E01F120
:10EB88000C08D6F834E0F36BD6F838C0A146104626
:10EB98008A46403672E018F8011B8E44002B6CD070
:10EBA800052B05D92F2916D939290DD8013B64E041
:10EBB80005D12F290FD9392906D804235DE0042B64
:10EBC80002D1562947D148E0032B04D12F2942D935
:10EBD80039294DD93FE0022B04D12F293BD93929B6
:10EBE80048D938E0012B36D12F2934D9392932D8E0
:10EBF80018F8013C1C4FD37482F81490611D00234F
:10EC08000B29D4BF13F806B011F80AB0013387F8FE
:10EC18000CB001310137072BF2D1137B312B05D111
:10EC2800537B332B02D1937B312B25D00523837162
:10EC38003A23037546234375612383756923C37596
:10EC48006C2303762123437680F81A9040F2777C70
:10EC58004FF4FA5311E008230FE003230DE000BF3F
:10EC68000C4A0020AC570020B8580020B8570020A4
:10EC7800022302E0012300E000230134AC428AD3DE
:10EC8800794AFF2DC2F834E0D363C2F838C00AD9F4
:10EC9800191DC3F108004D19002B36D07349002304
:10ECA80040326D182FE093B9D36AB3F5802F03D2A1
:10ECB8004FF4403002F068FA04226D486D4902F0C2
:10ECC800ADF96D486D49042202F0A8F91DE0082B42
:10ECD8001BD86B4B0521997140F2767191634922DB
:10ECE8001A736E225A7376229A736122DA736C222F
:10ECF8001A7469225A7464229A740022DA7404E03D
:10ED0800E95C995401338342FAD1574A5C49936BC1
:10ED1800180A4872180C0B728872180E0133C872E0
:10ED2800936341F20C1020220FE0214631F8470B83
:10ED38006268FFF776FD04F1470004F14F01FEF722
:10ED480079FA2089E26804F14F01FFF738FD464C53
:10ED5800636A082B40F0868040F61400FFF794FCA5
:10ED6800C3057FD56269208A2C2A28BF2C2204F18A
:10ED78005801FFF756FDA36D022B05D0032B07D0D2
:10ED8800012B0BD1042000E0012000210A4602E0FB
:10ED980005200E210022E36DFEF71EFA00210A4627
:10EDA8000B460620FEF718FA2F4C0022C4F8840000
:10EDB800012113460620FEF70FFA0022C4F8880046
:10EDC800E92113460620FEF707FA0022C4F88C0052
:10EDD800D12113460620FEF7FFF90022C4F890005F
:10EDE800022113460620FEF7F7F90022C4F8940022
:10EDF800032113460620FEF7EFF90022C4F8980015
:10EE0800832113460620FEF7E7F90022C4F89C0088
:10EE1800122113460620FEF7DFF97B21C4F8A00073
:10EE2800062000221346FEF7D7F90022C4F8A400F2
:10EE38000E2113460620FEF7CFF90022C4F8A800D9
:10EE4800E62113460620FEF7C7F9E269C4F8AC00CC
:10EE5800208B2C2A28BF2C2204F18401BDE8F84F0E
:10EE6800FFF7ADBCBDE8F88F0C4A0020AC57002076
:10EE7800F8FF03003C4A0020FCFF0300404A002042
:10EE8800B85800200000000003464FF6FF70834288
:10EE98004DDDB3F1807F27DBB3F1805F11DBB3F188
:10EEA800804F08DB394A93426FDC394A191652F809
:10EEB8002120120212E0364A991552F82120D20177
:10EEC8000CE0B3F1806F324A04DB191552F82120A7
:10EED800920103E0991452F821205201511C93FB2E
:10EEE800F2F28A1852101CE0B3F5801F284A0CDB96
:10EEF800B3F5800F04DB191452F82120120110E039
:10EF0800991352F82120D2000BE0B3F5802F04DBCF
:10EF1800191352F82120920003E0991252F8212087
:10EF28005200501C93FBF2F2801840101EE0FF2B99
:10EF380022DDB3F5805F164A0BDBB3F5804F03DBA8
:10EF4800191252F8210010E0991152F821004010CE
:10EF58000BE0B3F5806F04DB191152F82100801023
:10EF680003E0991052F82100C010013000FB00F2B4
:10EF78009A420ADD01387047002B04DB044A52F834
:10EF88002300001170474FF0FF3070470080FE7F6C
:10EF9800C07C01081D4B5A7E1D4BD2B9597BCB074B
:10EFA80009D51C4B1B69180705D51B4B1868002889
:10EFB800BCBF1A605A608B0726D5164B1B69D8064A
:10EFC80022D5154B1A68002A1EDD00221A605A60E5
:10EFD80070475A7BD1070AD50E4B196911F0080101
:10EFE80005D10D4B18680028BCBF196059609307FC
:10EFF8000AD5084B1A6912F0100205D1064B196898
:10F008000029C4BF1A605A60704700BF040000207E
:10F018009C4C002000040240BC4A002038B51A4B22
:10F0280005461A7A62B1FBF70FF9184B2846597A48
:10F03800F9F7F2F9164A00231370164A137038BD0F
:10F048005A7A12B1012A1DD10FE01C68D4B9DA68C6
:10F058001B699A4216D0FBF7F7F80C4B2846597AE9
:10F06800F9F7DAF90A4B1C7038BD1C6854B95B69AA
:10F0780043B1FBF7E9F8054B2846597AF9F7CCF97B
:10F08800034B1C7038BD00BFBC4A00209C4C0020BC
:10F09800FD4C0020F458002008B50020FBF746F886
:10F0A800A8B9FAF7CDFF013005F02EFF14A3D3E974
:10F0B800002305F08FFF14A3D3E9002306F0B4F86A
:10F0C8000022154B05F086FF06F01EFA08BD002049
:10F0D800FAF7B6FF013005F017FF0DA3D3E90023B7
:10F0E80005F078FF08A3D3E9002306F09DF8002275
:10F0F800094B05F06FFF06F007FA08BDAFF3008073
:10F1080049922449924CB1401B0DE02D90A0F63F46
:10F1180024499224496AA2400000A03F684620F092
:10F1280007018D4631B5194CA36973B118480121FF
:10F1380003F02AFA0028F9D01548A56903F0EBF97D
:10F14800C5F10305C0B264192077104CA369022BDE
:10F158000BD8A3690E48C3F10202A218013392F832
:10F168002010A36103F0DAF90CE0002208487121AD
:10F1780003F0FCF9074B10221A83002384F824308B
:10F1880084F82530BDE8314085467047BC4A0020E8
:10F198000030014000000240684620F007018D461B
:10F1A8002DE9F14F012184B04FF0804003F00FFFAB
:10F1B800002800F0FF8601214FF0804003F012FF85
:10F1C800914B9A6A122A10D9012283F82C20002226
:10F1D8009A628E4B1A6801321A608D4B1B783BB9C4
:10F1E8008C4B1A6801321A6002E09A6A01329A62FC
:10F1F800854B1A6B22B1012283F83420002201E0EA
:10F208001A6B01321A630020F9F7E4FC0020F9F7C1
:10F2180047FA0390039B7C4CA36394F82C30002B93
:10F2280060D07B4B1B78002B48D0039AE36BD31A32
:10F23800002BB8BF5B42082B764B26DD1968226C81
:10F24800914222D0039A62641B68A364606CE36BEA
:10F25800A76CC01A06F08AFA266C0546B81B06F099
:10F2680081FA0146284606F089FB05F05FFE64A393
:10F27800D3E9002305F0AEFE06F046F9664B1860A8
:10F28800636CE363A36C23640CE019685E4B1A6C2F
:10F298008A1A002AB8BF5242642A03DD5E49002256
:10F2A8000A60DA64584B5C4AD96CD86C1268821AC6
:10F2B800102092FBF0F28A1ADA6413E0534A1268BB
:10F2C800642A554A05DD1360E364544B08221A800A
:10F2D80008E0E16CE06C13681022C31A93FBF2F3A8
:10F2E800CB1AE364484C237A062B00F0F98094F893
:10F2F8003420002A00F0FA85032B00F0F785637AA2
:10F30800002B35D1E2682369D31A236594F8543069
:10F3180013B9A36DE3650EE0E0682369C01A0028FD
:10F32800B8BF4042FFF7B0FD0546206E4000FFF72A
:10F33800ABFD4543E565344BD9681A69914207DD51
:10F34800D96D9A6D9142B4BFDA6D9A6D5A6112E027
:10F35800D9681A69914207DAD96D9A6D9142B4BF9A
:10F36800DA6D9A6D5242F1E700225A611A6002E0A2
:10F378006FF000432365244B19685A6991427DD088
:10F38800596E1A6E8A185A665A6E12149A66596E0F
:10F398009A6E12048A1A5A6693F854200AB95A695E
:10F3A8001A60194B19685A69914209DA1868996EF6
:10F3B8005A694118914211DA1A689B6ED3180EE007
:10F3C80019685A6991420CDD1868996E5A69411A90
:10F3D800914203DD1A689B6ED31A00E05B690A4A02
:10F3E8001360094BDA6E002A4BDD5A69C2B91868F6
:10F3F800D96E0028B8BF4042884242DA1CE000BFFC
:10F408000000000000408F40BC4A0020F058002057
:10F41800544C0020EC580020E8580020FE580020EA
:10F428005A69002A1A4613DD1968002906DD18688A
:10F43800D96E884202DADA6E1A6022E01268A14BAD
:10F44800002A1EDA1968DA6E5242914219DDF2E793
:10F458005969002915DA1968002904DA1868D96E7B
:10F468004942884207DC1268964B002A09DD196870
:10F47800DA6E914205DADA6E5242DDE700225A6608
:10F488009A66904C8F4D226F2368D3182367236F99
:10F498001B146367626F236D002AB8BF5242002BAA
:10F4A800B8BF5B429A42C4BF236D6367226F636F24
:10F4B8001B04D31A23672269636FD3182361FFF7EC
:10F4C80069FDA36F062B05D8EA6F696FAB6F01FA68
:10F4D80003F301E0EB6F6A6FD318EB6700F006BD2A
:10F4E80094F82C30002B3ED0E26CD4F88030002AFF
:10F4F800B8BF52429A4233DDD4F88400E36CD4F8A2
:10F508008050002BB8BF5B425B1B4343D4F8881084
:10F51800D4F880208A1A93FBF2F3C4F88C30E36C99
:10F52800002B04DAD4F88C305B42C4F88C30654B7D
:10F53800D3F88C10D3F884209142C4BFD3F8842028
:10F54800C3F88C20D3F88C10D3F884305D4A5B4222
:10F55800994208DAD2F884305B42C2F88C3002E073
:10F568000023C4F88C30574B93F83420002A00F05D
:10F578003583554A1578002D40F0D4825A7A022AEC
:10F5880000F06B82D3F890109A6D914256DDD3F853
:10F598009410D3F89820891A4C4A11605B68002BA4
:10F5A800134602DA126852421A601A68002A02DA0E
:10F5B800464A002111601968424BD3F89C209142B9
:10F5C80002DA424A00211160404A1268D3F8A0309A
:10F5D80082FB0323002A73F1000104DAFF200021D3
:10F5E800121843EB0103120A42EA0362354BD3F8BF
:10F5F80090509B6DED1A364BAA425B69D8BF22EA40
:10F60800E275002B1ADD314A12689A4216DD2D4B3D
:10F6180000225A611A60C3F8A4205A60D3F89820CF
:10F62800C3F89420D3F89820DA602A4B01221A7084
:10F63800294B5A7D012A01D102225A75214C637A3D
:10F64800002B4FD1E268D4F89830D31A236594F888
:10F6580054301BB9A36D5B19E3650FE0E068D4F87B
:10F668009830C01A0028B8BF4042FFF70DFC064684
:10F67800206E4000FFF708FC4643E665114BD96849
:10F68800D3F89820914209DDD96D9A6D52199142AB
:10F6980001DADA6D0EE09A6D551910E0D968D3F8E1
:10F6A800982091421ADAD96D9A6D5219914203DA6B
:10F6B800DA6D52425A6118E09A6D55196D425D61D2
:10F6C80013E000BFBC4A0020F4580020E058002096
:10F6D8009C4C00207D4C0020044D002000225A61E3
:10F6E8001A6002E06FF000432365924B19685A696B
:10F6F80091426CD0596E1A6E8A185A665A6E121454
:10F708009A66596E9A6E12048A1A5A6693F85420A9
:10F718000AB95A691A60874B19685A69914209DA15
:10F728001868996E5A694118914211DA1A689B6EE5
:10F73800D3180EE019685A6991420CDD1868996E61
:10F748005A69411A914203DD1A689B6ED31A00E088
:10F758005B69784A1360774BDA6E002A3ADD5A699A
:10F768003AB91868D96E0028B8BF4042884231DAE1
:10F778000BE05A69002A1A4613DD1968002906DDCC
:10F788001868D96E884202DADA6E1A6022E01268C6
:10F79800684B002A1EDA1968DA6E5242914219DD66
:10F7A800F2E75969002915DA1968002904DA186896
:10F7B800D96E4942884207DC12685E4B002A09DD8F
:10F7C8001968DA6E914205DADA6E5242DDE70022F4
:10F7D8005A669A66574B574C196F1A688A181A67EF
:10F7E8001A6F12145A67596F1A6D0029B8BF494227
:10F7F800002AB8BF52429142C4BF1A6D5A67196FA6
:10F808005A6F12048A1A1A67D3F898105A6F8A180E
:10F81800C3F898205B7A002B42D1E268D4F8943080
:10F82800D31AC4F8A83094F854301BB9A36DC4F89F
:10F83800AC3010E0E068D4F89430C01A0028B8BFA3
:10F848004042FFF721FB0546206E4000FFF71CFBF6
:10F858004543C4F8AC50374BD968D3F8942091424B
:10F868000ADDD3F8AC109A6D9142B4BFD3F8AC203E
:10F878009A6DC3F8A42017E0D968D3F89420914270
:10F8880009DAD3F8AC109A6D9142B4BFD3F8AC2022
:10F898009A6D5242EDE70022C3F8A4205A6003E0B3
:10F8A8006FF00043C4F8A830224B5968D3F8A4205D
:10F8B800914200F08480D3F8B0101A6E8A18C3F809
:10F8C800B020D3F8B0201214C3F8B420D3F8B01085
:10F8D800D3F8B42012048A1AC3F8B02093F854203D
:10F8E80012B9D3F8A4205A60124B5968D3F8A4204F
:10F8F80091420CDA5868D3F8B410D3F8A420411810
:10F90800914219DA5A68D3F8B430D31816E0596816
:10F91800D3F8A420914213DD5868D3F8B410D3F873
:10F92800A420411A914207DD5A68D3F8B430D31A9B
:10F9380004E000BFBC4A0020D3F8A4308E4A5360CC
:10F948008D4BDA6E002A3FDDD3F8A4203AB9586807
:10F95800D96E0028B8BF4042884235DA0CE0D3F8A7
:10F96800A420002A1A4613DD5968002906DD5868C4
:10F97800D96E884202DADA6E5A6025E052687E4B08
:10F98800002A21DA5968DA6E524291421CDDF2E708
:10F99800D3F8A410002917DA5968002904DA58683E
:10F9A800D96E4942884207DC5268734B002A0BDD46
:10F9B8005968DA6E914207DADA6E5242DCE70022C1
:10F9C800C3F8B020C3F8B4206B4CD4F8B8206368EF
:10F9D800D318C4F8B830D4F8B8301B14C4F8BC3005
:10F9E800D4F8BC20D4F8A830002AB8BF5242002B63
:10F9F800B8BF5B429A42C4BFD4F8A830C4F8BC3040
:10FA0800D4F8B820D4F8BC301B04D31AC4F8B830E2
:10FA1800D4F89420D4F8BC30D318C4F89430FFF745
:10FA2800B9FAD4F898202369D31AC4F8C0302269E7
:10FA3800D4F8C030D318236123690399039AFF329D
:10FA4800934204DCA1F1FF029A42B8BF1A464A4B1E
:10FA58001A611A69C3F898206EE0D3F8C420002A06
:10FA680001DDFF2205E0D3F8C420002A04DA6FF094
:10FA7800FE02C3F8C02001E0C3F8C0503F4B597ED6
:10FA88003F4B5B7BC9B9DE070AD53E4A12691507A9
:10FA980006D5394AD2F8C4000028B8BFC2F8C01049
:10FAA8009C0726D5374B1B69D80622D5324BD3F88D
:10FAB800C420002A1DDD002219E0D9070BD5314AE0
:10FAC800126912F0080106D12B4AD2F8C4000028A6
:10FAD800B8BFC2F8C0109A070BD52A4B1B6913F0A0
:10FAE800100206D1244BD3F8C410002901DDC3F855
:10FAF800C020214B1969D3F8C0208A181A611969E6
:10FB08000398039AFF32914204DCA0F1FF028A4273
:10FB1800B8BF0A461A611A69DA601A69C3F89820E8
:10FB28001A6907E000225A611A60C3F8A4205A60D3
:10FB3800D3F89820C3F894200F4B134ADC68106858
:10FB48000399201A884227DA0399D868126882181C
:10FB5800914221DA0D4A1168002903DD1368013B3F
:10FB6800136020E00A4901220A70D3F89410DB6878
:10FB7800994218D1074B15E0BC4A00200400002028
:10FB88009C4C00200004024000590020E45800204A
:10FB9800FC580020F4580020BF4B1A68BF4B1A606D
:10FBA800BF4B00221A70BF4BBF4A0398DC6811682C
:10FBB800611A884205DB0399D86812688218914255
:10FBC80002DDBA4A002111705B7A012B03D0B54BD4
:10FBD8005B7A022B02D1B54B00221A70B14A039905
:10FBE8001369C2F8C830B14B187820B1B04B1C6803
:10FBF800B04B186800E00A24D2F8C860D2F8CC509C
:10FC0800A84B75196D1AC2F8D050D2F8D050C2F866
:10FC1800D450D2F8D050D2F8D820002DB8BF6D42B9
:10FC2800954232DCD3F8D02042B3D3F8D060D3F871
:10FC3800D0507443D3F8DC200A26AA1A94FBF6F4B1
:10FC480000FB0240C3F8D400D3F8D400D3F8D8207E
:10FC58009042C4BFD3F8D820C3F8D420914BD3F82E
:10FC6800D400D3F8D8205242904204DAD3F8D820EE
:10FC78005242C3F8D420D3F8D42001E0D3F8D020DE
:10FC88008918C3F8E010874B15E0D3F8D000D3F8F3
:10FC9800D8205242904203DAD3F8D820891A08E0D3
:10FCA800D3F8D000D3F8D82090420DDDD3F8D8206F
:10FCB8008918C3F8E010D3F8E010D3F88C208A181C
:10FCC8009205920DC3F8E420764CD4F8D03026463D
:10FCD800C4F8DC30D4F8E430E367637A022B32D11D
:10FCE800FFF7DAF9D4F8C43005468342C8BFC4F830
:10FCF800C400D4F8C42043429A42B8BF694A694C48
:10FD0800B8BFC2F8C430D4F8C4000028B8BF404215
:10FD180005F02CFD0646284605F028FD014630462C
:10FD280005F02CFE05F002F959A3D3E9002305F0EC
:10FD380051F905F0E9FBFF28A8BFFF20C4F8E80047
:10FD4800C4F8EC00D2E0D4F8F030002B00F0CA8000
:10FD5800D4F8F430D4F8F80023B1D4F8FC30D4F84F
:10FD6800D4B003E0D4F8FC30D4F8D0B00130C01AD5
:10FD780005F0FCFCD4F80061BBF1000FB8BFCBF173
:10FD8800000B0546C6EB0B0005F0F0FCD4F804A107
:10FD9800D4F8F8700646C7EB0A0005F0E7FCD4F87B
:10FDA8000891D4F800810746C8EB090005F0DEFC8D
:10FDB8000146384605F0E2FD0146304605F02AFDC9
:10FDC8000146284605F01EFC05F074FE354BC4F8C4
:10FDD800E800D3F8E810D3F8F8209142BCBFD3F874
:10FDE800F820C3F8E820D3F8E800D3F804112D4A26
:10FDF8008842C4BFD2F80411C2F8E810D3F80C3115
:10FE0800284A002B04DDD2F80C31013BC2F80C3132
:10FE1800244AD2F81031002B04DDD2F81031013B0E
:10FE2800C2F81031D2F8E810D2F8EC201D4B9142FC
:10FE38001DDDD3F814211AB3D3F80C21002A55D1AB
:10FE4800D3F8EC10D3F8FC208A18C3F8EC20D3F8C8
:10FE5800EC10D3F804219142C4BFD3F80421C3F8AD
:10FE6800EC20104BD3F81421C3F80C213EE0D3F852
:10FE7800E810D3F8EC20914238DAD3F81821DAB92F
:10FE8800D3F8E820C3F8EC2030E000BFAFF30080DF
:10FE98000000000000E06F40F8580020E4580020FF
:10FEA800FC580020BC4A002004590020F4580020C7
:10FEB800105900200C590020D3F81021B2B9D3F8FA
:10FEC800EC00D3F81C11884204DBD3F8EC10D3F80B
:10FED8001C218A1AC3F8EC20394BD3F81821C3F82F
:10FEE800102103E0D4F80431C4F8EC30344B93F813
:10FEF8002520002A58D193F82021002A54D193F8BC
:10FF08002420002A40D19A6F062A07D8DA6F2D4993
:10FF1800920501EB1252D2F800240CE09A6FD96FC7
:10FF2800072A294A01F00F0102EB81020CBFD2F81F
:10FF38000823D2F848231A62214B1A7A062A26D1B6
:10FF480093F8202001920199D3F8EC205143FF2225
:10FF5800B1FBF2F10191196A4908196293F821106D
:10FF680002910298D3F8EC104143B1FBF2F20292ED
:10FF7800029AD2B283F821201A6A52001A62019AB0
:10FF8800D2B283F8202002E0D3F824211A620F4B62
:10FF980010225A830A4B0021012283F825200C489D
:10FFA8009961712102F0E2FA054B002283F82C20B6
:10FFB80083F8342004B0BDE8F14F8546704700BF90
:10FFC800BC4A0020C07C0108B88D0108000002402E
:10FFD80000300140F8B5464B464A5D6AA3F57043C8
:10FFE8005B6A00211360444B1960444B42F2107164
:08FFF8001E881068B6B28842B1
:020000040801F1
:1000000007DD198889B2082903D91988C1F34E017F
:1000100019801368B3F57A7F0ADA3A4B1A8892B2DC
:10002000B2F5804F04D21A8892B2520092B21A806E
:10003000314C0821204602F0CEFF98B12F4B2046CC
:100040001A68082152421A6002F0D0FF2D4B1A881C
:1000500092B2AA1AE2631B8801229BB2EB182364B6
:10006000294B9A82244C1021204602F0B4FF78B12B
:100070002046102102F0BAFF224B1A8892B2AA1A27
:10008000E2631B8801229BB2ED181F4B25649A8204
:100090001A4B30461C6805F06DFB04F04BFF14A3AF
:1000A000D3E9002304F09AFF064620460F4605F0E8
:1000B00061FB04F03FFF02460B463046394605F02F
:1000C000B7F8124B044618680D4604F033FF024699
:1000D0000B462046294604F081FF05F019FA0C4A28
:1000E0000C4B1278186012B11A6852421A60F8BDAF
:1000F00000000000006AF84000040140EC580020B5
:10010000F0580020FE580020001400404C4C002005
:10011000484C0020E858002010B50446084605F079
:1001200029FB04F007FF08A3D3E9002304F056FFDE
:1001300005F0EEF9064B58615A692046C3F8A42031
:10014000BDE81040FEF76EBF2D431CEBE2361A40AF
:10015000BC4A002010B50446084605F00BFB04F02D
:10016000E9FE09A3D3E9002304F038FF05F0D0F934
:10017000074B18601A6820465A60BDE81040FEF729
:1001800051BF00BFAFF300802D431CEBE2361A4095
:10019000BC4A002008B581EAE170A0EBE17005F0EF
:1001A000E9FA04F0C7FE06A3D3E9002304F016FF22
:1001B00005F0AEF9044BD86608BD00BFAFF3008070
:1001C0002D431CEBE2361A40BC4A0020054B0022AE
:1001D0001A70054B1A7A12B1044A1268891AD9604A
:1001E000FEF720BFF4580020BC4A00200859002028
:1001F000084B10B51A7A0C4632B10020F8F754FAC1
:10020000054B241A1C6010BD1961BDE81040FEF7B3
:1002100009BF00BFBC4A00200859002010B50446A1
:1002200081EAE170A0EBE17005F0A4FA04F082FE2F
:1002300007A3D3E9002304F0D1FE05F069F9064BCA
:1002400018662046BDE81040FEF7ECBEAFF3008014
:100250003A8C30E28E794540BC4A002010B5044605
:1002600081EAE170A0EBE17005F084FA04F062FE2F
:1002700007A3D3E9002304F0B1FE05F049F9064BCA
:1002800098652046BDE81040FEF7CCBEAFF3008075
:100290002D431CEBE2361A40BC4A0020022902D84A
:1002A000024BC9B25972FEF7BDBE00BFBC4A002066
:1002B000054B1A7A19B12AB901221A727047062A17
:1002C00008BF1972704700BFBC4A0020014B83F879
:1002D00054107047BC4A0020082903D8024BC1F1D2
:1002E00008019967704700BFBC4A002008B50A4B57
:1002F000586905F03FFA04F01DFE05A3D3E9002379
:1003000004F096FF05F004F908BD00BFAFF30080CC
:100310002D431CEBE2361A40BC4A002008B50A4BBC
:10032000186805F027FA04F005FE05A3D3E90023B9
:1003300004F07EFF05F0ECF808BD00BFAFF30080CD
:100340002D431CEBE2361A40BC4A0020014BD86C0E
:10035000704700BFBC4A002008B5094BD86E05F0B5
:1003600009FA04F0E7FD04A3D3E9002304F060FFD9
:1003700005F0CEF808BD00BF2D431CEBE2361A4055
:10038000BC4A0020044B1A7AD8681AB1034B1B6888
:10039000C0187047704700BFBC4A002008590020B1
:1003A000044B1A7A18691AB1034B1B68C0187047BE
:1003B000704700BFBC4A00200859002008B50A4B0E
:1003C000186E05F0D7F904F0B5FD05A3D3E90023B5
:1003D00004F02EFF05F09CF808BD00BFAFF30080CD
:1003E0003A8C30E28E794540BC4A002008B50A4B71
:1003F000986D05F0BFF904F09DFD05A3D3E9002336
:1004000004F016FF05F084F808BD00BFAFF30080CC
:100410002D431CEBE2361A40BC4A0020014B587AAF
:10042000704700BFBC4A0020024B187A003018BF4A
:1004300001207047BC4A0020014B93F854007047DC
:10044000BC4A0020024B986FC0F10800C0B2704750
:10045000BC4A002010B50748C469200911B1E40C5A
:1004600064010C6012B1C0F38421117003B11870E3
:1004700010BD00BFBC4A0020074B1A7A062A08D0DC
:100480001869DB68C3EB000CDCF1000040EB0C00EA
:100490007047024B18787047BC4A0020FC58002077
:1004A000B4235843024900F580700422F9F7F9B8E3
:1004B0001C4B0020B4235843024900F582700422EB
:1004C000F9F7EFB8144B0020B4235843024900F564
:1004D00084700422F9F7E5B8284B002002494FF454
:1004E00080700422F9F76EB91C4B002002494FF4CA
:1004F00082700422F9F766B9144B002002494FF4C8
:1005000084700422F9F75EB9284B0020034B0122C6
:100510005A7200225A611A60704700BFBC4A00201C
:10052000024B186900F00800C0B270470004024096
:10053000024B186900F01000C0B27047000402407E
:1005400010B5044659B101214FF08040002202F05D
:100550002DFD20460021BDE81040F9F79DBD012189
:10056000F9F79AFD01214FF080400A46BDE810409E
:1005700002F01CBD4FF08043988900F001007047E5
:10058000074A92F82400064B0028FAD10122C3F84A
:10059000241183F8242093F82420002AFBD17047EB
:1005A000BC4A0020014BC3F8D8007047BC4A002069
:1005B000014BD3F8D8007047BC4A0020014BC3F868
:1005C000CC007047BC4A0020014BD3F8CC007047E8
:1005D000BC4A0020034B187AA0F10603584240EBB6
:1005E00003007047BC4A0020014BC3F8F800704775
:1005F000BC4A0020014BC3F804017047BC4A0020EC
:10060000014BC3F800017047BC4A0020014BC3F8FE
:1006100008017047BC4A0020014BC3F8FC0070473A
:10062000BC4A0020014BC3F81C017047BC4A0020A3
:1006300032235843014BC3F814017047BC4A0020D1
:1006400032235843014BC3F818017047BC4A0020BD
:10065000014BC3F8F0007047BC4A0020014BC3F8BF
:1006600080007047BC4A0020014BC3F888007047E7
:10067000BC4A0020014BC3F884007047BC4A0020EC
:10068000014B1860704700BFF8580020014B1860FC
:10069000704700BF00590020014B1860704700BF31
:1006A00010590020014B1860704700BF0C59002002
:1006B000014B1860704700BF04590020014BD3F86C
:1006C000F8007047BC4A0020014BD3F80401704782
:1006D000BC4A0020014BD3F800017047BC4A0020FF
:1006E000014BD3F808017047BC4A0020014BD3F8F6
:1006F000FC007047BC4A0020014BD3F81C01704736
:10070000BC4A0020034BD3F81401322390FBF3F0D2
:10071000704700BFBC4A0020034BD3F818013223B6
:1007200090FBF3F0704700BFBC4A0020024BD3F8A7
:10073000F000C0B2704700BFBC4A0020014BD3F8A4
:10074000EC007047BC4A0020014BD3F8E80070472A
:10075000BC4A0020014BD3F8D0007047BC4A0020AF
:10076000014BD3F8E0007047BC4A0020014BD3F89E
:10077000E4007047BC4A0020014BD3F8800070476A
:10078000BC4A0020014BD3F888007047BC4A0020C7
:10079000014BD3F884007047BC4A0020014BD3F8CA
:1007A0008C007047BC4A0020014B1868704700BF9E
:1007B000F8580020014B1868704700BF005900200E
:1007C000014B1868704700BF10590020014B186892
:1007D000704700BF0C590020014B1868704700BFDC
:1007E00004590020014BD3F8C0007047BC4A0020D8
:1007F000014BC3F8A0007047BC4A0020014BD3F85E
:10080000A0007047BC4A002008B50028B8BF40428D
:1008100004F0B0FF04F08EFB05A3D3E9002304F03D
:10082000DDFB04F075FE044BC3F8900008BD00BF6B
:100830002D431CEBE2361A40BC4A002008B50A4B97
:10084000D3F8900004F096FF04F074FB04A3D3E9FE
:10085000002304F0EDFC04F05BFE08BDAFF3008064
:100860002D431CEBE2361A40BC4A0020014BC3F872
:100870009C007047BC4A0020014BD3F89C00704795
:10088000BC4A0020014BC3F8F4007047BC4A00206A
:10089000014BD3F8F4007047BC4A0020084B10B558
:1008A0000446187A30B10020F7F7FEFE054B241AF3
:1008B0001C6010BD2146BDE81040F7F70FBF00BF18
:1008C000BC4A00200859002008B50020F7F7ECFECC
:1008D000014B1B68C01808BD08590020014BC3F824
:1008E000C4007047BC4A0020014BD3F8C4007047D5
:1008F000BC4A002038B51D4C237A062B04D00020BA
:100900000121FFF7CBFC27E0637A012B24D002D32F
:10091000022B2AD126E020682368256E80FB030184
:100920002A46EB1705F010F902460B46C90F52187C
:1009300043F100035B104FEA32022368D4F89810A9
:10094000002B0B4B1B681944CCBF8918C2EB01016B
:100950000020BDE8384039E400200146BDE83840B9
:10096000FFF7DABB0023C4F8C43038BDBC4A00200E
:1009700008590020014BC3F828017047BC4A0020E9
:10098000014BD3F828017047BC4A002038B5114C00
:10099000237A062B14D10020FFF7A8FCD4F82821D5
:1009A000E36C801A984212DC0020E56CFFF79EFC95
:1009B000D4F82831C0188542CCBF0020012038BDB2
:1009C00020686369C21A504240EB020038BD002023
:1009D00038BD00BFBC4A002010B50A20F8F798FCCB
:1009E00004460B20F8F794FC404304FB0400BDE8E8
:1009F0001040FEF74DBA034BD3F89400024B1B682E
:100A0000C0187047BC4A00200859002008B50A4B9E
:100A1000D3F8A40004F0AEFE04F08CFA04A3D3E9EA
:100A2000002304F005FC04F073FD08BDAFF3008063
:100A30002D431CEBE2361A40BC4A002008B50A4B95
:100A4000586804F097FE04F075FA05A3D3E9002373
:100A500004F0EEFB04F05CFD08BD00BFAFF30080C6
:100A60002D431CEBE2361A40BC4A0020094B1A7A8F
:100A70002AB983F82C2107221A7201207047062A0E
:100A800005D10120072283F82C011A72704700203B
:100A9000704700BFBC4A0020014B93F82D017047FE
:100AA000BC4A0020054B1A682AB95869D0F10100E8
:100AB00038BF002070470020704700BFBC4A0020AC
:100AC00070B5A94C237A013B082B00F24B81DFE87B
:100AD00013F009002D006A004700590049019700F2
:100AE000BE00E9000020FFF781FCC4F830010020BF
:100AF000FFF764FC4FF44841C4F834010020FFF7CD
:100B0000ADFB4FF448410020FFF788FB0025002093
:100B1000FFF7FCFC25612846E560FEF783FAF7F74E
:100B20008DFBE567C4F8380102238EE0F7F786FBFA
:100B3000D4F838318C4DC01A0028B8BF4042B0F507
:100B4000FA7F40F30F8100200146F7F7C7FD4FF40D
:100B500080630020EB600146FFF7A0FB04239FE0C9
:100B60000020FFF789FC002800F0FC800020F7F748
:100B70009BFD7D4B0022A0F58060C3F8CC00DA60BD
:100B800005220EE00020FFF777FC002800F0EA8045
:100B90000020FFF7BBFCF7F751FB734B0322C3F8B0
:100BA00038011A7270BDF7F749FBD4F838316E4D31
:100BB000C01A0028B8BF4042B0F5FA7F40F3D28097
:100BC00000200146F7F78AFD0020F7F76DFD286148
:100BD0002B690024EB60EB682046C5F89830EB6881
:100BE000D5F83011C5F89430604B1C60FFF736FB28
:100BF0002046D5F83411FFF711FB6C7206234FE045
:100C00000020FFF7F3FBC4F830010020FFF7D6FB0C
:100C10004FF44841C4F834010020FFF71FFB4FF4A4
:100C200048410020FFF7FAFA0020FFF76FFC4F4A17
:100C30000023E3672361E3601360012384F82D310F
:100C4000F7F7FCFA0823C4F83801237270BDF7F7F0
:100C5000F5FAD4F83831444DC01A0028B8BF4042E4
:100C6000FA287FDD424B00241969204621F02F41EC
:100C70001961404B090E1C70F7F7C0FD20464FF478
:100C80008031F7F763FD20462146F7F727FD3A4B01
:100C900020461B6821461B02EB60FFF7FFFA092381
:100CA0002B7270BD0020FFF7E7FB00285AD0002010
:100CB000F7F7FAFC0028044608DA00200121F7F7CC
:100CC0009DFD2B4B1A6942F080721A6184EAE4722E
:100CD000A2EBE472294B00246FF0C705C82012E094
:100CE00091FBF5F68E1996420CDC91FBF0F68E190D
:100CF000B24207DC0020F8F7D7F81B4B022283F83A
:100D00002D2105E0013453F8041FB1F1FF3FE7D175
:100D10001B4B53F82430144C013305D1002384F8C5
:100D20002C31032384F82D3100250020FFF7EEFB42
:100D3000256128462946E560F7F7D0FC94F82C3168
:100D400028465B1B18BF0123D4F83011237284F8A6
:100D50002C51FFF783FAD4F834112846BDE87040CF
:100D6000FFF75CBA70BD00BFBC4A002008590020E4
:100D70009C4C0020514C0020444C0020B800002026
:100D8000BC0000207FB5234D234C08262E80636ACB
:100D90002988204689B2591A01F008FF636A298818
:100DA000204689B2C91801F003FF204631460122CE
:100DB00002F0FCF801221021204602F0F7F82E2361
:100DC0000124164D8DF80C3003A802238DF80D3048
:100DD0008DF80E408DF80F4002F0D4F92146202006
:100DE00001F09AF9284601F071FC4FF6FF73019368
:100DF0004FF41673ADF80030284600236946ADF86D
:100E00000830ADF8023001F00BFD2846214601F014
:100E10009CFD7FBDFE5800200004014000140040EE
:100E20007FB50020FFF75AFB0020FFF75FFB002093
:100E3000FFF764FB3F4B0026FF220F213E48C3F81B
:100E4000D8200124C3F8CC60C3F8EC10C3F8F81024
:100E50000A21C3F80421C3F80061C3F80821C3F8CC
:100E6000FC40C3F81C41C3F81461C3F81861C3F80F
:100E7000F040C3F8F44083F8544001602F486425E3
:100E800006602F4802602F4805602F4835460160F4
:100E90004FF4FA61C3F8A0104B21C3F89C102B4902
:100EA0002046C3F89010C3F88420294A2146C3F88D
:100EB0008020284AC3F888204FF4FA72C3F828210A
:100EC00001F02AF94FF0804001F000FC40F6B83301
:100ED00069464FF080400193ADF80060ADF80860BE
:100EE000ADF8026001F09CFC224621464FF08040A4
:100EF00002F05CF821464FF0804001F026FDFFF73C
:100F000041FF1C2303A88DF80C308DF80D408DF89F
:100F10000E408DF80F4002F035F9232303A88DF819
:100F20000C308DF80D608DF80E408DF80F4002F0FA
:100F300029F97FBDBC4A0020105900200C5900201F
:100F40000459002000590020F8580020703D0A0084
:100F500020A10700804F120038B5012204460D463B
:100F600003200621F8F796F8052100220320F8F760
:100F700091F8032000210122F8F78CF88307F3D5BC
:100F800010F08C0F26D0012100220320F8F782F800
:100F9000032000210122F8F77DF80521002203201B
:100FA000F8F778F8032000210122F8F773F8C10759
:100FB000F3D4032006210122F8F76CF80521002262
:100FC0000320F8F767F8032000210122F8F762F800
:100FD0008207F3D5022100220320F8F75BF8C4F35F
:100FE000074100220320F8F755F8C4F30721002237
:100FF0000320F8F74FF8E1B200220320F8F74AF88F
:10100000032029460122F8F745F805210022032094
:10101000F8F740F8032000210122F8F73BF8C30756
:10102000F3D438BD2DE9F84304468946174603201A
:1010300006210122F8F72EF8052100220320F8F7F7
:1010400029F8032000210122F8F724F88107F3D5BD
:1010500010F08C0F26D0012100220320F8F71AF897
:10106000032000210122F8F715F8052100220320B2
:10107000F8F710F8032000210122F8F70BF8C20757
:10108000F3D4032006210122F8F704F805210022F9
:101090000320F7F7FFFF032000210122F7F7FAFFF3
:1010A0008307F3D5022100220320F7F7F3FFC4F3EF
:1010B000074100220320F7F7EDFFC4F307210022C8
:1010C0000320F7F7E7FFE1B203200022F7F7E2FF82
:1010D00000257E1E4CE001345FFA84F819F80510F3
:1010E000B8F1000F06D0C6EB050EDEF1000242EBB0
:1010F0000E0200E00122D2B20320F7F7CBFFB8F1D5
:10110000000F34D1B54232D2052100220320F7F777
:10111000C1FF032000210122F7F7BCFFC007F3D471
:10112000032006210122F7F7B5FF05210022032045
:10113000F7F7B0FF032000210122F7F7ABFF81078B
:10114000F3D5022100220320F7F7A4FFC4F30741DF
:1011500000220320F7F79EFFC4F30721002203209B
:10116000F7F798FFE1B203200022F7F793FF01356C
:10117000BD42B0D1052100220320F7F78BFF0320E9
:1011800000210122F7F786FFC207F3D4BDE8F883F8
:1011900010B50621044601220320F7F77BFF052145
:1011A00000220320F7F776FF032000210122F7F742
:1011B00071FF8107F3D510F08C0F26D0012100229A
:1011C0000320F7F767FF032000210122F7F762FFF2
:1011D000052100220320F7F75DFF032000210122F3
:1011E000F7F758FFC207F3D4032006210122F7F7CF
:1011F00051FF052100220320F7F74CFF03200021B7
:101200000122F7F747FF8307F3D5D82100220320F7
:10121000F7F740FFC4F3074100220320F7F73AFF36
:10122000C4F3072100220320F7F734FFE1B20320C3
:101230000122F7F72FFF052100220320F7F72AFFED
:10124000032000210122F7F725FFC007F3D410BDCA
:1012500008B5032006210122F7F71CFF0521002213
:101260000320F7F717FF032000210122F7F712FFF1
:101270008107F3D510F08C0F26D001210022032026
:10128000F7F708FF032000210122F7F703FF0521EC
:1012900000220320F7F7FEFE032000210122F7F7CA
:1012A000F9FEC207F3D4032006210122F7F7F2FE6C
:1012B000052100220320F7F7EDFE03200021012283
:1012C000F7F7E8FE8307F3D5032060210122F7F743
:1012D000E1FE052100220320F7F7DCFE03200021B8
:1012E0000122F7F7D7FEC007F3D408BD10B50446B6
:1012F000032000220146F7F7CDFEC4F30741002288
:101300000320F7F7C7FEC4F3072100220320F7F7F5
:10131000C1FEE1B200220320F7F7BCFE032000214A
:101320000122BDE81040F7F7B5BEF8B5044603202A
:1013300015460F4600220146F7F7ACFEC4F30741FD
:1013400000220320F7F7A6FEC4F3072100220320A2
:10135000F7F7A0FEE1B203200022F7F79BFE00247E
:101360006E1E09E0A01B424242EB00020320002156
:10137000F7F790FE38550134AC42F3D1F8BD704711
:10138000FEE7FEE7FEE7FEE77047704770477047ED
:101390002E4B82B01A6842F001021A6000229A6055
:1013A000196821F0847121F480311960284959604D
:1013B000196821F480211960DA60009201921A689C
:1013C00042F480321A601A6802F400320192009AE4
:1013D00001320092019A1AB9009AB2F5A06FF2D1C7
:1013E0001A4B1B6813F4003318BF01230193019BB0
:1013F000012B25D1154B9A689A609A6842F40042F5
:101400009A609A6842F4A0529A60124A5A601A6826
:1014100042F080721A6019680C4A8901FBD50E4BA4
:1014200040F203711960936823F00303936093689B
:1014300043F002039360936803F00C03082BFAD186
:10144000064B074A9A6002B0704700BF003802405E
:1014500010300024081E4005003C024000ED00E072
:1014600000800008154B16499868164A00F00C00D9
:10147000042801D0082801D00A6013E05868596890
:101480005B6801F03F01C3F38813B2FBF1F25A43EA
:101490000A4B5B68C3F3014301335B00B2FBF3F219
:1014A000074B1A60054B9A68054BC2F303129A1852
:1014B0001279196821FA02F21A6070470038024066
:1014C000040100200024F400012108B54FF48070CD
:1014D00000F06AFE4FF480700021BDE8084000F083
:1014E00063BE43680A6823F0407323F48073134398
:1014F0000A7930B543EA02234360CA680B698468FD
:101500008D681A43084B2A43234013434A7943EA20
:10151000420383600B7DC26A013B22F47002DBB29E
:1015200042EA0353C36230BDFDF7FFC000230360EE
:10153000037143718360C3600361012303757047C6
:1015400010B5074A074B51680B4090E81200214341
:101550008468C068214301430B43536010BD00BF42
:1015600000230140E030FCFF002303604360836000
:10157000C3607047836811B143F0010301E023F0B9
:10158000010383607047436823F4400323F400732E
:10159000194341607047416282627047436823F09B
:1015A0001F03194341607047044B5A6810B142F45D
:1015B000000201E022F400025A607047002301405B
:1015C000044B5A6810B142F4800201E022F4800218
:1015D0005A60704700230140092970B54FF0030499
:1015E0000DD94C4307251E3C05FA04F503FA04F314
:1015F000C66826EA050545EA0304C4600BE04C43CF
:10160000072505FA04F503FA04F4066926EA050538
:1016100045EA04030361062A4FF005030CD8013A9A
:1016200053431F2202FA03F201FA03F3446B24EA44
:1016300002021343436370BD0C2A0DD853431F228B
:10164000233B02FA03F201FA03F1046B24EA0202DB
:1016500042EA0103036370BD53431F22413B02FA78
:1016600003F201FA03F1C46A24EA020242EA010326
:10167000C36270BD836843F08043836070478068B5
:10168000C0F380507047836811B143F4806301E078
:1016900023F4806383607047836811B143F00203D1
:1016A00001E023F00203836070474368013923F4AB
:1016B000604343EA413141607047436811B143F4EC
:1016C000006301E023F4006343607047C06C80B2A4
:1016D0007047014B1868704708230140836811B1B7
:1016E00043F4807301E023F4807383607047836860
:1016F00011B143F4007301E023F400738360704779
:10170000044B5A6810B142F4005201E022F4005236
:101710005A60704700230140092970B54FF0030457
:101720000DD94C4307251E3C05FA04F503FA04F3D2
:10173000C66826EA050545EA0304C4600BE04C438D
:10174000072505FA04F503FA04F4066926EA0505F7
:1017500045EA04030361836BC3F30154121B023295
:101760000524D2B262431F2404FA02F401FA02F102
:1017700023EA04030B43836370BD836B013923F4B5
:10178000401343EA01518163704782B00023019303
:101790000190019BC9180191019B1A6002B070472A
:1017A000836823F47023194381607047836823F4AE
:1017B0004013194381607047836843F4800383605A
:1017C00070478068C0F380507047436811B143F49C
:1017D000806301E023F4806343607047436811B184
:1017E00043F4805301E023F480534360704782B098
:1017F000002301930190019B283359180191019B0B
:10180000186880B202B070470123C9B203FA01F12F
:1018100043680AB1194301E023EA010141607047BE
:10182000036819420CBF002001207047C9430160C2
:1018300070474368006810EA112007D00122C9B23E
:1018400002FA01F119420CBF0020012070476FEA33
:1018500011210160704700BF036823F0010303609A
:101860000023036043608360C360036121234361FD
:101870002C4B98421CD02C4B984220D02B4B98429A
:1018800025D02B4B98422AD02A4B98422FD02A4B56
:10189000984233D0294B984237D0294B984204D1F3
:1018A0004FF03D5243F8AC2C7047264B984203D181
:1018B0003D2243F8082C7047234B984204D14FF443
:1018C000746243F8202C7047204B984204D14FF4A7
:1018D000741243F8382C70471D4B984204D14FF0D6
:1018E000746243F8502C70471A4B984203D11A4A3D
:1018F00043F8642C7047194B984203D1184A43F8B7
:101900007C2C7047174B984203D1174A43F8942C0C
:101910007047164B984204BF4FF03D5243F8AC2C31
:10192000704700BF106002402860024040600240E3
:10193000586002407060024088600240A06002402F
:10194000B8600240106402402864024040640240D3
:1019500058640240706402403D00002088640240E8
:10196000400F0020A064024000003D20B864024007
:101970000268134B10B51340CC680A6822434C69C7
:1019800022438C692243CC6922430C6A22434C6A6D
:1019900022438C6A22434C6B22438C6B22431343B9
:1019A000036042690C6BCB6A22F0070223431343A6
:1019B00043610B6943604B6883608B68C36010BDF3
:1019C0003F801CF00023036043608360C3600361B9
:1019D00043618361C361036243628362C3620363E1
:1019E000436383637047036811B143F0010301E06F
:1019F00023F0010303607047036811B143F400430F
:101A000001E023F4004303607047036811B143F021
:101A1000200301E023F0200303607047416070471A
:101A2000406880B27047036812B143F4002301E0BC
:101A300023F40023036001617047036811B143F48C
:101A4000802301E023F48023036070470AB1016121
:101A50007047C16070470068C0F3C04070470068BD
:101A600000F001007047406900F03800704710B581
:101A7000084A094B094CA0428CBF104618468B00FF
:101A8000074B4CBF426802680B4013420CBF00205A
:101A9000012010BD00640240006002400F6402405B
:101AA0007D0F7D0F10B5084B084A094CA0428CBF32
:101AB00010461846074B11F0005F01EA030314BFFC
:101AC000C360836010BD00BF00600240006402403C
:101AD0000F6402407D0F7D0F0B0607D5436912B1DD
:101AE00043F0800301E023F080034361802909D0A3
:101AF00001F01E01036812B119430160704723EA27
:101B0000010101607047104B10B5104A104CA04203
:101B10008CBF14461C460F4B0B402BB1026802F0E1
:101B20001E0202EAD12202E0426902F0800288002D
:101B3000094B4CBF606820680B40184002D0101C55
:101B400018BF012010BD00BF0060024000640240C9
:101B50000F6402403C0F3C0F7D0F7D0F10B5084B0A
:101B6000084A094CA0428CBF10461846074B11F09A
:101B7000005F01EA030314BFC360836010BD00BFB0
:101B800000600240006402400F6402407D0F7D0F40
:101B9000044B00221A605A609A60DA60024A5A6165
:101BA000704700BF003C0140FFFF7F00837910B504
:101BB000002B29D01A4B01681C68CA4314401C60D2
:101BC0005C6822405A60027902F1804202F59E323E
:101BD00014682143116002689C68D1430C409C60EA
:101BE000DC682140D9604179102906D199681143F8
:101BF0009960D9680A43DA6010BD01F1804303F5AA
:101C00009E3319680A4308E00379016803F18043B1
:101C100003F59E331A6822EA01021A6010BD00BF64
:101C2000003C014000230C22036003714271837168
:101C30007047024B1A69104318617047003C01401D
:101C4000034B5B6918420CBF00200120704700BFA6
:101C5000003C0140014B5861704700BF003C01400F
:101C6000054B1A685B69034004D010420CBF00208A
:101C70000120704718467047003C0140014B5861F5
:101C8000704700BF003C014008B52C4B984205D17D
:101C90000120014600F058FA012048E0284B984204
:101CA00005D10220012100F04FFA02203FE0254B30
:101CB000984205D10420012100F046FA042036E0C4
:101CC000214B984205D10820012100F03DFA08205F
:101CD0002DE01E4B984205D11020012100F034FA6E
:101CE000102024E01A4B984205D12020012100F059
:101CF0002BFA20201BE0174B984205D140200121F0
:101D000000F022FA402012E0134B984205D18020C7
:101D1000012100F019FA802009E0104B98420BD104
:101D20004FF48070012100F00FFA4FF48070002111
:101D3000BDE8084000F008BA08BD00BF000002403E
:101D40000004024000080240000C02400010024063
:101D50000014024000180240001C02400020024013
:101D60002DE9F0470023D1F800801A464FF0010C0E
:101D700003270CFA02F404EA0805A54231D107FA58
:101D800003F40668E443264006600E79D0F800901C
:101D900006FA03FA013EF6B24AEA0909012EC0F832
:101DA000009015D891F80590866809FA03F9264045
:101DB0008660866849EA06068660466826EA050562
:101DC00045608D79466805FA02F5ADB23543456048
:101DD000C5682C40C460CC79C56804FA03F42C4370
:101DE000C46001320233102AC3D1BDE8F0874FF638
:101DF000FF7303600023037143718371C3717047E4
:101E000082B04FF480330193019B0B430193019BFC
:101E1000C361C161019BC361C3690193C36901933C
:101E200002B07047036919420CBF002001207047BF
:101E3000006980B27047436919420CBF002001203D
:101E40007047406980B27047018370474183704793
:101E50000AB101837047418370474161704743690C
:101E600059404161704701F0070330B59B000F24D2
:101E700004FA03F402FA03F3C908083150F82150B8
:101E800025EA040440F8214050F82140234340F85B
:101E9000213030BD0A4B1A6842F001021A6000225C
:101EA0009A60196821F0847121F480311960054924
:101EB0005960196821F480211960DA60704700BF09
:101EC0000038024010300024024B00221A701870B3
:101ED000704700BF02380240034B1A6822F0F80234
:101EE00042EAC0001860704700380240014B186099
:101EF000704700BF00004742064B002201281A70BD
:101F00001A7002D0042804D101E01870704705222D
:101F10001A70704770380240014B1860704700BF5C
:101F2000800E4742014341EA8212009942EA016170
:101F30005A08013A024B41EA02425A60704700BF18
:101F400000380240014B1860704700BF60004742F4
:101F50008001034B40EA0170C3F88400704700BF62
:101F600000380240014B1860704700BF68004742CC
:101F7000014B1860704700BF4C004742034B9A6802
:101F800022F0EC621043084398607047003802402A
:101F9000034B9A6822F078421043084398607047D8
:101FA00000380240034B9A6822F003021043986005
:101FB000704700BF00380240024B986800F00C00E8
:101FC000704700BF00380240034B9A6822F0F002CD
:101FD00010439860704700BF00380240034B9A6876
:101FE00022F4E05210439860704700BF003802406E
:101FF000034B9A6822F4604242EAC000986070473E
:102000000038024010B51A4B1A4A996801F00C01C9
:10201000042913D0082911D15C6859685B6801F064
:102020003F01C3F38813B2FBF1F25A43104B5B68D4
:10203000C3F3014301335B00B2FBF3F20C490260CE
:102040008B680D4AC3F30313D35C046824FA03F3CB
:1020500043608C68C4F38224145D23FA04F4846022
:102060008968C1F34231525C23FA02F3C36010BDA8
:10207000003802400024F4001801002000F44073EE
:10208000B3F5407F084B08D1996820F0704221F4E5
:10209000F81122F440720A439A601A6F000542EA6E
:1020A00010501867704700BF00380240014B18609D
:1020B000704700BF3C0E4742014B1860704700BF9D
:1020C000400E4742014B1860704700BF5C01474219
:1020D000044B1A6B09B1104301E022EA00001863B7
:1020E000704700BF00380240044B5A6B09B11043DF
:1020F00001E022EA00005863704700BF0038024048
:10210000044B9A6B09B1104301E022EA0000986386
:10211000704700BF00380240044B1A6C09B11043ED
:1021200001E022EA00001864704700BF0038024056
:10213000044B5A6C09B1104301E022EA00005864D4
:10214000704700BF00380240044B1A6909B11043C0
:1021500001E022EA00001861704700BF0038024029
:10216000044B5A6909B1104301E022EA00005861AA
:10217000704700BF00380240044B9A6909B1104310
:1021800001E022EA00009861704700BF0038024079
:10219000044B1A6A09B1104301E022EA00001862F8
:1021A000704700BF00380240044B5A6A09B110431F
:1021B00001E022EA00005862704700BF0038024088
:1021C000044B1A6D09B1104301E022EA00001865C2
:1021D000704700BF00380240044B5A6D09B11043EC
:1021E00001E022EA00005865704700BF0038024055
:1021F000044B9A6D09B1104301E022EA0000986592
:10220000704700BF00380240044B1A6E09B11043FA
:1022100001E022EA00001866704700BF0038024063
:10222000044B5A6E09B1104301E022EA00005866DF
:10223000704700BF00380240044B1A7809B11043C0
:1022400001E022EA00001870704700BF0D3802401C
:102250004309012B074A01D1136803E0022B0CBF8D
:10226000136F536F00F01F0023FA00F000F001001D
:10227000704700BF0038024007B5002301933120AA
:10228000FFF7E6FF019B01330193019BB3F5A06FBC
:1022900001D00028F3D03120FFF7DAFF003018BF5B
:1022A00001200EBD024B5A6F42F080725A67704790
:1022B00000380240034BDB6818420CBF00200120AD
:1022C000704700BF00380240014B1870704700BFD4
:1022D0000E38024008B5154B98420BD101214FF43E
:1022E0008050FFF761FF4FF480500021BDE80840A7
:1022F000FFF75ABF0E4B984207D14FF4804001219F
:10230000FFF746FF4FF4804009E00A4B98420BD19B
:102310004FF400400121FFF73BFF4FF40040002144
:10232000BDE80840FFF734BF08BD00BF00300140E2
:1023300000380040003C00400B8810B54C880288F3
:1023400023438C8802F441522343CC8823430C89D5
:1023500023434C8923438C892343CC892343134350
:102360009BB20380838B23F400631B041B0C8383C9
:102370000B8A038210BD838BF0B523F47A6323F0BC
:102380001F031B041B0C8383022303848B68858B30
:10239000022BADB238D0294A8E889468002E14BF23
:1023A00002260126240203D5946824F400049460D4
:1023B000D2F88440D2F884705268DFF884C002F00A
:1023C0003F02BCFBF2F2C4F388145443C7F3027219
:1023D000B4FBF2F4CA88B2F5007F4FF00A0201D1D3
:1023E000240A02E07601B4FBF6F46243B2FBF3F395
:1023F00005330A229BB2B3FBF2F303F0010212028F
:10240000C3F34F0392B200E000229C1EA4B2FE2C44
:1024100028BF0022CC8828BF0223134323439BB24A
:1024200003840B884A882B4343F4006313438A8850
:1024300013438A8913439BB28383F0BD0038024063
:102440000024F4000023038043808380C380038141
:1024500043818381C38107230382704700230222C3
:10246000038043808380C3808260838170470388B8
:1024700019B19BB243F0400303E023F040031B0477
:102480001B0C03807047838B19B19BB243F48063AC
:1024900003E023F480631B041B0C838370470388D1
:1024A00023F400631B041B0C038003889BB21943B5
:1024B00001807047B1F5804F038803D19BB243F48C
:1024C000804303E023F480431B041B0C038070470C
:1024D0004FF6FF639942038803D09BB243F48073A5
:1024E00003E023F480731B041B0C03807047838874
:1024F00019B19BB243F0040303E023F004031B046F
:102500001B0C83807047838819B19BB243F0100382
:1025100003E023F010031B041B0C838070478089A9
:1025200080B2704781817047038819B19BB243F430
:10253000005303E023F400531B041B0C038070477B
:1025400003889BB243F4805303807047012902D073
:10255000008B80B27047808A80B27047008A80B258
:10256000704783889BB20AB1194301E023EA010155
:10257000818070470123090903FA01F1838889B238
:102580009BB20AB1194301E023EA0101818070473F
:10259000038919420CBF002001207047C94389B24A
:1025A00001817047012301F00F0203FA02F210B516
:1025B00084880089A4B280B2104006D0090903FAC9
:1025C00001F31C420CBF0020012010BD01F00F01DF
:1025D000012303FA01F3DB439BB20381704700BF81
:1025E000012108B54FF48040FFF7DEFD4FF4804035
:1025F0000021BDE80840FFF7D7BD014B18607047C8
:102600000038014001F0030230B592000F2404FAB3
:1026100002F400FA02F2074B8908023153F8215004
:1026200025EA040443F8214053F82140224343F8AB
:10263000212030BD00380140014B1860704700BFB9
:10264000DC002742014B1860704700BF000427429E
:10265000024B186AC0F30020704700BF00380140E9
:1026600030B5048C24F001042404240C0484058B6C
:10267000048CADB225F0F305A4B22A4342EA03125A
:1026800024F00A0343F0010392B219430283018448
:1026900030BD30B5058C25F010052D042D0C0584BA
:1026A000048B058C24F440742405240DADB244EA57
:1026B000022242EA033225F0A00343F0100343EA6A
:1026C000011192B289B20283018430BD08B5474B33
:1026D000984205D101200146FFF766FD01203DE04B
:1026E000B0F1804F05D101200146FFF751FD0120D7
:1026F00076E03F4B984205D102200121FFF748FDCB
:1027000002206DE03B4B984205D104200121FFF7E8
:102710003FFD042064E0384B984205D10820012198
:10272000FFF736FD08205BE0344B984205D11020BE
:102730000121FFF72DFD102052E0314B984205D1C9
:1027400020200121FFF724FD202049E02D4B984255
:1027500009D102200121FFF727FD02200021BDE859
:102760000840FFF721BD284B984207D14FF4803035
:102770000121FFF719FD4FF48030EFE7234B98421A
:1027800007D14FF400300121FFF70EFD4FF4003068
:10279000E4E71F4B984207D14FF480200121FFF757
:1027A00003FD4FF48020D9E71A4B984205D1402011
:1027B0000121FFF7EDFC402012E0174B984205D1B4
:1027C00080200121FFF7E4FC802009E0134B9842B0
:1027D0000BD14FF480700121FFF7DAFC4FF48070C9
:1027E0000021BDE80840FFF7D3BC08BD0000014050
:1027F0000004004000080040000C004000100040B1
:102800000014004000040140004001400044014029
:102810000048014000180040001C0040002000401B
:102820001C4A038890429BB212D002F5806290420B
:102830000ED0B0F1804F0BD0A2F58032904207D07D
:1028400002F58062904203D002F58062904203D18B
:102850004A8823F0700313430F4A904208D002F5D0
:102860008062904204D023F440730A899BB21343E0
:1028700003804B68C3620B880385064B984203D0E4
:1028800003F58063984201D18B7A0386012383820A
:10289000704700BF00000140001000404FF0FF33C0
:1028A0004360002303800381438083727047018566
:1028B00082827047038823F070031B041B0C0B43B8
:1028C0000380704741627047C1627047406A704739
:1028D000008D80B27047038819B19BB243F00203A8
:1028E00003E023F002031B041B0C038070470388E2
:1028F00019B19BB243F0040303E023F004031B046B
:102900001B0C03807047038819B19BB243F080030E
:1029100003E023F080031B041B0C03807047038833
:1029200023F008031B041B0C038003889BB219438C
:1029300001807047038823F440731B041B0C038041
:1029400003889BB2194301807047038819B19BB279
:1029500043F0010303E023F001031B041B0C03807D
:102960007047038C70B523F001031B041B0C038418
:10297000038C8488028B0D8822F073021204120CDF
:102980002A434E888D8923F002031B0435431B0C18
:10299000ADB22B430E4DA4B2A84203D005F580651D
:1029A000A8420ED1CD8923F008032B438D8823F054
:1029B00004032B434E8A0D8A24F440743543ADB290
:1029C0002C43848002838A684263038470BD00BF05
:1029D00000000140038C30B523F010031B041B0CD6
:1029E0000384038C8288048B0D8824F4E644240439
:1029F000240C23F0200344EA05241B048D891B0CBE
:102A000043EA05134D8892B243EA0513124DA4B26E
:102A1000A8429BB203D005F58065A84215D1CD89A7
:102A200023F080039BB243EA05134FF6BF751D40A8
:102A30008B8822F4406245EA03130D8A9BB242EA76
:102A400085024D8A42EA850292B282808A680483B6
:102A50008263038430BD00BF00000140038C30B5A9
:102A600023F480731B041B0C0384038C8288848BE7
:102A70000D8824F073042404240C23F400731B0435
:102A80002C438D891B0C43EA05234D8892B243EAFF
:102A90000523124D9BB2A84203D005F58065A842DC
:102AA00015D1CD8923F400639BB243EA05234FF689
:102AB000FF351D408B8822F4405245EA03230D8ADE
:102AC0009BB242EA05124D8A42EA051292B2828016
:102AD0008A688483C263038430BD00BF0000014064
:102AE000038C30B523F480531B041B0C0384038C2C
:102AF0008488828B0D8822F4E6421204120C23F49F
:102B0000005342EA05221B048D891B0C43EA05335E
:102B10004D88A4B243EA05330A4D92B2A8429BB253
:102B200003D005F58065A84205D10D8A24F48044C0
:102B300044EA8514A4B2848082838A680264038490
:102B400030BD00BF0000014000230380438083802C
:102B500083608381C38103824382704730B501243F
:102B600004FA01F4058C00F11803ADB225EA04045F
:102B7000048409B1082907D14908CC584FF68F7051
:102B80002040C850C8580AE00439C1F34E01CC585F
:102B900048F6FF702040C8501202C85892B2024353
:102BA000CA5030BD4163704781637047C16370474D
:102BB00001647047038B23F070031B041B0C0B4351
:102BC00003837047038B23F4E0431B041B0C43EA8D
:102BD00001239BB203837047838B23F070031B0494
:102BE0001B0C0B4383837047838B23F4E0431B044C
:102BF0001B0C43EA01239BB283837047038B23F0B2
:102C000008031B041B0C0B4303837047038B23F443
:102C100000631B041B0C43EA01239BB20383704730
:102C2000838B23F008031B041B0C0B438383704727
:102C3000838B23F400631B041B0C43EA01239BB228
:102C400083837047038B23F004031B041B0C0B438B
:102C500003837047038B23F480631B041B0C43EA3C
:102C600001239BB203837047838B23F004031B046F
:102C70001B0C0B4383837047838B23F480631B04FB
:102C80001B0C43EA01239BB283837047038B23F021
:102C900080031B041B0C0B4303837047038B090247
:102CA0005B0441EA534189B201837047838B23F06F
:102CB00080031B041B0C0B4383837047838B090227
:102CC0005B0441EA534189B281837047038C23F04E
:102CD00002031B041B0C0B4303847047038C23F07B
:102CE00008031B041B0C0B4303847047038C23F065
:102CF00020031B041B0C43EA01139BB2038470479F
:102D0000038C23F080031B041B0C43EA01139BB2CA
:102D100003847047038C23F400731B041B0C43EAE9
:102D200001239BB203847047038C23F400631B04CC
:102D30001B0C43EA01239BB203847047038C23F4EA
:102D400000531B041B0C43EA01339BB203847047FE
:102D5000012303FA01F302FA01F110B5048CA4B2C5
:102D600024EA03030384038C194389B2018410BD50
:102D7000042303FA01F302FA01F110B5048CA4B2A2
:102D800024EA03030384038C194389B2018410BD30
:102D900000230122038043808280C3800381704727
:102DA000406B7047806B7047C06B7047006C70471A
:102DB000038B23F00C031B041B0C0383038B9BB2BC
:102DC000194301837047038B23F440631B041B0CDE
:102DD0000383038B9BB243EA012189B201837047CD
:102DE000F8B50C4605464988A288208800290CBF02
:102DF00002270027012A14BF01260226238988B949
:102E00002846FFF72DFCE1882846FFF7D1FF28462A
:102E1000394623893246FFF73CFCE1882846BDE865
:102E2000F840D0E72846FFF734FCE1882846FFF752
:102E3000CAFF2846394623893246FFF711FCE1884C
:102E40002846BDE8F840B3E7838B23F00C031B044E
:102E50001B0C8383838B9BB2194381837047838BC5
:102E600023F440631B041B0C8383838B9BB243EAD4
:102E7000012189B2818370470B8870B50D460446E5
:102E80004988AA883BB92B89FFF7EAFBE9882046E5
:102E9000BDE870408CE7042B07D12B89FFF7F9FBC5
:102EA000E9882046BDE870408DE7082B2E89038C09
:102EB0001CD123F480731B041B0C0384808B238C94
:102EC00080B29BB220F0F30023F4206340EA0616A0
:102ED00043EA0121B6B289B2324341F48071A28340
:102EE0002184E9882046BDE87040ADE723F4805393
:102EF0001B041B0C0384808B238C20F4407023F470
:102F0000005300055B04000D5B0C40EA022243EA1B
:102F1000013342EA06329BB2E98892B243F480530D
:102F20002046A2832384BDE8704098E74A880B8836
:102F300013438A881343CA8813430A8913434A896F
:102F400013438A8913439BB2A0F84430704700238F
:102F5000038043808380C3800381438183817047E2
:102F6000B0F8443029B16FEA43436FEA53439BB250
:102F700001E05B045B0CA0F844307047838819B112
:102F80009BB243F0040303E023F004031B041B0C77
:102F900083807047838819B19BB243F0010303E03B
:102FA00023F001031B041B0C8380704783899BB2B1
:102FB0000AB1194301E023EA01018181704781824E
:102FC0007047038A19420CBF002001207047C94393
:102FD00089B201827047038A828911EA030092B2A2
:102FE00003D011420CBF002001207047C94389B2B1
:102FF000018270471143A0F84810704783899BB243
:103000000AB1194301E023EA0101818170478388F5
:1030100019B19BB243F0080303E023F008031B043B
:103020001B0C83807047038923F007031B041B0CD0
:1030300003817047038923F070031B041B0C0B43AF
:10304000038103899BB243F007030381704738B5BE
:103050000D4611460122602D044602D1FFF719FBEF
:1030600001E0FFF7FDFA238923F070031B041B0C1A
:103070001D43258123899BB243F00703238138BD7B
:10308000038923F070031B041B0C0B43038170475F
:10309000838823F070031B041B0C838083889BB2FE
:1030A000194381807047038923F007031B041B0C1D
:1030B000038103899BB2194301817047038923F07F
:1030C00080031B041B0C038103899BB219430181FC
:1030D000704710B50489E4B221430A4342EA03224F
:1030E00092B2028110BD10B50446FFF7F2FF2389AA
:1030F0009BB243F48043238110BD10B50446FFF713
:10310000E8FF238923F077031B041B0C43F07703AC
:10311000238110BD70B50589048B25F00705068C49
:103120002D0424F440742D0CB6B224F0030429437A
:10313000240426F02205240C2A4344F4807442EA35
:10314000031244F0010492B201810483028470BD31
:10315000838819B19BB243F0800303E023F080031E
:103160001B041B0C83807047A0F85010704700BFF1
:1031700040F0BE60024B40F42020D860704700BF92
:1031800000ED00E0C37810B503B3164B4278DB685E
:103190008478DB43C3F30223C3F10401C9B202FA0A
:1031A00001F10F2242FA03F2C9B222400A430E4B48
:1031B00001781201CB18D2B283F8002303780122E0
:1031C000590903F01F0302FA03F307E00378012211
:1031D000590903F01F0302FA03F32031024A42F8AF
:1031E000213010BD00ED00E000E100E021F0604181
:1031F00021F07F01014B08439860704700ED00E02B
:10320000044B1A6909B1104301E022EA0000186179
:10321000704700BF00ED00E0044B04281A680CBFA3
:1032200042F0040222F004021A60704710E000E04D
:10323000D0F8E83510B51B6904469847032384F895
:103240001231002010BD08B590F8123180F813310A
:10325000042380F81231D0F8E835DB689847002065
:1032600008BD08B5D0F8E435DB6903B19847002004
:1032700008BD08B5D0F8E4351B6A9847002008BDA2
:1032800008B5D0F8E4355B6A9847002008BDD0F84F
:10329000E83510B55B6904469847012384F8153179
:1032A000002010BDD0F8E83510B59B69044698475A
:1032B000D4F8E43520465B6800219847002084F864
:1032C000150110BD002110B5402204460B4601F047
:1032D0006BF9802140220023204601F065F901238B
:1032E00084F81231D4F8E835A0785B68984700205C
:1032F00010BD13B56946044600F078FA9DF8001039
:1033000001F01F03012B07D0022B0AD073B920460E
:10331000694600F015FB0FE02046694600F0F6FA1A
:103320000AE02046694600F091FA05E021F07F01AD
:10333000C9B2204601F0AAF900201CBD38B50446E8
:10334000002948D190F81131022B38D1D0F838211A
:10335000D0F824319A4211D9C178D21A0129C0F883
:10336000382104D1D0F82811CB18C0F8283192B2F6
:103370002046D4F8281100F0F3F920E0D0F83C21E1
:10338000B2FBF3F503FB152565B99A420AD3D0F8D1
:1033900040319A4206D229462A4600F0E1F9C4F8A3
:1033A00040510CE0D4F8E435DB682BB194F81221DD
:1033B000032A01D120469847204600F002FA94F8EB
:1033C0001631012B10D1094A236912685A60002373
:1033D00084F8163108E0D0F8E4355B6923B190F841
:1033E0001221032A00D19847002038BD145900202B
:1033F00010B5044659BB90F81131032B30D1D0F8E9
:103400009023D0F87C339A4214D9C178D21A01297A
:10341000C0F8902304D1D0F88013C918C0F88013E5
:103420009A4228BF1A4692B22046D4F8801300F080
:10343000B0F915E0D0F8E4351B6923B190F81221FA
:10344000032A00D19847204600F0ACF908E0D0F8F4
:10345000E4359B6923B190F81221032A00D19847E3
:10346000002010BD2DE9F041069F044616469846FF
:103470000D46F7F709F820462946C4F8E485C4F854
:10348000E875C4F8EC6501F041F8D4F8E8351B683C
:1034900098472046BDE8F041F7F748B8002070474C
:1034A000D0F8E43510B51B6804469847D4F8E835E1
:1034B0009B689847002010BD08B5D0F8E4355B68DC
:1034C0009847002008BD00BF43230B800048704789
:1034D0005801002038B51D4B1A68511C052A196087
:1034E00031D11979002201291A602CD09968B1F5DF
:1034F000006F08BF9A60154B9968DC681A46A142B4
:1035000002D100221A711EE095BFC1EB0404C1F57F
:1035100000631461136115690C4C402D8AB205D902
:103520004031403DA1602561402304E06918A1605D
:103530000021ABB22161054901240C7104498A18AC
:10354000812101F087F8002038BD00BF144C002015
:10355000A359002038B5282303FB0101074C084B71
:103560000546B1F88C131B6920469847284601216F
:103570002246402301F052F8002038BD5B5900205C
:10358000A800002070B50B78064613F060050C46C5
:1035900025D0202D1FD1CD88B5B113F0800F4878EC
:1035A00008D0224B22492A469B689847E288304639
:1035B0001F4928E01F4B1E4958641F4B30465D6170
:1035C0002A4600F0D6F820E0184B48789B68294638
:1035D0002A46984728E000F02BF9022524E04B7892
:1035E0000A2B14D00B2B17D0062B1DD14B881B0A8E
:1035F000212B05D1CA8811493A2A28BF3A2201E075
:103600000F493A22304600F09BF800250CE00D49A6
:10361000012200F095F807E08B781BB9064A1D4699
:10362000936101E000F004F9284670BDA800002075
:103630009B59002058010020144C00206A010020F2
:10364000610100202C4C002010B58121044600F0BF
:10365000CCFF0121204600F0C8FF8221204600F067
:10366000C4FF024B5B689847002010BDA8000020F3
:1036700038B5812104464022022300F095FF012144
:1036800040220223204600F08FFF822108220323DC
:10369000204600F089FF084B022200251A715D7157
:1036A000064B1B68984720460121054A402300F03D
:1036B000B5FF284638BD00BF44000020A800002008
:1036C0005B59002010B5074C606CFF2807D0064BF3
:1036D000064A9B68064952699847FF2363640020A5
:1036E00010BD00BF58010020A8000020144C00208D
:1036F0009B59002038B510490B79012B19D10C6961
:103700000CB90C7115E0402C07D98B68403C9AB27B
:1037100040338B600C61402306E08D68A3B22C1906
:103720008C600024AAB20C6104495218812100F077
:1037300091FF002038BD00BF144C0020A359002089
:1037400010B513460C46C0F83C21C0F838210222BF
:1037500080F811210021224600F07CFF002010BDDE
:1037600010B50C4613460021224600F073FF0020DE
:1037700010BD10B513460C46C0F89423C0F8902332
:10378000032280F811210021224600F047FF00208B
:1037900010BD10B50C4613460021224600F03EFF36
:1037A000002010BD0021042310B50A46044680F80D
:1037B00011310B4600F04EFF204600F0CFFD0020F7
:1037C00010BD0021052310B50A46044680F81131CA
:1037D0000B4600F023FF204600F0C0FD002010BD86
:1037E000282303FB0100B0F88C03704790F8CC3518
:1037F0000B7090F8CD354B7090F8CF2590F8CE3502
:1038000003EB02234B8090F8D12590F8D03503EBE1
:1038100002238B8090F8D32590F8D23503EB022356
:103820009BB2CB80C0F84031012380F81131704742
:1038300010B58021044600F029FF2046002100F049
:1038400025FF2046BDE8104000F088BD38B50D4684
:103850006B780446012B097910D027D3032B51D163
:1038600090F81231022B28D0032B47D16B889BB9DB
:1038700091B1802910D000F009FF0DE090F81231CD
:10388000022B1AD0032B39D16B88002B3AD149B1C6
:10389000802907D000F018FFD4F8E43520469B6853
:1038A000294698472046FFF77DFF2BE090F812311C
:1038B000022B02D0032B21D106E019B3802921D09D
:1038C000204600F0E3FE1DE011F0800F4FF02803CA
:1038D00006D001F07F0103FB010393F81E2103E0F2
:1038E00003FB010191F87623074B02B101221A6014
:1038F000204605490222FFF723FF03E02046294620
:10390000FFF796FF002038BD304C002038B590F806
:1039100012310446032B0D460CD10B79012B09D82B
:10392000D0F8E4359B689847EB883BB92046FFF711
:1039300039FF03E020462946FFF77AFF002038BD13
:1039400073B54B7804460D46092B00F21C81DFE865
:1039500013F0CD0008011A01E0001A0172000A00FC
:103960001A01BD0091006B881A0A013A062A00F27A
:103970000A81DFE812F007001A0027000801080199
:1039800008010801D0F8EC350DF106011B688078BC
:103990009847EB880146402B03D094F81231012B55
:1039A0003AD10823ADF8063036E0D0F8E4350DF111
:1039B00006019B6A80789847022343700146C4F849
:1039C000F00529E0DBB2052B00F2DD80DFE803F033
:1039D00003080D12171CD0F8EC3580785B6817E0EF
:1039E000D0F8EC3580789B6812E0D0F8EC35807820
:1039F000DB680DE0D0F8EC3580781B6908E0D0F882
:103A0000EC3580785B6903E0D0F8EC3580789B6911
:103A10000DF1060198470146BDF80630002B00F075
:103A2000B680EA88002A00F0B2809A4228BF1A467F
:103A3000ADF8062058E0AB88002B40F0A480EB885E
:103A4000002B40F0A08090F812216B88032A00F030
:103A50009A8003F07F0580F81451294600F05EFE3D
:103A60002046FFF79FFE0DB1022300E0012384F8FA
:103A700012318CE0A978474E0129317100F2838020
:103A800090F81231022B02D0032B7CD108E00029E0
:103A900063D00121032380F8101180F8123111E066
:103AA00039B9022380F8123180F81011FFF704FDB4
:103AB00053E090F81011012950D0FFF7FDFC317947
:103AC00084F810112046FFF7EBFC46E0EA88012A53
:103AD00059D190F81231022B02D0032B53D101E0BF
:103AE0002D4913E000F5887120460FE090F812315F
:103AF000023B012B47D8274B0122DA60D0F818216E
:103B00000AB10322DA60254920460222FFF718FE97
:103B10003DE06B88012B2DD0022B38D1AB8813F000
:103B2000FF0F34D102691B0A013B5268042B0FD8E6
:103B3000DFE803F0030507090B00012306E0022379
:103B400004E0032302E0042300E0052363F30612EC
:103B5000134B1A60012384F816312046FFF722FE2A
:103B600015E090F81231023B012B0CD86B88012B29
:103B70000DD10023C4F81831D4F8E43520469B68F1
:103B800029469847E9E720462946FFF751FE0020DD
:103B90007CBD00BF304C0020384C00203C4C002045
:103BA0001459002030B5C8B10023DDB20133C41868
:103BB00014F8014C002CF8D16B1C5B0013800B70C7
:103BC00003234B70022305E0CA545A1CD2B20233BD
:103BD0008C54DBB210F8012B002AF5D130BD00BFA8
:103BE00037B50023104C054601930320F6F7B2FCCD
:103BF000EB68013C1A69019213D0019A002AF4DAA9
:103C0000019A42F001020192019A1A61064A196969
:103C1000013A019102D00199C907F8D40320F6F7BF
:103C200099FC00203EBD00BF410D030010B5C478D3
:103C300074B900EB820003339B10D0F8D000224609
:103C400003E051F8044C0132046004319A42F8D187
:103C5000002010BD033230B59210D0F8D0400B4692
:103C6000002003E02568013043F8045C04339042EF
:103C7000F8D101EB800030BD0122F0B50023827045
:103C800040220129C37082800CD1082303700423D1
:103C900043704FF4A073C38002230372C1724FF0CC
:103CA000A04309E041B90C230370062343704FF48D
:103CB000A063C3801F4BC17203F500620261C36041
:103CC0004678044601461A46002508E002F5106CC5
:103CD00002F530620A65C1F814C001353A46043174
:103CE000B54202F12007F1D303F58062426103F58A
:103CF0008862C0F8CC20067803F5A0650146002252
:103D000003E0C1F88C50013220350431B242F8D3BF
:103D10001946002202E0C4F8CC1001320434B24249
:103D200001F58051F7D303F56063C0F80C31002032
:103D3000F0BD00BF0000044038B5037A0025012B18
:103D40000446C2681FD1936B417A65F3104309B1F1
:103D500043F480139363D36820466FF386136FF3A5
:103D600096536FF351436FF3D343D360FFF738FF9C
:103D7000E378012B19D1052363F34405E36845F08B
:103D800020059D6011E0D36843F04003D360FFF746
:103D900027FF637AE268002B0CBF4FF450234FF4E7
:103DA000E81393631420F6F7DFFBE378012B07D1C8
:103DB000E36805229D6862F3440545F020059D6097
:103DC000002038BDC36800209A6842F001029A6062
:103DD0007047C36800209A6822F001029A60704719
:103DE00007B500230193019B43F020030193019B3E
:103DF00061F38A130193019BC2681361064B116939
:103E0000013B019102D001998806F8D40320F6F70E
:103E1000A1FB00200EBD00BF410D030007B500232C
:103E20000193019B43F010030193019BC26813614E
:103E3000064B1169013B019102D00199C906F8D4E2
:103E40000320F6F787FB00200EBD00BF410D0300E5
:103E500008B5C2680129D3686FF35D736FF39E7371
:103E600002D143F0005302E009B943F0804332200D
:103E7000D360F6F779FB002008BDC368586900F0ED
:103E800001007047C3685B6913F0010F14BF002085
:103E900001207047C368586900F001007047C3688B
:103EA0005A69986910407047C36858687047036939
:103EB0001A6861F301021A607047C26800239361B7
:103EC0004FF0FF316FF080435361516053610C4BF1
:103ED0009361C3789169002B14BF4FF400634FF4D2
:103EE000016343F0804343F4701343F4405343F0C1
:103EF0000C0321EA03010B4393610020704700BFCC
:103F000000080080F8B5D0F80C3100221A6003696F
:103F100015461A68044665F3CC221A60C37A012B51
:103F200021D10321FFF7C3FFE36880214FF4001282
:103F300061F30F0259629A62A02262F30F0561F3E6
:103F40001F454FF49072C3F8045162F30F05C0F29D
:103F500020054FF4A072C3F8085162F30F056FF308
:103F60001F45C3F80C5110212046FFF739FF2046AA
:103F7000FFF754FF226900234FF0FF311361204601
:103F800053611E469161FF25D361214610E082698D
:103F9000013317680430C7F3076707F08007FFB2E3
:103FA000002F14BF4FF090470027176016619560EF
:103FB00062789342EBD300231D46FF2010E04A6D48
:103FC000013316680431C6F3076606F08006F6B2C0
:103FD000002E14BF4FF090460026166015619060C9
:103FE00062789342EBD323691A6942F480721A61B2
:103FF000E278012A04D1054A402161F359421A634B
:104000002046FFF75AFF0020F8BD00BF0301010062
:1040100003699B68C3F34103013B022B9ABF024A29
:10402000D05C0320704700BF4091010810B50369C0
:1040300081699C680A68C4F34100022802D06FF3CA
:104040000A0202E0032060F30A020A605A680020B4
:1040500042F480725A6010BD30B54D780B78002262
:10406000012D00EB830405D105FA03F3A46963F382
:104070000F0205E0012505FA03F3646D63F31F42A7
:104080002368C3F3072505F08005EDB26DB98D688F
:1040900065F30A03CD78C98865F3934361F39953B7
:1040A00043F0805343F40043236003690020D9693F
:1040B0000A43DA6130BD30B54D780B780024012D0C
:1040C000224600EB830105D105FA03F3896963F306
:1040D0000F0205E0012505FA03F3496D63F31F4262
:1040E00003696FF3CF340C60D969002021EA020222
:1040F000DA6130BDF8B54F780B78012F00EB830300
:1041000049D19E694C69356833692A4664F31203C4
:1041100014B967F3DC430BE08F68E419013CB4FB8E
:10412000F7F7CC7867F3DC43012C08BF64F35E73C8
:104130003361C378012B06D10B780C6900EB830344
:104140009B695C610CE0CB78012B09D04B693BB1DA
:104150000C78012707FA04F403695E6B34435C634F
:10416000CB78012B07D103699B68DB0554BF45F071
:10417000005245F080520B7842F0044200EB83037A
:104180009B691A60CB78012B38D10A788B8AC96871
:10419000FFF74CFD32E05E6D4F6935688C682A464A
:1041A00033692FB964F31203012464F3DC430AE09A
:1041B0003F19013FB7FBF4F7BF05BF0D7C4367F321
:1041C000DC4364F312033361C378012B05D10B7810
:1041D0000C6900EB83035B6D5C61CB78012B06D12E
:1041E0004B7913B145F0005201E045F080520B7855
:1041F00042F0044200EB8300436D1A600020F8BDDA
:1042000073B54D78012D3DD183694A691E681C69DB
:104210000094E4B242B962F306048DF800409DF8C0
:10422000024065F3C4040EE08D68AA4286BF4D616A
:1042300065F3060462F306048DF800409DF8024021
:10424000012262F3C4048DF80240009A1A61C27818
:10425000012A05D10A780C6900EB82029269546147
:1042600046F004421A60C378002B34D14B69002B0E
:1042700031D00A78012101FA02F20369586B024336
:104280005A6328E00B784E6900EB83035B6D8C6802
:104290001A681D690095EDB206B14C6164F306051C
:1042A0009DF802408DF80050012565F3C4048DF897
:1042B0000240009C1C61C378012B05D10B780C696E
:1042C00000EB83035B6D5C610B7842F0044200EB12
:1042D0008300436D1A6000207CBD4B78012B0B7866
:1042E00000EB83000AD182691368C3F3076101F010
:1042F0008001C9B221B143F0804301E0426D1368EF
:1043000043F400131360002070474B78012B0B78A7
:10431000C97800EB83000CBF8269426D02391368D3
:10432000C9B26FF35553012998BF43F0805313600E
:104330000020704703699A69D8691040000C7047E3
:1043400000EB81014B6D02699B6850691840704712
:1043500003699869DB69184080B2704782B0002316
:104360000093C0238DF803300122002362F3C403BD
:104370008DF8023018238DF80030009A436D1A61D1
:10438000C278012A07D100F5B8600C3058611A686C
:104390004FF080221A6002B07047D0F8183110B583
:1043A0000446D3B103699A68D20716D5827A42B11E
:1043B000D0F80C21D0F80C116FF341026FF300021A
:1043C0000A605A68052042F001025A60F6F7CCF8FC
:1043D00023695A6822F001025A6010BD837A63B1E2
:1043E00003699B68D90708D5D0F80C31D0F80C21A7
:1043F0006FF341036FF3000313607047012310B59F
:10440000002280F8123104460346FF2104E0586977
:1044100001328160186D8160607804338242F6D386
:10442000236900221A615A61DA614FF0FF329A6102
:104430002046FFF7F3FC20461021BDE81040CFE4F2
:104440004B78012B0B7800EB83000FD18369186840
:10445000C0F3074000F02003DBB2CBB900F002004C
:10446000C0B200280CBF302020207047436D186870
:10447000C0F3074000F02003DBB25BB900F002009C
:10448000C0B200280CBF4FF440504FF400507047AA
:10449000102070474FF4805070474B7810B5012BB7
:1044A0000B7800EB83030AD19C69102A236802D1A0
:1044B000BDE8104011E7202A0CD0302A0FE05C6DD7
:1044C000B2F5805F236802D143F400131BE0B2F51C
:1044D000005F02D143F0006315E0B2F5405F0FD1F9
:1044E000C3F3074202F02002D2B222B100234B7183
:1044F000BDE8104009E743F0806343F0802302E009
:104500000AB962F3CF33236010BD00BFF8B504468B
:10451000FFF7B2FB0122002384F8122184F8143142
:10452000282716461946402510E007FB034080F86F
:104530001C31A0F8223180F81D6180F81F11C0F8ED
:104540002451C0F82811C0F8301101336278934229
:10455000EBD3002328261946402510E006FB034034
:1045600080F87433A0F87A3380F8751380F87713E5
:10457000C0F87C53C0F88013C0F888130133627808
:104580009342EBD32046FFF724FC2046FFF7D4FBF1
:1045900000212046FFF75CFC2046FFF7B3FC2046D5
:1045A000BDE8F840FFF70EBC70B5CDB20C464FF039
:1045B000280601F07F0106FB010115F0800F14BFF2
:1045C00001F58E7101F55D7104F07F04ED090C7049
:1045D0004D708A60CB7005B1CC80022B01D10023D5
:1045E0000B71FFF739FD002070BD10B501F07F039E
:1045F0004FF0280404FB0303CAB212F0800F14BF6B
:1046000003F58E7303F55D7301F07F01D209197014
:104610005A701946FFF74FFD002010BD38B501F064
:104620007F05282404FB050404F55D714B6100231C
:104630008B614B70EBB2CA6084F87433C478012C80
:1046400008BF0A6113B9FFF7DBFD01E0FFF752FD78
:10465000002038BD70B501F07F04282505FB040556
:1046600005F58E710126E4B2CA600A61002285F860
:104670001C414E7005F58C758A614B6114B9FFF7CA
:10468000BFFD01E0FFF736FD002070BDCAB212F099
:10469000800F10B54FF0280306D001F07F0403FB14
:1046A000040303F58E7303E003FB010303F55D735D
:1046B000D209012401F07F0119709C705A701946CB
:1046C000FFF70BFE002010BDCAB212F0800F10B52C
:1046D0004FF0280306D001F07F0403FB040303F529
:1046E0008E7303E003FB010303F55D730024D2091D
:1046F00001F07F0119709C705A701946FFF705FE92
:10470000204610BD08B50B0604D501F07F01FFF768
:1047100067FB01E0FFF782FB002008BD0369002270
:1047200061F30A1219680A431A607047036903208B
:104730005A686FF341025A60F5F716BF0369032008
:104740005A6842F002025A60F5F70EBF11F0800F6E
:104750004FF0280306D001F07F0103FB010101F5B2
:104760008E7103E003FB010101F55D71FFF768BE87
:1047700011F0800F4FF0280306D001F07F0103FBFA
:10478000010101F58E7103E003FB010101F55D718B
:10479000FFF783BE2DE9F04F85B00446FFF772FBAB
:1047A000002800F05D822046FFF779FB05460028CF
:1047B00000F05682C0F3074000F00800C0B20028A5
:1047C0005AD02046FFF7B6FD27468246A1464FF055
:1047D0000008DFF868B32E4649E01AF0010F3FD019
:1047E0005FFA88F2114620460092FFF7A9FD10F00B
:1047F000010F0546009A20D07B6D01259D60E17870
:10480000A94207D11B69D9F87C13C3F31203CB1A51
:10481000C9F88C33DBF8003020461B6811469847F6
:10482000E378012B09D1B8F1000F06D194F81131CA
:10483000052B02D12046FFF791FD05F00203DBB204
:1048400013B17B6D02259D6005F00805EDB23DB109
:10485000DBF8003020469B6898477B6D0820986005
:1048600008F101084FEA5A0A043709F12809BAF198
:10487000000FB2D135460120C5F3074303F004030E
:10488000DBB2002B00F0A1802046FFF761FD274638
:1048900083464FF00008019591E01BF0010F00F0F6
:1048A000898023695FFA88F919695D6B04EB8902D5
:1048B00025FA09F59269ED019268EDB20D431540B4
:1048C000EA071CD5012000FA08F15A6B054622EAD6
:1048D00001025A63BB69994A9860136820465B6875
:1048E00049469847E378AB4209D1B8F1000F06D1A9
:1048F00094F81131042B02D12046FFF72FFD05F06B
:104900000803DBB213B1BB6908259D6005F01003F5
:10491000DBB213B1BB6910259D6005F04003DBB22B
:1049200013B1BB6940259D6005F00203DBB213B1F2
:10493000BB6902259D6025F07F0515F0FF0F39D07A
:10494000282505FB084505F58E75AB696A69C246E1
:10495000C3EB020CAB68A0469C4528BF9C460CF1FB
:10496000030CBB694FEA9C0C9B69664614E0AA687D
:104970001C1B944228BF1446A3B24046E9684A462D
:10498000FFF754F9EB68E61C1B19EB60AB69B6083E
:104990001C19AC61BB699B699BB2B34205D9AC6978
:1049A0006B699C4201D2002BE1D1BB698025444652
:1049B0009D60D04608F101084FEA5B0B0437BBF15C
:1049C000000F7FF46AAF019D012005F00203DBB206
:1049D00013B1E36802225A61C5F3076303F0800351
:1049E000DBB2CBB1A37A43B1D4F80C31D4F80C21AB
:1049F0006FF341036FF300031360236920465A6885
:104A000022F001025A604D4B1B689B699847E3688E
:104A10004FF000425A610120C5F3072303F0080359
:104A2000DBB2002B2ED000238DF80F3094F812311A
:104A300020468DF80F30414B1B685B69984723690E
:104A4000E2684FF400619B685161A27ACAB1DB074A
:104A500017D594F81501012813D19DF80F30032BB9
:104A600010D1D4F80C311A6842F001021A601A68A9
:104A700042F003021A60324B1A6942F006021A61D0
:104A800000E0012005F00803DBB243B12B4B2046C8
:104A90001B68DB689847E36808225A61012005F02B
:104AA0001003DBB2002B34D0E36828269A6922F089
:104AB00010029A611F6A07F00F0306FB0346C7F353
:104AC0004343022B06F55D7602D0062B1BD10EE088
:104AD00047F6F0733B40B3B1C7F30A172046F168BD
:104AE0003A46FFF7B7F8F368DB19F36008E004F51E
:104AF000B8610C3120460822FFF7ACF8C7F30A175B
:104B0000B369DF19B761E36801209A6942F01002C6
:104B10009A61C5F3072303F01003DBB2002B38D0F2
:104B2000236900265A68314622F001025A60204665
:104B3000FFF756F923463246FF2108E028010020FE
:104B400000ED00E0586901328160186D8160607885
:104B500004338242F6D3236901274FF0FF3267F313
:104B60000F069A6167F31F460B22DE615A611A61D4
:104B70001A6820466FF30A121A60FFF7EFFBE3682A
:104B80004FF480525A61384B20461B681B69984786
:104B90003846C5F3072303F02003DBB2EBB1204610
:104BA000FFF744FAE3682046DE68FFF731FA03288E
:104BB00006D10023A3704FF40073A380092304E0FF
:104BC0000123A3704023A380052363F38D26E368AC
:104BD0004FF40052DE6001205A61C5F3074303F031
:104BE0001003DBB24BB1204B20461B68DB699847B2
:104BF000E3684FF480125A610120C5F3074303F0C4
:104C00002003DBB24BB1184B20461B681B6A984748
:104C1000E3684FF400125A610120C5F3076303F003
:104C20004003DBB24BB1104B20461B685B6A9847D0
:104C3000E3684FF080425A61012005F00405EDB2AF
:104C400075B1E3685D6805F00403DBB223B1064B80
:104C500020461B689B6A9847E36801205D60FFE778
:104C600005B0BDE8F08F00BF2801002081F00041B1
:104C700002E000BF83F0004330B54FEA41044FEA41
:104C8000430594EA050F08BF90EA020F1FBF54EADC
:104C9000000C55EA020C7FEA645C7FEA655C00F078
:104CA000E2804FEA5454D4EB5555B8BF6D420CDD49
:104CB0002C4480EA020281EA030382EA000083EACC
:104CC000010180EA020281EA0303362D88BF30BD6C
:104CD00011F0004F4FEA01314FF4801C4CEA1131C2
:104CE00002D0404261EB410113F0004F4FEA033321
:104CF0004CEA133302D0524263EB430394EA050FAC
:104D000000F0A780A4F10104D5F1200E0DDB02FA1A
:104D10000EFC22FA05F2801841F1000103FA0EF2AE
:104D2000801843FA05F359410EE0A5F120050EF174
:104D3000200E012A03FA0EFC28BF4CF0020C43FAA5
:104D400005F3C01851EBE37101F0004507D54FF0B2
:104D5000000EDCF1000C7EEB00006EEB0101B1F502
:104D6000801F1BD3B1F5001F0CD349085FEA300048
:104D70004FEA3C0C04F101044FEA445212F5800F53
:104D800080F09A80BCF1004F08BF5FEA500C50F1F0
:104D9000000041EB045141EA050130BD5FEA4C0CD3
:104DA000404141EB010111F4801FA4F10104E9D15C
:104DB00091F0000F04BF01460020B1FA81F308BF53
:104DC0002033A3F10B03B3F120020CDA0C3208DD1F
:104DD00002F1140CC2F10C0201FA0CF021FA02F1FA
:104DE0000CE002F11402D8BFC2F1200C01FA02F16A
:104DF00020FA0CFCDCBF41EA0C019040E41AA2BF8F
:104E000001EB0451294330BD6FEA04041F3C1CDA56
:104E10000C340EDC04F11404C4F1200220FA04F076
:104E200001FA02F340EA030021FA04F345EA030120
:104E300030BDC4F10C04C4F1200220FA02F001FAE2
:104E400004F340EA0300294630BD21FA04F0294664
:104E500030BD94F0000F83F4801306BF81F48011FD
:104E60000134013D4EE77FEA645C18BF7FEA655C70
:104E700029D094EA050F08BF90EA020F05D054EA42
:104E8000000C04BF1946104630BD91EA030F1EBF47
:104E90000021002030BD5FEA545C05D1400049414B
:104EA00028BF41F0004130BD14F580043CBF01F53E
:104EB000801130BD01F0004545F0FE4141F4700124
:104EC0004FF0000030BD7FEA645C1ABF19461046FF
:104ED0007FEA655C1CBF0B46024650EA013406BF00
:104EE00052EA033591EA030F41F4002130BD00BFBF
:104EF00090F0000F04BF0021704730B54FF480647C
:104F000004F132044FF000054FF0000150E700BFFC
:104F100090F0000F04BF0021704730B54FF480645B
:104F200004F1320410F0004548BF40424FF0000148
:104F30003EE700BF42004FEAE2014FEA31014FEA8B
:104F400002701FBF12F07F4393F07F4F81F06051DA
:104F5000704792F0000F14BF93F07F4F704730B549
:104F60004FF4607401F0004521F0004120E700BFDC
:104F700050EA010208BF704730B54FF000050AE063
:104F800050EA010208BF704730B511F0004502D564
:104F9000404261EB41014FF4806404F132045FEA66
:104FA000915C3FF4DCAE4FF003025FEADC0C18BF0B
:104FB00003325FEADC0C18BF033202EBDC02C2F101
:104FC000200300FA03FC20FA02F001FA03FE40EA93
:104FD0000E0021FA02F11444C1E600BF70B54FF093
:104FE000FF0C4CF4E06C1CEA11541DBF1CEA135575
:104FF00094EA0C0F95EA0C0F00F0DEF82C4481EADD
:10500000030621EA4C5123EA4C5350EA013518BFFC
:1050100052EA033541F4801143F4801338D0A0FBE9
:1050200002CE4FF00005E1FB02E506F00042E0FB96
:1050300003E54FF00006E1FB03569CF0000F18BF9C
:105040004EF0010EA4F1FF04B6F5007F64F5407444
:1050500004D25FEA4E0E6D4146EB060642EAC621D7
:1050600041EA55514FEAC52040EA5E504FEACE2E44
:10507000B4F1FD0C88BFBCF5E06F1ED8BEF1004F47
:1050800008BF5FEA500E50F1000041EB045170BDC3
:1050900006F0004646EA010140EA020081EA030107
:1050A000B4EB5C04C2BFD4EB0C0541EA045170BD03
:1050B00041F480114FF0000E013C00F3AB8014F17D
:1050C000360FDEBF002001F0004170BDC4F10004C6
:1050D000203C35DA0C341BDC04F11404C4F1200547
:1050E00000FA05F320FA04F001FA05F240EA0200A2
:1050F00001F0004221F0004110EBD37021FA04F6D8
:1051000042EB06015EEA430E08BF20EAD37070BD91
:10511000C4F10C04C4F1200500FA04F320FA05F0F0
:1051200001FA04F240EA020001F0004110EBD370F2
:1051300041F100015EEA430E08BF20EAD37070BD62
:10514000C4F1200500FA05F24EEA020E20FA04F33B
:1051500001FA05F243EA020321FA04F001F00041EA
:1051600021FA04F220EA020000EBD3705EEA430E5B
:1051700008BF20EAD37070BD94F0000F0FD101F08A
:105180000046400041EB010111F4801F08BF013CC3
:10519000F7D041EA060195F0000F18BF704703F001
:1051A0000046520043EB030313F4801F08BF013D88
:1051B000F7D043EA0603704794EA0C0F0CEA135544
:1051C00018BF95EA0C0F0CD050EA410618BF52EAFE
:1051D0004306D1D181EA030101F000414FF0000004
:1051E00070BD50EA410606BF1046194652EA430612
:1051F00019D094EA0C0F02D150EA013613D195EA86
:105200000C0F05D152EA03361CBF104619460AD1CD
:1052100081EA030101F0004141F0FE4141F47001D7
:105220004FF0000070BD41F0FE4141F4780170BDC7
:1052300070B54FF0FF0C4CF4E06C1CEA11541DBF2C
:105240001CEA135594EA0C0F95EA0C0F00F0A7F82E
:10525000A4EB050481EA030E52EA03354FEA01315B
:1052600000F088804FEA03334FF0805545EA13136E
:1052700043EA12634FEA022245EA111545EA106536
:105280004FEA00260EF000419D4208BF964244F1CD
:10529000FD0404F5407402D25B084FEA3202B61AEC
:1052A00065EB03055B084FEA32024FF480104FF4C0
:1052B000002CB6EB020E75EB030E22BFB61A754634
:1052C00040EA0C005B084FEA3202B6EB020E75EBC7
:1052D000030E22BFB61A754640EA5C005B084FEA2F
:1052E0003202B6EB020E75EB030E22BFB61A7546FC
:1052F00040EA9C005B084FEA3202B6EB020E75EB07
:10530000030E22BFB61A754640EADC0055EA060EC7
:1053100018D04FEA051545EA16754FEA06164FEA0A
:10532000C30343EA52734FEAC2025FEA1C1CC0D1B6
:1053300011F4801F0BD141EA00014FF000004FF043
:10534000004CB6E711F4801F04BF01430020B4F104
:10535000FD0C88BFBCF5E06F3FF6AFAEB5EB030CBC
:1053600004BFB6EB020C5FEA500C50F1000041EBB9
:10537000045170BD0EF0004E4EEA113114EB5C0486
:10538000C2BFD4EB0C0541EA045170BD41F4801159
:105390004FF0000E013C90E645EA060E8DE60CEA61
:1053A000135594EA0C0F08BF95EA0C0F3FF43BAF7E
:1053B00094EA0C0F0AD150EA01347FF434AF95EA35
:1053C0000C0F7FF425AF104619462CE795EA0C0F19
:1053D00006D152EA03353FF4FDAE1046194622E7E6
:1053E00050EA410618BF52EA43067FF4C5AE50EAC0
:1053F00041047FF40DAF52EA43057FF4EBAE12E7B0
:105400004FF0FF3C06E000BF4FF0010C02E000BF90
:105410004FF0010C4DF804CD4FEA410C7FEA6C5C73
:105420004FEA430C18BF7FEA6C5C1BD001B050EA16
:10543000410C0CBF52EA430C91EA030F02BF90EA01
:10544000020F0020704710F1000F91EA030F58BFC0
:10545000994208BF90422CBFD8176FEAE37040F022
:10546000010070474FEA410C7FEA6C5C02D150EAC0
:10547000013C07D14FEA430C7FEA6C5CD6D152EA7B
:10548000033CD3D05DF8040B704700BF8446104640
:1054900062468C461946634600E000BF01B5FFF73F
:1054A000B7FF002848BF10F1000F01BD4DF808ED0F
:1054B000FFF7F4FF0CBF012000205DF808FB00BFE0
:1054C0004DF808EDFFF7EAFF34BF012000205DF83A
:1054D00008FB00BF4DF808EDFFF7E0FF94BF012087
:1054E00000205DF808FB00BF4DF808EDFFF7CEFF88
:1054F00094BF012000205DF808FB00BF4DF808EDC7
:10550000FFF7C4FF34BF012000205DF808FB00BF97
:105510004FEA410212F5001215D211D56FF47873DB
:10552000B3EB625212D94FEAC12343F0004343EA7E
:10553000505311F0004F23FA02F018BF4042704759
:105540004FF00000704750EA013005D111F00040E3
:1055500008BF6FF0004070474FF00000704700BF79
:105560004FEA4102B2F1E04324BFB3F5001CDCF185
:10557000FE5C0DD901F0004C4FEAC0024CEA5070BD
:10558000B2F1004F40EB830008BF20F001007047EC
:1055900011F0804F21D113F13872BCBF01F00040EF
:1055A000704741F480114FEA5252C2F11802C2F121
:1055B000200C10FA0CF320FA02F018BF40F00100A2
:1055C0004FEAC1234FEAD32303FA0CFC40EA0C0054
:1055D00023FA02F34FEA4303CCE77FEA625307D191
:1055E00050EA01331EBF4FF0FE4040F440007047C8
:1055F00001F0004040F0FE4040F40000704700BF62
:1056000080F0004002E000BF81F0004142001FBF77
:105610005FEA410392EA030F7FEA226C7FEA236C80
:105620006AD04FEA1262D2EB1363C1BFD218414075
:1056300048404140B8BF5B42192B88BF704710F00B
:10564000004F40F4000020F07F4018BF404211F0AE
:10565000004F41F4000121F07F4118BF494292EA16
:10566000030F3FD0A2F1010241FA03FC10EB0C0042
:10567000C3F1200301FA03F100F0004302D54942CF
:1056800060EB4000B0F5000F13D3B0F1807F06D37C
:1056900040084FEA310102F10102FE2A51D2B1F174
:1056A000004F40EBC25008BF20F0010040EA030069
:1056B0007047490040EB000010F4000FA2F1010216
:1056C000EDD1B0FA80FCACF1080CB2EB0C0200FAA0
:1056D0000CF0AABF00EBC25052421843BCBFD040EE
:1056E0001843704792F0000F81F4000106BF80F468
:1056F00000000132013BB5E74FEA41037FEA226C2B
:1057000018BF7FEA236C21D092EA030F04D092F0F5
:10571000000F08BF0846704790EA010F1CBF002029
:10572000704712F07F4F04D1400028BF40F0004086
:10573000704712F100723CBF00F50000704700F0A6
:10574000004343F0FE4040F4000070477FEA2262CD
:1057500016BF08467FEA23630146420206BF5FEA9E
:10576000412390EA010F40F4800070474FF000039E
:1057700004E000BF10F0004348BF40425FEA000C65
:1057800008BF704743F0964301464FF000001CE00D
:1057900050EA010208BF70474FF000030AE000BF63
:1057A00050EA010208BF704711F0004302D54042A1
:1057B00061EB41015FEA010C02BF84460146002013
:1057C00043F0B64308BFA3F18053A3F50003BCFA2E
:1057D0008CF2083AA3EBC25310DB01FA02FC6344DB
:1057E00000FA02FCC2F12002BCF1004F20FA02F2E2
:1057F00043EB020008BF20F00100704702F12002D5
:1058000001FA02FCC2F1200250EA4C0021FA02F235
:1058100043EB020008BF20EADC7070474FF0FF0C3A
:105820001CEAD0521EBF1CEAD15392EA0C0F93EA35
:105830000C0F6FD01A4480EA010C400218BF5FEAD7
:1058400041211ED04FF0006343EA501043EA51114A
:10585000A0FB01310CF00040B1F5000F3EBF490044
:1058600041EAD3715B0040EA010062F17F02FD2A48
:105870001DD8B3F1004F40EBC25008BF20F001002B
:10588000704790F0000F0CF0004C08BF49024CEA42
:10589000502040EA51207F3AC2BFD2F1FF0340EAD4
:1058A000C250704740F400004FF00003013A5DDC45
:1058B00012F1190FDCBF00F000407047C2F1000286
:1058C000410021FA02F1C2F1200200FA02FC5FEA73
:1058D000310040F1000053EA4C0308BF20EADC70BD
:1058E000704792F0000F00F0004C02BF400010F42F
:1058F000000F013AF9D040EA0C0093F0000F01F0DC
:10590000004C02BF490011F4000F013BF9D041EAFD
:105910000C018FE70CEAD15392EA0C0F18BF93EAFF
:105920000C0F0AD030F0004C18BF31F0004CD8D129
:1059300080EA010000F00040704790F0000F17BFB0
:1059400090F0004F084691F0000F91F0004F14D0F6
:1059500092EA0C0F01D142020FD193EA0C0F03D14E
:105960004B0218BF084608D180EA010000F0004051
:1059700040F0FE4040F40000704740F0FE4040F42C
:10598000400070474FF0FF0C1CEAD0521EBF1CEACB
:10599000D15392EA0C0F93EA0C0F69D0A2EB0302E9
:1059A00080EA010C49024FEA402037D04FF0805383
:1059B00043EA111143EA10130CF000408B4238BF48
:1059C0005B0042F17D024FF4000C8B4224BF5B1A56
:1059D00040EA0C00B3EB510F24BFA3EB510340EAA4
:1059E0005C00B3EB910F24BFA3EB910340EA9C0052
:1059F000B3EBD10F24BFA3EBD10340EADC001B01C2
:105A000018BF5FEA1C1CE0D1FD2A3FF650AF8B4265
:105A100040EBC25008BF20F0010070470CF0004C72
:105A20004CEA50207F32C2BFD2F1FF0340EAC2509D
:105A3000704740F400004FF00003013A37E792F05E
:105A4000000F00F0004C02BF400010F4000F013ABC
:105A5000F9D040EA0C0093F0000F01F0004C02BFB7
:105A6000490011F4000F013BF9D041EA0C0195E720
:105A70000CEAD15392EA0C0F08D142027FF47DAFB9
:105A800093EA0C0F7FF470AF084676E793EA0C0FA9
:105A900004D14B023FF44CAF08466EE730F0004CA7
:105AA00018BF31F0004CCAD130F000427FF45CAF37
:105AB00031F000437FF43CAF5FE700BF4FEA4002A4
:105AC000B2F1FE4F0FD34FF09E03B3EB12620DD92C
:105AD0004FEA002343F0004310F0004F23FA02F096
:105AE00018BF404270474FF00000704712F1610F3D
:105AF00001D1420205D110F0004008BF6FF0004014
:105B000070474FF00000704742000ED2B2F1FE4FD6
:105B10000BD34FF09E03B3EB126209D44FEA00237C
:105B200043F0004323FA02F070474FF00000704743
:105B300012F1610F01D1420202D14FF0FF307047E4
:105B40004FF00000704700BF73B96AB9002908BF61
:105B50000028BCBF00204FF00041C4BF6FF00041DF
:105B60004FF0FF3001F072B882B0EC462DE90050E2
:105B700000F006F8DDF804E002B00CBC704700BF8E
:105B80002DE970431546804689461C4601F060F8B1
:105B900005FB01F6A5FB002300FB0464E318069C4B
:105BA000B8EB020269EB0303C4E90023BDE870838C
:105BB000F8B5144606460F461D4601F0ADF900FB48
:105BC00005F5A0FB042304FB0154E318069CB21A5C
:105BD00067EB0303C4E90023F8BD00BF036803B10A
:105BE0001B181846704700BF03685A004CBF43F0AB
:105BF000004323F00043C018704700BF2DE9F84F61
:105C00000446914641B301F1FF3BDA46002707EB1A
:105C10000A0000EBD0756D1004EBC5063046FFF7A7
:105C2000E3FFAB45804610D0691C04EBC100FFF7D1
:105C3000DBFF0138C84504D9BD4209D005F1FF3A60
:105C4000E5E7484505D26F1CE1E74FF0FF30F1E78B
:105C500000263046BDE8F88F0E463046BDE8F88F86
:105C600030B52B4B83B004468D1E002B49D02846FF
:105C700001A9AFF300800346002822D02A46184627
:105C80000199FFF7BBFF054600281DD0FFF7ACFFC9
:105C90006B68A064012B10D0281D002B22DBFFF7BE
:105CA000A3FF0021E06421650368002B0FDBFFF7F1
:105CB0009BFF2061002003B030BD0023236105203D
:105CC000F9E720610920F6E720610920F3E7C3F333
:105CD000036058B101280CD002280ED000202061AA
:105CE0000920E8E70122E0642265DDE7094B236132
:105CF000E1E7094A00202261DDE70849002021612F
:105D0000D9E7074A07491346881AC2100192B5E736
:105D10000000000025620108216201081D620108DF
:105D20001C93010804940108036810B50446D807C1
:105D300006D4990704F1480009D500F009FD23684D
:105D40005A0709D518070ED5D90613D510BD00F08E
:105D5000F7FC23685A07F5D404F1D00000F000FDE9
:105D600023681807F0D404F5D87000F001FD23680B
:105D7000D906EBD404F50C70BDE8104000F03CBD32
:105D80002DE9F047ADF5916D02AC0F1D261D0546BE
:105D900091460FCF0FC60FCF0FC60FCF0FC697E894
:105DA0000F00D5F80C800027D5F818A086E80F0062
:105DB000216C28462760FFF753FF0646B94514BFFC
:105DC0004FF00A094FF00909FEB1A16B49F0100923
:105DD000616401208DE8100449462A462B46C047DD
:105DE00000282BD1002E2AD1204692A94FF4107200
:105DF00001F040FE082F28D1216C2846FFF730FF24
:105E000006464FF00909002EDFD1206C21464FF4E1
:105E10001072686192A801F02DFE2F69294692AA9E
:105E20004846B847A09B0746636401208DE81004EC
:105E300049462A462B46C0470028D3D0092630467B
:105E400022B00DF5806DBDE8F087072FF6D1201D3B
:105E500000F06AFC38B504460D46296C2046FFF771
:105E6000FFFE50B92A6C01206261236921462A464F
:105E700098470828F1D0072801D001F0F3FD281D2C
:105E800000F052FC11B933B10220704704298CBFD5
:105E90000220012070470F2A01D90220704700EB31
:105EA000820042681846009B1A60704710B50A4687
:105EB00084B000210B4603AC0094FFF7E3FF039886
:105EC00004B010BD11B933B10220704704298CBF52
:105ED0000220012070470F2A01D902207047009943
:105EE00000EB8202096818465160704700B585B022
:105EF00004AB43F8042D0A46002100930B46FFF73C
:105F0000E1FF05B000BD00BF2DE9F04FCD6C0C46A0
:105F100055F8041B8BB0174600F008021E4603928A
:105F200000F003080795002B40F0E080090206917D
:105F3000216D8DF821300323B8F1020F8DF8203048
:105F400008BFA56B11F0010340F0E480019304F158
:105F500058030293D5F80090B9F1000F00F0DC80EF
:105F6000022E00F0BF80B5F80090B5F802A004350D
:105F7000A26C0F212AF0010B38469344FFF796FFDD
:105F8000834518D829F0010CE3440AF0010A09F00E
:105F90000103584543EA4A092CBF00200120B9F10A
:105FA000010F12D032D2B8F1000F02D0002840F019
:105FB00017810435CEE70AF0010A09F0010343EA2C
:105FC0004A090020B9F1010FECD1B8F1000F40F0FF
:105FD000C880C8B16B68D5F800909A1C19D0029A95
:105FE000013309920DD0281DFFF7F8FD4FEAD97251
:105FF000014609AB2046AFF30080002800F0EC809A
:10600000099A002A40F0CC800835A3E7B9F1020FC5
:1060100003D009200BB0BDE8F08F2B6823F00042BD
:106020000092B8F1000F40F08380002853D003980D
:10603000002840F0B2800098002800F0B180009B5A
:1060400005F1040ADB07DDF80C9010D402995046E4
:106050000991FFF7C3FD039A014609AB2046AFF350
:106060000080002833D10AF1040A4FF00109CDF86D
:106070001080AB46B84650460596029F11E0009945
:106080008E4200F0C0800997FFF7A8FD52460146F6
:1060900009AB2046AFF30080B14698B9281D06F140
:1060A0000109051D0997FFF799FD09AB014600227B
:1060B0002046AFF30080824609F101062846BAF176
:1060C000000FDCD04746059EDDF810805D46009A43
:1060D0004A4565D02B68002B7CDB0099481C05EBFA
:1060E000800537E7D5F804A0083541E70B04C1F374
:1060F0000740216D0222B8F1020F069305EB8005DF
:1061000008BFA56B11F001038DF821008DF8202048
:106110003FF41CAF00200190384606A900F004FCB3
:1061200000287FF476AF019A002A43D1082071E756
:106130000D213846D4F82090FFF7B8FE8145C9D12B
:10614000A26A9542C6D10098291D00220423A062AC
:10615000E262236361632868002857DB0122019211
:10616000BBE70D213846D4F82090FFF79FFE81450C
:106170007FF44AAFA16A8D427FF446AF2846FFF70D
:1061800033FD0F2102463846FFF7B0FE38460021A6
:106190002246FFF7ABFE07203CE7009900299AD181
:1061A00038460D21FFF782FE099B20626362A562DB
:1061B00006202FE70F213846FFF778FE0E21024612
:1061C0003846FFF793FE38460F21134AFFF78EFE3D
:1061D00007201FE7043580E7CDF824800835B9E6AD
:1061E0002846FFF701FD04350646A5632046AFF3B8
:1061F000008000283FF40DAF38460F213246FFF7EC
:1062000075FE072006E75D464746C9E7009B591C17
:1062100005EB8100B3E700BF00000000022373E636
:10622000012371E600236FE62DE9F0470446E8B04C
:1062300004290CD8DFE801F0390392940F00150C03
:10624000012B96B200F07881052B00F0C880022067
:1062500068B0BDE8F087002BF9D1102AF7D8236881
:10626000D90600F1738164A8019200F0CFFA019A77
:10627000A36BD00744BF53F8040B6490910744BF4D
:1062800053F8041B6591500748BF53F8041B64A8DA
:1062900048BF6691110748BF53F8042BA36348BF5A
:1062A000679200F0A9FA0020D2E7002BCFD1A36BB0
:1062B000D00791B244BF53F8042B62608A0744BFF1
:1062C00053F8042BA260480744BF53F8042BE26044
:1062D0000A0744BF53F8042B2261C80644BF53F891
:1062E000042B62618A0644BF53F8042BA26148065E
:1062F00044BF53F8042BE2610A0644BF53F8042B51
:106300002262C80544BF53F8042B62628A0544BF69
:1063100053F8042BA262480544BF53F8042BE262F1
:106320000A0544BF53F8042B2263C80444BF53F842
:10633000042B626311F400501CBF53F8042BA263BA
:106340004A0444BF53F8042BE2630A0444BF53F8E1
:10635000042B2264002840D1A36379E7012077E76A
:10636000032B7FF474AF160C95B2AA19102A3FF6CE
:106370006EAF2368180700F10A8144A800F01AFAEA
:10638000A76B4FEA450E3B460DB30EF1FF3C44A907
:1063900053F8040B01EBC60662460CF0010146F807
:1063A000040B92B129B153F8041B013A46F8041BBF
:1063B0000BD0184650F8045B314641F8045B5D6829
:1063C000031D75600E1D023AF3D107EB8E0344A83E
:1063D000A36300F0CDF900203AE7002038E77719F1
:1063E0002022BA42FFF433AF012B00F0A8800F2D1A
:1063F00040F2A8803746F6B1052B7FF428AF0F2D69
:1064000011D82268D0070ED522F00101052B21609A
:1064100000F0DA8022F00302204640F8482B019376
:1064200000F092F9019B1FB12268510700F1B7807B
:10643000012B00F0BE800F2D74D9002F40F09F80FB
:10644000D4F83890002EC8462EDD49464FEA46085B
:106450000DF1080C51F8046B0CEBC50208F1FF308C
:1064600000F0010A42F8046BA8F1020CD0B1BAF1B5
:10647000000F08D051F8040B0CF1FF3CBCF1FF3FBA
:1064800042F8040B0ED00E4656F804AB104640F806
:1064900004AB4968ACF1020C5160311D021DBCF126
:1064A000FF3FF0D109EB88089FB3102D2CBF2E467B
:1064B000102668AA414602EBC60A4FEA470951F87E
:1064C000046BAAF5C87209F1FF3000F0010A42F826
:1064D000046BA9F1020CD0B1BAF1000F08D051F849
:1064E000040B0CF1FF3CBCF1FF3F42F8040B0ED053
:1064F0000E4656F804AB104640F804AB4968ACF1C0
:10650000020C5160311D021DBCF1FF3FF0D108EBC0
:106510008908012B2BD00F2DC4F8388008D9FFB97A
:10652000384695E602A8019300F016F9019B84E72E
:1065300002A800F00DF9F2E77719102251E70F2DAC
:106540003FF685AE102F10D9103F55E723F010030A
:10655000236004F50C70019200F058F9019A82E66C
:1065600024A800F0FDF8002072E6002747E708F1B4
:10657000040302A8A36300F0E3F8002068E624A85F
:106580000193C5F1100600F0EFF8019B58E723F0E6
:10659000080704F5D870276000F00CF9EDE622F04A
:1065A0000401204640F8D01B019300F0DDF8019B68
:1065B0003EE702A8019300F0C7F8019B002F3FF4CB
:1065C0003FAFC5F110063BE741F00201204640F81D
:1065D000481B019300F0C0F8019B24E7406C704712
:1065E000F0B50D46C96BADF5117D296401AE2F1DC7
:1065F00004460FCF0FC60FCF0FC60FCF0FC697E8B9
:106600000F0086E80F004FF0FF33009310992046EB
:10661000FFF726FB58B9266921466A46B047082885
:106620000646F3D06846FFF77FFB062E03D009200D
:106630000DF5117DF0BD20462946FFF70BFC00BF8C
:1066400010B4DC6BC1608261194600221C6410BC6E
:10665000FFF796BB38B54269C36804460D460A6425
:1066600023B10122FFF78CFB01F0FCF903692146FD
:1066700002202A469847072803D0082804D001F0B2
:10668000F1F9281D00F050F820462946FFF7E2FBFB
:10669000C36823B1CA6B0A640022FFF771BB9FE78E
:1066A000704700BF08B5836801460BB101209847C9
:1066B00008BD00BFF0B5D46BADF5277D146401AE05
:1066C000171D05460C460FCF0FC60FCF0FC60FCFB5
:1066D0000FC697E80F0086E80F004FF0FF330093D6
:1066E000109990A8FFF7BCFA034690AA68460C21BF
:1066F000BBB9FFF7FBFB21466846A847064690A9B1
:1067000008206A466EB9949B98470528064601D032
:106710000928E5D16846FFF707FB30460DF5277DD0
:10672000F0BD0926F6E700BF00F1340191E838001A
:106730009C46A6464CF8045D90E8FF0FE54600BD78
:1067400090EC210B704700BF80EC210B704700BF1D
:1067500090EC200B704700BF80EC200B704700BF0F
:10676000D0EC200B704700BFC0EC200B704700BF7F
:10677000F0EC0201F0EC0211F0EC0221F0EC02313D
:10678000F0EC0241F0EC0251F0EC0261F0EC02712D
:10679000F0EC0281F0EC0291F0EC02A1F0EC02B11D
:1067A000F0EC02C1F0EC02D1F0EC02E1F0EC02F10D
:1067B000704700BFE0EC0201E0EC0211E0EC0221C6
:1067C000E0EC0231E0EC0241E0EC0251E0EC02616D
:1067D000E0EC0271E0EC0281E0EC0291E0EC02A15D
:1067E000E0EC02B1E0EC02C1E0EC02D1E0EC02E14D
:1067F000E0EC02F1704700BFB0FC0181B0FC0191F8
:10680000B0FC01A1B0FC01B1704700BFA0FC018148
:10681000A0FC0191A0FC01A1A0FC01B1704700BF48
:10682000EC4600B52DE900502DE9FF1F4FF00003A5
:106830002DE90C0001A9FFF7D3FEDDF840E012B00E
:10684000704700BFEC4600B52DE900502DE9FF1F51
:106850004FF000032DE90C0001A9FFF7FBFEDDF866
:1068600040E012B0704700BFEC4600B52DE9005083
:106870002DE9FF1F4FF000032DE90C0001A9FFF7E0
:1068800007FFDDF840E012B0704700BFEC4600B5EE
:106890002DE900502DE9FF1F4FF000032DE90C00FA
:1068A00001ABFFF7CDFEDDF840E012B0704700BF4E
:1068B000EC4600B52DE900502DE9FF1F4FF0000315
:1068C0002DE90C0001AAFFF7F5FEDDF840E012B05B
:1068D000704700BF027A03461AB9427A42B9B02023
:1068E00070470068013A01021A72000E1960704781
:1068F0004168501E587251F8040B0322596001027E
:106900001A72000E1960704710B5002184B00C2275
:106910000DEB02040B460094FFF7B4FA039804B0A1
:1069200010BD00BFF0E700BF2DE9F043064685B07B
:106930000D464FF000094FF47F672846FFF7CAFF66
:10694000B028044600F0B18010F0800120D000F0A3
:10695000F003802B75D0902B37D0A02B45D0B02BD7
:1069600056D0C02B00F0868000F0F800D0280BD164
:1069700004F007035A1C42F400223046012105238B
:10698000FFF752FC0028D8D0092005B0BDE8F083FD
:106990004FEA800203A85FFA82F800900D220B46AE
:1069A0003046FFF76FFA039B600608F104084CBFFE
:1069B000C8EB0303434403AC039300940021304627
:1069C0000D220B46FFF77EFAB7E700F00F020D2A03
:1069D000DAD00F2AD8D0002103AC009430460B4601
:1069E00003ACFFF74FFA0094E8E7C24302F0070C4C
:1069F00047FA0CF0210700F47F6248BF42F480425E
:106A0000002130460B46FFF70FFC0028BCD194E76D
:106A1000B1285ED0B2286FD0B32800F0968000F085
:106A2000FC0CBCF1B40F46D000F007014A1C42F444
:106A30000022012130460B46FFF7F6FB0028A3D1C8
:106A40007BE72846FFF746FF210240EA0104B4F540
:106A5000004F99D0230500211A0C30460B46240123
:106A6000FFF7E2FB00288FD114F4004F18BF4FF05E
:106A7000010962E7C62873D0C72800F0848000F0BF
:106A8000F801C02900F09280C82800F0A680C9282B
:106A90007FF47AAF2846FFF71DFF00F00F0100F0EA
:106AA000F0024B1C43EA023267E7B9F1000F00F035
:106AB0008380002069E700F00300431C022143F4B7
:106AC000802230460B46FFF7AFFB00287FF45CAF17
:106AD00033E72846FFF7FEFE024600283FF454AF96
:106AE00010F0F0017FF450AF30460B46FFF79CFBEF
:106AF00000287FF449AF20E700210D220B4603ACAC
:106B000030460094FFF7BEF92846FFF7E3FE022463
:106B100002060DD500F07F0000FA04FE039B284614
:106B200003EB0E010391FFF7D5FE07340306F1D402
:106B300000F07F0E0EFA04F4039903AB01F5017C1B
:106B40000CEB04020093039238E72846FFF7C2FEDD
:106B500000F00F014A1C00F0F00042EA003268E742
:106B60002846FFF7B7FE00F00F02531C00F0F000BC
:106B700043EA0032032130460B46FFF755FB00285D
:106B80007FF402AFD9E62846FFF7A4FE02460028AC
:106B90003FF4FAAE10F0F0037FF4F6AE3046042175
:106BA000FFF742FB00287FF4EFAEC6E600F00F03CC
:106BB000581C40F42022DDE703AC49460E224B4628
:106BC00030460094FFF75EF9304649460F224B46A7
:106BD0000094FFF777F94846D7E62846FFF77AFE94
:106BE00000F0F00200F00F001032411C41EA0232C6
:106BF000C3E600BF10B5C26C84B0032054688DF8A2
:106C00000C00D37924020832084601A901940292AB
:106C10008DF80D30FFF788FE04B010BD08B5FFF702
:106C200081FE806C08BD00BF08B5FFF77BFEC16C1C
:106C3000C87901EB800303F1080008BD08B500F036
:106C400011FF00BF08B500F00DFF00BF704700BF87
:106C50002DE9F00F00291D46C0F29D800024002D73
:106C6000C0F2948007460D4616469C46002B3DD147
:106C70008A4253D9B2FA82F343B1C3F1200620FA13
:106C800006F501FA03F19A4098402943130CB1FB31
:106C9000F3F697B203FB161107FB06F54FEA104C0B
:106CA0004CEA01418D4209D9891806F1FF3C80F078
:106CB00014818D4240F21181023E8918491BB1FBBB
:106CC000F3F503FB151307FB05F780B240EA034316
:106CD0009F4207D9691E9B1880F005819F4240F2B0
:106CE0000281023D45EA0642002303E08B420AD9B5
:106CF00000231A461046194614B1404261EB410187
:106D0000BDE8F00F7047B3FA83F3002B40F08780A3
:106D10008C4501D38242ECD80122EBE712B901275E
:106D2000B7FBF2F2B2FA82F6002E3AD1891A150CAC
:106D30001FFA82FC0123B1FBF5F705FB17110CFBD1
:106D400007F64FEA104848EA01418E4207D98918F0
:106D500007F1FF3802D28E4200F2DA804746891BE3
:106D6000B1FBF5F605FB16110CFB06FC80B240EA00
:106D70000140844507D9711E821880F0B080944587
:106D800040F2AD80023E46EA0742B3E7E443524296
:106D900063EB430366E7404261EB41014FF0FF3490
:106DA0005DE7B240C6F1200521FA05F320FA05F9A6
:106DB00001FA06F1150CB3FBF5F805FB18371FFABD
:106DC00082FC0CFB08F349EA01094FEA194141EA48
:106DD0000747B040BB420AD9BF1808F1FF3180F025
:106DE0009580BB4240F29280A8F10208BF18FE1ABB
:106DF000B6FBF5F305FB13670CFB03F61FFA89F9E5
:106E000049EA07418E4206D95F1E891878D28E4220
:106E100076D9023B8918891B43EA08438BE7C3F103
:106E2000200122FA01F80CFA03F725FA01FB20FAF7
:106E300001F205FA03F548EA070C4FEA1C48BBFBD0
:106E4000F8F908FB19B71FFA8CFA0AFB09FB15437E
:106E50002A0C42EA0747BB4506FA03F609D917EBA5
:106E60000C0709F1FF324FD2BB454DD9A9F10209F8
:106E70006744CBEB0701B1FBF8F208FB12170AFBE2
:106E800002FAADB245EA07418A4507D9551E11EB12
:106E90000C0137D28A4535D9023A614442EA0942A7
:106EA0001FFA86F84FEA124C08FB0CF7360C95B225
:106EB00008FB05F806FB057506FB0CFC05EB184501
:106EC000AF4288BF0CF5803CCAEB01010CEB1546C4
:106ED000B14212D309D000230CE76646EEE60E4617
:106EE00046EA074206E70D46FCE600FA03F31FFAFE
:106EF00088F808EB0545AB42EDD2013A0023F9E6EC
:106F00003B4688E72A46C9E79146B2E788466EE7DE
:106F1000023F891823E700BF2DE9F0071446054614
:106F20000E46002B3FD18A424AD9B2FA82F343B1CE
:106F3000C3F1200025FA00F201FA03F69C409D40BF
:106F40001643230CB6FBF3F1A0B203FB116C00FB5C
:106F500001F22F0C47EA0C46B24208D94F1E3619EF
:106F600080F0FF80B24240F2FC8002393619B61A36
:106F7000B6FBF3F203FB126300FB02F0ADB245EA8D
:106F80000343984207D9561E1B1980F0EC809842A3
:106F900040F2E980023A42EA0142002310461946D3
:106FA000BDE8F00770478B4243D8B3FA83F4002C56
:106FB00042D18B42234601D382423BD80122EDE7E6
:106FC00012B90127B7FBF2F4B4FA84F2002A40F0B8
:106FD0008A80091B260CA7B20123B1FBF6F006FB41
:106FE000101107FB00F24FEA154C4CEA01418A42AE
:106FF00007D9091900F1FF3C02D28A4200F2D4807D
:107000006046C2EB010CBCFBF6F206FB12C107FBAB
:1070100002F7ADB245EA0145AF4207D9511E2C191E
:1070200080F0A380A74240F2A080023A42EA0042E8
:10703000B4E700231A46B1E7C4F1200703FA04F8C5
:1070400022FA07F321FA07F920FA07FA01FA04F104
:1070500043EA08031E0CB9FBF6FC06FB1C991FFA59
:1070600083F808FB0CF74AEA010A4FEA1A4545EA99
:107070000945AF4202FA04F905D9ED180CF1FF32C7
:10708000C0F087809446EA1BB2FBF6F706FB172692
:1070900008FB07F81FFA8AFA4AEA0641884503D92D
:1070A0007A1EC91870D3174647EA0C42170C1FFA0C
:1070B00089FC0CFB07F695B24FEA19430CFB05FC63
:1070C00003FB056503FB07F305EB1C45AE4288BFD8
:1070D00003F58033C8EB010103EB1543994250D30C
:1070E00047D000235AE79440C2F1200621FA06F562
:1070F00020FA06F901FA02F1260CB5FBF6F806FBB8
:107100001855A7B207FB08F349EA01094FEA1941EC
:1071100041EA054C634500FA02F509D91CEB040C61
:1071200008F1FF323ED263453CD9A8F10208A444DD
:10713000C3EB0C02B2FBF6F306FB132007FB03F2D2
:107140001FFA89F949EA00418A4206D9581E0919ED
:1071500026D28A4224D9023B0919891A43EA0843F4
:107160003BE7394603E7324615E70A4642EA004262
:1071700014E700FA04F01FFA8CF101EB0545A84270
:10718000AFD2013A002309E788458CD9023FC918DC
:107190008AE7AF427FF676AFACF1020CED1872E7EA
:1071A0000346DAE79046C3E70238091929E700BF2A
:1071B000002103E00A4B5B584350043109480A4B55
:1071C00042189A42F6D3094A02E0002342F8043BEF
:1071D000074B9A42F9D3FAF7DBF800F00DF8704745
:1071E000109401080000002004060020080600207A
:1071F000A8620020FEE7000008B562B6F1F724F8A7
:10720000F1F762FEF1F706F8F1F7C2FFF2F7E8FADC
:10721000F3F7FCF9F2F756FDF1F74AFBF9F700FE38
:10722000F7F7C8FBF5F768FFF6F7DAFAF6F72AFD85
:107230000B4B04225A83F6F74BF8F6F7D2FAF6F71F
:107240003FFDF1F7F7F9F1F719FA28B1F2F73AFD36
:10725000F5F752FFF6F716FDF7F7C6FBEBE700BFB1
:1072600000100240014600200246034600F0DAB852
:1072700000210A2200F0C8B838B5084D084C641B3C
:10728000A41006D005EB840555F8043D9847013C51
:10729000FAD1BDE8384002F023B800BF0C940108D1
:1072A000109401080F4B70B41E68054615F8013B99
:1072B00011F8014BF21850781A4600F0030001282B
:1072C00008BF03F1200233195878234600F0030069
:1072D000012808BF04F12003D01A01D1002BE5D109
:1072E00070BC7047FC0500202DE9F00F454C82B0C2
:1072F00024680190084605780646671997F801A0AA
:1073000001301AF0080A0746F5D12D2D5BD02B2D40
:1073100004BF7578B71C002B42D0102B40D0994683
:107320006619BAF1000F76780CBF6FF0004B4FF082
:10733000004BBBFBF9F84FF0000C16F0040F09FBF3
:1073400018BB604613D0303DAB421ADDBCF1FF3FA5
:1073500006D040452ED82BD009FB00504FF0010C31
:1073600017F8015B6619767816F0040FEBD116F06A
:10737000030606D0012E14BF57263726AD1BAB429D
:10738000E4DCBCF1FF3F23D0BAF1000F19D11AB1F0
:10739000BCF1000F13D1116002B0BDE8F00F7047CF
:1073A000302D20D0002BBAD1302D27D00A23B6E7BC
:1073B0005D45D1DD4FF0FF3C17F8015BD2E7791E48
:1073C000E9E74042E3E77578B71C4FF0010AA2E70E
:1073D000BAF1000F019C0CBF6FF000404FF000406D
:1073E00022232360D3E73878782801D05828D9D1D0
:1073F0004FF010097D784B46023791E708239946F4
:107400008EE700BFFC05002030B440F2F853C2F212
:1074100000031D680C46134601462246284630BC30
:10742000FFF762BF2DE9F0410546274884B00468A4
:10743000D4F84801002841D046681F2E1CDD23489F
:1074400010B94FF0FF301EE04FF4C8700391029264
:107450000193AFF300800399029A019B0028F0D0BA
:10746000D4F84861002780E8C000C4F848013E46CF
:10747000C0F88871C0F88C7145B9B31C013640F86A
:1074800023104660002004B0BDE8F081012404FA16
:1074900006F4D0F8887100EB860847EA040C022D48
:1074A0004746C8F88820C0F888C1C8F80831E4D138
:1074B000D0F88C311C43C0F88C41DEE704F5A6708F
:1074C000C4F84801B8E700BFC491010800000000FB
:1074D000024B13B10248FFF7C5BE70470000000021
:1074E000797201082DE9D0438AB006460F4600F0B4
:1074F00077F8384C804694F900308946013336D00D
:107500003046394600F06CFA002830D03046394613
:1075100000220023FDF7F2FF002828D12E4B24780B
:10752000019300230893CDE90267CDE90467002C9D
:1075300022D04FF000094FF00008CFF6F079304626
:10754000394600220023CDE90689FDF7AFFF002868
:1075500022D002239C42009331D0684600F074FA96
:1075600000282CD0089B002B24D1DDE90689404659
:1075700049460AB0BDE8D0834FF6FF794FF0604826
:10758000CCF2EF793046394600220023CDE9068956
:10759000FDF78CFF0028DCD10123022C009313D0CF
:1075A000684600F051FA78B10C4800F04FFACDE986
:1075B0000601D7E700F050FA089B0360D5E700F01A
:1075C0004BFA22230360CDE700F046FA2123036043
:1075D000EAE700BF00060020CC920108D092010823
:1075E0002DE9F04FB1F5801F87B00B460C465FDAEE
:1075F00021F00043034300F0FD800029C0F2AC817C
:1076000000230022C4F25033FDF7E8FC4FF6FF726E
:107610000B46C7F6EF7293426FF035074FDC23F04D
:107620007F4545F6647425F47005C0F209042C19F1
:1076300004F4801484F07E521E1582F4E0020023CC
:1076400042EA0501C3F6F0730022FDF713FBA6F52D
:107650007E76AB1C073E23F47003F6190022022B42
:1076600006EB145482468B4630DC0023FDF71EFFE8
:10767000002800F0C880002C00F077812046FDF73C
:1076800047FCA1A3D3E9002304460D46FDF7A6FC61
:107690009FA3D3E9002306460F4620462946FDF75F
:1076A0009DFC02460B4630463946FDF7E5FA0AE0F6
:1076B0004FF6FF72C7F6EF7200279342AFDD024626
:1076C0000B46FDF7D9FA07B0BDE8F08F4FF08043C5
:1076D000FDF7D2FA02460B4650465946FDF7A8FD83
:1076E000CDE900012046FDF713FCCDE90201DDE9FB
:1076F000000102460B46FDF771FC02460B46804630
:107700008946FDF76BFC84A3D3E9002306460F46A8
:10771000FDF764FC82A3D3E90023FDF7ADFA3246FE
:107720003B46FDF75BFC80A3D3E90023FDF7A4FAF9
:1077300032463B46FDF752FC7DA3D3E90023FDF71B
:107740009BFA42464B46FDF749FC7BA3D3E9002355
:107750008046894630463946FDF740FC78A3D3E998
:107760000023FDF789FA32463B46FDF737FC76A346
:10777000D3E90023FDF780FA32463B46FDF72EFCA5
:1077800002460B4640464946FDF776FA4EF68633EA
:107790004BF65102CFF6F973C0F20602EB18521BFA
:1077A0001343002B06460F4656DD00230022C3F686
:1077B000E07350465946FDF711FC52465B46FDF713
:1077C0000DFC80468946002C6AD132463B46FDF7C7
:1077D00053FADDE90023FDF701FC02460B46404663
:1077E0004946FDF747FA02460B4650465946FDF713
:1077F00041FA68E70021002000220023CCF250313A
:10780000FDF716FD5FE752465B4650465946FDF7C9
:10781000E5FB4FA3D3E9002306460F4650465946E1
:10782000FDF7DCFB0B4600210246C3F6E0710020A9
:10783000FDF720FA02460B4630463946FDF7CEFBEF
:1078400006460F46002C40F093805046594632467B
:107850003B46FDF70FFA36E7002C00F0AD802AA377
:10786000D3E90023DDE90201FDF7B8FB32463B46D0
:107870008046894650465946FDF7FCF9DDE900236C
:10788000FDF7ACFB22A3D3E9002304460D46DDE956
:107890000201FDF7A3FB02460B46204629467EE087
:1078A00019A3D3E90023DDE90201FDF797FB324676
:1078B000CDE904013B4640464946FDF7DDF9DDE9E7
:1078C0000023FDF78BFB12A3D3E9002304460D46EA
:1078D000DDE90201FDF782FB02460B462046294600
:1078E000FDF7CAF902460B4640464946FDF7C2F984
:1078F00052465B46FDF7BEF902460B46DDE9040140
:10790000FDF7B8F9DFE600BF0000E0FE422EE63FDB
:10791000763C7935EF39EA3D44523EDF12F1C23F01
:10792000DE03CB966446C73F599322942449D23F45
:10793000935555555555E53F9FC678D0099AC33F95
:10794000AF788E1DC571CC3F04FA97999999D93FAC
:10795000555555555555D53F02460B46FDF78AF905
:1079600000220023FDF764FCADE600200021AAE61A
:107970002046FDF7CDFA16A3D3E9002304460D46B1
:10798000FDF72CFB14A3D3E900238046894620464B
:107990002946FDF723FB02460B4630463946FDF7E4
:1079A00069F952465B46FDF765F902460B464046CB
:1079B0004946FDF75FF986E632463B465046594652
:1079C000FDF758F9DDE90023FDF708FB0BE700BFE1
:1079D0000000E0FE422EE63F763C7935EF39EA3D85
:1079E0000B4661B1B1F1004F09D04FF6FF72A3F51C
:1079F0008011C7F6DF72914205D804207047002835
:107A0000F3D10220704703F1FE4101F5700191426C
:107A1000F3D94FF6FF72C0F20F02934201D8032050
:107A2000704703F100419142F9D90022C7F6F07284
:107A3000934204D013F5801F01D000207047D0F18D
:107A4000010038BF0020704700207047002100204F
:107A5000C7F6F871704700BF40F2F853C2F2000356
:107A60001868704708B5062000F072F80120F1F799
:107A700027FA00BF0F2AF0B43AD941EA00039B0766
:107A800038D10C46034615462668103D1E606668D0
:107A90005E60A6689E60E6681034DE6010330F2DCD
:107AA000F2D8A2F1100424F00F0402F00F021034F7
:107AB000032A00EB0403214411D90E461D46144647
:107AC00056F8047B043C032C45F8047BF8D8141FBB
:107AD00024F00304043402F0030209191B192AB12B
:107AE00011F8014B013A03F8014BF9D1F0BC704792
:107AF0000346F4E70346F3E71F2938B50C4605466D
:107B000020D8D0F8DC229AB152F8213083B1012B71
:107B10000CD0591C06D00025204642F82450984726
:107B2000284638BD16230360012038BD002038BD2B
:107B3000284600F02BF8224601462846BDE838408A
:107B400000F010B8162303604FF0FF3038BD00BFBF
:107B500040F2F853C2F200031B6801461846FFF7D3
:107B6000CBBF00BF38B5084C002305460846114678
:107B70002360F1F7A6F9431C00D038BD2368002B21
:107B8000FBD02B6038BD00BFA4620020F1F79AB98A
:107B900050C30000881300000180080800000000A6
:107BA000000001000000000000000000C80000000C
:107BB000EF8D2100B81E050000000000000000004D
:107BC00000000000000000000000000000000000B5
:107BD00000000000000000000000000000000000A5
:107BE000524F5200000106524F4C000002064D5306
:107BF00054000003024D565000000407534150004A
:107C00000005074741500000060353544150000748
:107C100003525341500008035347500000090747DF
:107C2000475000000A0353544750000B0352534778
:107C300050000C0352465300000D0353494F0000FF
:107C40000E0747494F00000F0353414300001D0733
:107C500053434F00001E0747434F00001F03434399
:107C60004F0000200341434F0000270355463000DA
:107C7000004007554631000041075546320000429A
:107C80000755463300004307554634000044075566
:107C9000463500004507554636000046075546372D
:107CA0000000470752554E0000810553544F5000C5
:107CB000800042494E00008B0000000000000000E0
:107CC0000000000010000000160000001B00000073
:107CD0002000000023000000270000002A00000010
:107CE0002D000000300000003200000035000000D0
:107CF00037000000390000003B0000003D0000009C
:107D0000400000004100000043000000450000006A
:107D100047000000490000004B0000004C0000003C
:107D20004E00000050000000510000005300000011
:107D300054000000560000005700000059000000E9
:107D40005A0000005B0000005D0000005E000000C3
:107D5000600000006100000062000000630000009D
:107D60006500000066000000670000006800000079
:107D70006A0000006B0000006C0000006D00000055
:107D80006E00000070000000710000007200000032
:107D90007300000074000000750000007600000011
:107DA0007700000078000000790000007A000000F1
:107DB0007B0000007C0000007D0000007E000000D1
:107DC00080000000800000008100000082000000B0
:107DD0008300000084000000850000008600000091
:107DE0008700000088000000890000008A00000071
:107DF0008B0000008C0000008D0000008E00000051
:107E00008F00000090000000900000009100000032
:107E10009200000093000000940000009500000014
:107E200096000000960000009700000098000000F7
:107E3000990000009A0000009B0000009B000000D9
:107E40009C0000009D0000009E0000009F000000BC
:107E5000A0000000A0000000A1000000A20000009F
:107E6000A3000000A3000000A4000000A500000083
:107E7000A6000000A7000000A7000000A800000066
:107E8000A9000000AA000000AA000000AB0000004A
:107E9000AC000000AD000000AD000000AE0000002E
:107EA000AF000000B0000000B0000000B100000012
:107EB000B2000000B2000000B3000000B4000000F7
:107EC000B5000000B5000000B6000000B7000000DB
:107ED000B7000000B8000000B9000000B9000000C1
:107EE000BA000000BB000000BB000000BC000000A6
:107EF000BD000000BD000000BE000000BF0000008B
:107F0000C0000000C0000000C1000000C10000006F
:107F1000C2000000C3000000C3000000C400000055
:107F2000C5000000C5000000C6000000C70000003A
:107F3000C7000000C8000000C9000000C900000020
:107F4000CA000000CB000000CB000000CC00000005
:107F5000CC000000CD000000CE000000CE000000EC
:107F6000CF000000D0000000D0000000D1000000D1
:107F7000D1000000D2000000D3000000D3000000B8
:107F8000D4000000D4000000D5000000D60000009E
:107F9000D6000000D7000000D7000000D800000085
:107FA000D9000000D9000000DA000000DA0000006B
:107FB000DB000000DB000000DC000000DD00000052
:107FC000DD000000DE000000DE000000DF00000039
:107FD000E0000000E0000000E1000000E10000001F
:107FE000E2000000E2000000E3000000E300000007
:107FF000E4000000E5000000E5000000E6000000ED
:10800000E6000000E7000000E7000000E8000000D4
:10801000E8000000E9000000EA000000EA000000BB
:10802000EB000000EB000000EC000000EC000000A2
:10803000ED000000ED000000EE000000EE0000008A
:10804000EF000000F0000000F0000000F100000070
:10805000F1000000F2000000F2000000F300000058
:10806000F3000000F4000000F4000000F500000040
:10807000F5000000F6000000F6000000F700000028
:10808000F7000000F8000000F8000000F900000010
:10809000F9000000FA000000FA000000FB000000F8
:1080A000FB000000FC000000FC000000FD000000E0
:1080B000FD000000FE000000FE000000FF000000C8
:1080C00001F0010002F0010004F0010005F00100E0
:1080D00007F0010008F001000AF001000BF00100B8
:1080E0000DF001000EF0010010EE010011EE010094
:1080F00013EE010015EE010016EE010018EE01006E
:1081000019EE01001BEE01001CEC01001EEC010049
:108110001FEC010021EC010022EC010024EA010027
:1081200025EA010027EA010028EA01002AE8010007
:108130002BE801002DE801002EE8010030E60100E7
:1081400031E6010033E6010034E4010036E40100C9
:1081500037E4010039E201003AE201003CE20100AB
:108160003DE001003EE0010040E0010041DE010091
:1081700043DE010044DC010046DC010047DC010075
:1081800049DA01004ADA01004CD801004DD801005B
:108190004FD6010050D6010051D4010053D4010044
:1081A00054D2010056D2010057D0010059D001002D
:1081B0005ACE01005BCE01005DCC01005ECA010019
:1081C00060CA010061C8010062C8010064C6010004
:1081D00065C4010067C4010068C2010069C20100F2
:1081E0006BC001006CBE01006DBE01006FBC0100E0
:1081F00070BA010072B8010073B8010074B60100D2
:1082000076B4010077B4010078B201007AB00100C1
:108210007BAE01007CAE01007EAC01007FAA0100B4
:1082200080A8010081A8010083A6010084A40100A8
:1082300085A2010087A00100889E0100899E01009F
:108240008A9C01008C9A01008D9801008E96010095
:108250008F9401009192010092920100939001008D
:10826000948E0100968C0100978A01009888010085
:10827000998601009A8401009C8201009D80010082
:108280009E7E01009F7C0100A07A0100A178010080
:10829000A3760100A4740100A5720100A67001007C
:1082A000A76E0100A86C0100A96A0100AA6801007C
:1082B000AC660100AD640100AE620100AF60010078
:1082C000B05E0100B15C0100B25A0100B358010078
:1082D000B4540100B5520100B6500100B74E010080
:1082E000B84C0100B94A0100BA480100BB46010080
:1082F000BC420100BD400100BE3E0100BF3C010088
:10830000C03A0100C1380100C2340100C33201008B
:10831000C4300100C52E0100C62C0100C728010091
:10832000C8260100C9240100C9220100CA1E01009B
:10833000CB1C0100CC1A0100CD180100CE140100A5
:10834000CF120100CF100100D00E0100D10A0100B0
:10835000D2080100D3060100D4020100D4000100BC
:10836000D5FE0000D6FC0000D7F80000D7F60000CC
:10837000D8F40000D9F00000DAEE0000DAEC0000DA
:10838000DBE80000DCE60000DCE40000DDE00000EB
:10839000DEDE0000DFDA0000DFD80000E0D60000FB
:1083A000E1D20000E1D00000E2CE0000E2CA00000D
:1083B000E3C80000E4C40000E4C20000E5C000001F
:1083C000E5BC0000E6BA0000E7B60000E7B4000034
:1083D000E8B20000E8AE0000E9AC0000E9A8000047
:1083E000EAA60000EAA20000EBA00000EB9E00005D
:1083F000EC9A0000EC980000ED940000ED92000073
:10840000EE8E0000EE8C0000EE880000EF8600008B
:10841000EF820000F0800000F07C0000F07A0000A5
:10842000F1780000F1740000F1720000F26E0000BB
:10843000F26C0000F2680000F3660000F3620000D6
:10844000F3600000F45C0000F45A0000F4560000F1
:10845000F4540000F5500000F54E0000F54A00000D
:10846000F5480000F6440000F6420000F63E000029
:10847000F63C0000F6380000F7360000F732000046
:10848000F7300000F72C0000F72A0000F726000064
:10849000F7220000F7200000F81C0000F81A000086
:1084A000F8160000F8140000F8100000F80E0000A4
:1084B000F80A0000F8080000F8040000F8020000C4
:1084C000F8020200F8040200F8080200F80A0200AC
:1084D000F80E0200F8100200F8140200F81602006C
:1084E000F81A0200F81C0200F7200200F72202002E
:1084F000F7260200F72A0200F72C0200F7300200EC
:10850000F7320200F7360200F6380200F63C0200AD
:10851000F63E0200F6420200F6440200F548020070
:10852000F54A0200F54E0200F5500200F454020034
:10853000F4560200F45A0200F45C0200F3600200F8
:10854000F3620200F3660200F2680200F26C0200BD
:10855000F26E0200F1720200F1740200F178020082
:10856000F07A0200F07C0200F0800200EF8202004C
:10857000EF860200EE880200EE8C0200EE8E020012
:10858000ED920200ED940200EC980200EC9A0200D9
:10859000EB9E0200EBA00200EAA20200EAA60200A3
:1085A000E9A80200E9AC0200E8AE0200E8B202006D
:1085B000E7B40200E7B60200E6BA0200E5BC02003A
:1085C000E5C00200E4C20200E4C40200E3C8020005
:1085D000E2CA0200E2CE0200E1D00200E1D20200D3
:1085E000E0D60200DFD80200DFDA0200DEDE0200A1
:1085F000DDE00200DCE40200DCE60200DBE8020071
:10860000DAEC0200DAEE0200D9F00200D8F402003F
:10861000D7F60200D7F80200D6FC0200D5FE020011
:10862000D4000300D4020300D3060300D2080300E1
:10863000D10A0300D00E0300CF100300CF120300B5
:10864000CE140300CD180300CC1A0300CB1C03008A
:10865000CA1E0300C9220300C9240300C826030060
:10866000C7280300C62C0300C52E0300C430030036
:10867000C3320300C2340300C1380300C03A030010
:10868000BF3C0300BE3E0300BD400300BC420300EC
:10869000BB460300BA480300B94A0300B84C0300C4
:1086A000B74E0300B6500300B5520300B4540300A4
:1086B000B3580300B25A0300B15C0300B05E03007C
:1086C000AF600300AE620300AD640300AC6603005C
:1086D000AA680300A96A0300A86C0300A76E030040
:1086E000A6700300A5720300A4740300A376030020
:1086F000A1780300A07A03009F7C03009E7E030004
:108700009D8003009C8203009A84030099860300E5
:1087100098880300978A0300968C0300948E0300C8
:108720009390030092920300919203008F940300B0
:108730008E9603008D9803008C9A03008A9C030098
:10874000899E0300889E030087A0030085A2030082
:1087500084A4030083A6030081A8030080A803006B
:108760007FAA03007EAC03007CAE03007BAE030057
:108770007AB0030078B2030077B4030076B4030044
:1087800074B6030073B8030072B8030070BA030034
:108790006FBC03006DBE03006CBE03006BC0030022
:1087A00069C2030068C2030067C4030065C4030014
:1087B00064C6030062C8030061C8030060CA030006
:1087C0005ECA03005DCC03005BCE03005ACE0300FB
:1087D00059D0030057D0030056D2030054D20300EF
:1087E00053D4030051D4030050D603004FD60300E6
:1087F0004DD803004CD803004ADA030049DA0300DD
:1088000047DC030046DC030044DC030043DE0300D6
:1088100041DE030040E003003EE003003DE00300D2
:108820003CE203003AE2030039E2030037E40300CC
:1088300036E4030034E4030033E6030031E60300CA
:1088400030E603002EE803002DE803002BE80300C8
:108850002AE8030028EA030027EA030025EA0300C8
:1088600024EA030022EC030021EC03001FEC0300C8
:108870001EEC03001CEC03001BEE030019EE0300CA
:1088800018EE030016EE030015EE030013EE0300CE
:1088900011EE030010EE03000EF003000DF00300D4
:1088A0000BF003000AF0030008F0030007F00300D8
:1088B00005F0030004F0030002F0030001F00300E0
:1088C00001F1030002F1030004F1030005F10300CC
:1088D00007F1030008F103000AF103000BF10300A4
:1088E0000DF103000EF1030010EF030011EF030080
:1088F00013EF030015EF030016EF030018EF03005A
:1089000019EF03001BEF03001CED03001EED030035
:108910001FED030021ED030022ED030024EB030013
:1089200025EB030027EB030028EB03002AE90300F3
:108930002BE903002DE903002EE9030030E70300D3
:1089400031E7030033E7030034E5030036E50300B5
:1089500037E5030039E303003AE303003CE3030097
:108960003DE103003EE1030040E1030041DF03007D
:1089700043DF030044DD030046DD030047DD030061
:1089800049DB03004ADB03004CD903004DD9030047
:108990004FD7030050D7030051D5030053D5030030
:1089A00054D3030056D3030057D1030059D1030019
:1089B0005ACF03005BCF03005DCD03005ECB030005
:1089C00060CB030061C9030062C9030064C70300F0
:1089D00065C5030067C5030068C3030069C30300DE
:1089E0006BC103006CBF03006DBF03006FBD0300CC
:1089F00070BB030072B9030073B9030074B70300BE
:108A000076B5030077B5030078B303007AB10300AD
:108A10007BAF03007CAF03007EAD03007FAB0300A0
:108A200080A9030081A9030083A7030084A5030094
:108A300085A3030087A10300889F0300899F03008B
:108A40008A9D03008C9B03008D9903008E97030081
:108A50008F95030091930300929303009391030079
:108A6000948F0300968D0300978B03009889030071
:108A7000998703009A8503009C8303009D8103006E
:108A80009E7F03009F7D0300A07B0300A17903006C
:108A9000A3770300A4750300A5730300A671030068
:108AA000A76F0300A86D0300A96B0300AA69030068
:108AB000AC670300AD650300AE630300AF61030064
:108AC000B05F0300B15D0300B25B0300B359030064
:108AD000B4550300B5530300B6510300B74F03006C
:108AE000B84D0300B94B0300BA490300BB4703006C
:108AF000BC430300BD410300BE3F0300BF3D030074
:108B0000C03B0300C1390300C2350300C333030077
:108B1000C4310300C52F0300C62D0300C72903007D
:108B2000C8270300C9250300C9230300CA1F030087
:108B3000CB1D0300CC1B0300CD190300CE15030091
:108B4000CF130300CF110300D00F0300D10B03009C
:108B5000D2090300D3070300D4030300D4010300A8
:108B6000D5FF0200D6FD0200D7F90200D7F70200B8
:108B7000D8F50200D9F10200DAEF0200DAED0200C6
:108B8000DBE90200DCE70200DCE50200DDE10200D7
:108B9000DEDF0200DFDB0200DFD90200E0D70200E7
:108BA000E1D30200E1D10200E2CF0200E2CB0200F9
:108BB000E3C90200E4C50200E4C30200E5C102000B
:108BC000E5BD0200E6BB0200E7B70200E7B5020020
:108BD000E8B30200E8AF0200E9AD0200E9A9020033
:108BE000EAA70200EAA30200EBA10200EB9F020049
:108BF000EC9B0200EC990200ED950200ED9302005F
:108C0000EE8F0200EE8D0200EE890200EF87020077
:108C1000EF830200F0810200F07D0200F07B020091
:108C2000F1790200F1750200F1730200F26F0200A7
:108C3000F26D0200F2690200F3670200F3630200C2
:108C4000F3610200F45D0200F45B0200F4570200DD
:108C5000F4550200F5510200F54F0200F54B0200F9
:108C6000F5490200F6450200F6430200F63F020015
:108C7000F63D0200F6390200F7370200F733020032
:108C8000F7310200F72D0200F72B0200F727020050
:108C9000F7230200F7210200F81D0200F81B020072
:108CA000F8170200F8150200F8110200F80F020090
:108CB000F80B0200F8090200F8050200F8030200B0
:108CC000F8030000F8050000F8090000F80B0000A8
:108CD000F80F0000F8110000F8150000F817000068
:108CE000F81B0000F81D0000F7210000F72300002A
:108CF000F7270000F72B0000F72D0000F7310000E8
:108D0000F7330000F7370000F6390000F63D0000A9
:108D1000F63F0000F6430000F6450000F54900006C
:108D2000F54B0000F54F0000F5510000F455000030
:108D3000F4570000F45B0000F45D0000F3610000F4
:108D4000F3630000F3670000F2690000F26D0000B9
:108D5000F26F0000F1730000F1750000F17900007E
:108D6000F07B0000F07D0000F0810000EF83000048
:108D7000EF870000EE890000EE8D0000EE8F00000E
:108D8000ED930000ED950000EC990000EC9B0000D5
:108D9000EB9F0000EBA10000EAA30000EAA700009F
:108DA000E9A90000E9AD0000E8AF0000E8B3000069
:108DB000E7B50000E7B70000E6BB0000E5BD000036
:108DC000E5C10000E4C30000E4C50000E3C9000001
:108DD000E2CB0000E2CF0000E1D10000E1D30000CF
:108DE000E0D70000DFD90000DFDB0000DEDF00009D
:108DF000DDE10000DCE50000DCE70000DBE900006D
:108E0000DAED0000DAEF0000D9F10000D8F500003B
:108E1000D7F70000D7F90000D6FD0000D5FF00000D
:108E2000D4010100D4030100D3070100D2090100DD
:108E3000D10B0100D00F0100CF110100CF130100B1
:108E4000CE150100CD190100CC1B0100CB1D010086
:108E5000CA1F0100C9230100C9250100C82701005C
:108E6000C7290100C62D0100C52F0100C431010032
:108E7000C3330100C2350100C1390100C03B01000C
:108E8000BF3D0100BE3F0100BD410100BC430100E8
:108E9000BB470100BA490100B94B0100B84D0100C0
:108EA000B74F0100B6510100B5530100B4550100A0
:108EB000B3590100B25B0100B15D0100B05F010078
:108EC000AF610100AE630100AD650100AC67010058
:108ED000AA690100A96B0100A86D0100A76F01003C
:108EE000A6710100A5730100A4750100A37701001C
:108EF000A1790100A07B01009F7D01009E7F010000
:108F00009D8101009C8301009A85010099870100E1
:108F100098890100978B0100968D0100948F0100C4
:108F20009391010092930100919301008F950100AC
:108F30008E9701008D9901008C9B01008A9D010094
:108F4000899F0100889F010087A1010085A301007E
:108F500084A5010083A7010081A9010080A9010067
:108F60007FAB01007EAD01007CAF01007BAF010053
:108F70007AB1010078B3010077B5010076B5010040
:108F800074B7010073B9010072B9010070BB010030
:108F90006FBD01006DBF01006CBF01006BC101001E
:108FA00069C3010068C3010067C5010065C5010010
:108FB00064C7010062C9010061C9010060CB010002
:108FC0005ECB01005DCD01005BCF01005ACF0100F7
:108FD00059D1010057D1010056D3010054D30100EB
:108FE00053D5010051D5010050D701004FD70100E2
:108FF0004DD901004CD901004ADB010049DB0100D9
:1090000047DD010046DD010044DD010043DF0100D2
:1090100041DF010040E101003EE101003DE10100CE
:109020003CE301003AE3010039E3010037E50100C8
:1090300036E5010034E5010033E7010031E70100C6
:1090400030E701002EE901002DE901002BE90100C4
:109050002AE9010028EB010027EB010025EB0100C4
:1090600024EB010022ED010021ED01001FED0100C4
:109070001EED01001CED01001BEF010019EF0100C6
:1090800018EF010016EF010015EF010013EF0100CA
:1090900011EF010010EF01000EF101000DF10100D0
:1090A0000BF101000AF1010008F1010007F10100D4
:1090B00005F1010004F1010002F1010001F10100DC
:1090C000E0C0020060C0030060C10300E0C1020014
:1090D000E0C1000060C1010060C00100E0C000000C
:1090E000E0C0020060C0030060C10300E0C10200F4
:1090F000E0C1000060C1010060C00100E0C00000EC
:10910000B4690100B4680100B4680300B4690300E5
:10911000B4690100B4680100B4680300B4690300D5
:10912000B4690100B4680100B4680300B4690300C5
:10913000B4690100B4680100B4680300B4690300B5
:10914000020102313331305631303700564350205E
:10915000496E746572666163650056435020436FC3
:109160006E66696700544D43313331300054726983
:109170006E616D6963204D6F74696F6E20436F6E11
:1091800074726F6C00544D434D2D313331302028B3
:109190007669727475616C20434F4D2900414253CA
:1091A0000052454C00434F4F5244005354415254D7
:1091B0000053544F50005354415455530000000085
:1091C00043000000D001002000202020202020208B
:1091D0002020282828282820202020202020202067
:1091E0002020202020202020208810101010101077
:1091F00010101010101010101004040404040404C3
:10920000040404101010101010104141414141415C
:10921000010101010101010101010101010101013E
:10922000010101011010101010104242424242424E
:10923000020202020202020202020202020202020E
:1092400002020202101010102000000000000000B6
:10925000000000000000000000000000000000000E
:1092600000000000000000000000000000000000FE
:1092700000000000000000000000000000000000EE
:1092800000000000000000000000000000000000DE
:1092900000000000000000000000000000000000CE
:1092A00000000000000000000000000000000000BE
:1092B00000000000000000000000000000000000AE
:1092C0000000000000000000000000006C6F67005C
:1092D00000000000F8B500BFF8BC08BC9E4670470F
:0C92E000F8B500BFF8BC08BC9E46704703
:1092EC00A1B20181B0B0AE010000000008B1018153
:1092FC00B0B000840000000008B10181B0B000845F
:10930C000000000008B10181B0B000840000000032
:10931C0064C8FF7FB03784808CC8FF7FAB08B180F6
:10932C00B0C8FF7F010000002CC9FF7FB0A90280EC
:10933C00ECC9FF7FB0B0A8803CCAFF7FA4FFFF7FC1
:10934C0008CBFF7FA908B18030CBFF7F0100000064
:10935C00ACCBFF7FB0AF0A80B8CEFF7F010000001E
:10936C00BCCEFF7FAE3F278068D2FF7F010000009C
:10937C0064D2FF7FAB10B280BCD2FF7F0100000033
:10938C00C8D2FF7FA908B180FCD2FF7F010000008A
:10939C0008D3FF7F58FFFF7F10D3FF7FAB26B2802F
:1093AC007CD3FF7F0100000054D5FF7FB0A8038061
:1093BC0068D5FF7F0100000064D5FF7FB0AD04804D
:1093CC0028D8FF7FB0A8038048D8FF7F2CFFFF7FF1
:1093DC004CD8FF7F30FFFF7F58D8FF7F0100000083
:1093EC0064D8FF7FB0B0A78024DBFF7FB0B0A6802D
:0893FC00B4DDFF7F0100000059
:08940400D1740108AD810008DC
:04940C00898100084A
:109410004391010800010200000800000100000063
:10942000020000000000000000000000000000003A
:10943000000000000000000000000000000000002C
:10944000000000000000000000000000000000001C
:10945000000000001201100202000040D0162B078D
:1094600000020102030104030904000000C201001C
:109470000000080057A3000865A30008F9A300082E
:1094800015A40008DDA30008C1A30008A5A30008D7
:1094900049A300084BA300084DA300084FA30008F0
:1094A00051A3000853A3000855A300080A060002B0
:1094B000000000400100000071A3000875A300082F
:1094C00031A4000879A300087DA30008E803000088
:1094D00000040000D007000000080000C4090000DC
:1094E000A00F00000010000088130000401F0000C3
:1094F000002000001027000000400000204E000067
:10950000007D000000800000409C00000000010081
:10951000FFFFFFFF000E2707000000000000000013
:109520000102030406070809000000000102030409
:1095300001020304060708092C010020F133010889
:109540003D330108F332010863320108C5320108D6
:1095500047320108313201087332010881320108B3
:109560008F320108A532010809024300020100C040
:109570003209040000010202010005240010010567
:1095800024010001042402020524060001070582CB
:10959000030800FF09040100020A0000000705019A
:1095A000024000000705810240000000FF000000AB
:1095B00071360108493601088535010800000000B0
:1095C000C5360108F536010855350108D5340108BE
:1095D0000000000000000000C93401080000000085
:1095E00000000000BC040020240500208C050020A1
:1095F000000000000000000000000000000000006B
:10960000000000000000000000000000000000005A
:1096100000000000C09101080000000000000000F0
:10962000000000000000000000000000000000003A
:10963000000000000000000000000000000000002A
:10964000000000000000000000000000000000001A
:10965000000000000000000000000000000000000A
:1096600000000000000000000000000000000000FA
:1096700000000000000000000000000000000000EA
:1096800000000000000000000100000000000000D9
:109690000E33CDAB34126DE6ECDE05000B0000009E
:1096A00000000000000000000000000000000000BA
:1096B00000000000000000000000000000000000AA
:1096C000000000000000000000000000000000009A
:1096D000000000000000000000000000000000008A
:109A00000000000000000000D0010020C891010803
:049A10000100000051
:04000005080171B1CC
:00000001FF
